:020000040000FA
:10000000000204000000000096720000A2720000CE
:10001000AE720000BA720000C6720000D272000018
:10002000DE720000F6720000EA720000EA72000060
:10003000EA720000EA720000EA720000EA72000050
:10004000EA72000066740000EA720000EA720000C2
:10005000EA720000906E0000EA720000EA7200008E
:10006000EA720000EA720000EA720000EA72000020
:10007000EA720000EA720000EA720000EA72000010
:10008000EA720000EA720000EA720000EA72000000
:10009000EA720000EA720000EA720000EA720000F0
:1000A000EA7200004A710000EA720000EA72000081
:1000B000EA720000EA720000EA720000EA720000D0
:1000C000EA720000EA720000EA720000EA720000C0
:1000D000EA720000EA720000EA720000EA720000B0
:1000E000EA720000EA720000EA720000EA720000A0
:1000F000EA720000EA720000EA720000EA72000090
:10010000EA720000EA720000EA720000EA7200007F
:10011000EA720000EA720000EA720000EA7200006F
:10012000EA720000EA720000EA72000060710000EA
:1001300066710000EA720000EA720000EA720000D4
:10014000EA720000EA720000EA720000EA7200003F
:10015000EA720000EA720000EA720000EA7200002F
:10016000EA720000EA720000EA7200009871000072
:100170006C71000082710000EA720000EA720000F7
:10018000EA720000EA720000EA720000EA720000FF
:10019000EA720000EA720000EA720000EA720000EF
:1001A000EA720000EA720000EA720000EA720000DF
:1001B000EA720000EA720000EA720000EA720000CF
:1001C000EA720000EA720000EA720000EA720000BF
:1001D000EA720000EA720000EA720000EA720000AF
:1001E000EA720000EA720000EA720000EA7200009F
:1001F000EA720000EA720000EA720000EA7200008F
:10020000EA720000EA720000EA720000EA7200007E
:10021000EA720000EA720000EA720000EA7200006E
:10022000EA720000EA720000EA720000EA7200005E
:10023000EA720000EA720000EA720000EA7200004E
:10024000EA720000EA720000EA720000EA7200003E
:10025000EA720000EA720000EA720000EA7200002E
:10026000EA720000EA720000FFFFFF00FFFFFF00DC
:10027000FFFFFF00FFFFFF00FFFFFF00FFFFFF008A
:10028000FFFFFF00FFFFFF00FFFFFF00FFFFFF007A
:10029000FFFFFF00FFFFFF00FFFFFF00FFFFFF006A
:1002A000FFFFFF00FFFFFF00FFFFFF00FFFFFF005A
:1002B000FFFFFF00FFFFFF00FFFFFF00FFFFFF004A
:1002C000FFFFFF00FFFFFF00FFFFFF00FFFFFF003A
:1002D000FFFFFF00FFFFFF00FFFFFF00FFFFFF002A
:1002E000FFFFFF00FFFFFF00FFFFFF00FFFFFF001A
:1002F000FFFFFF00FFFFFF00FFFFFF00FFFFFF000A
:10030000FFFFFF00FFFFFF00FFFFFF00FFFFFF00F9
:10031000FFFFFF00FFFFFF00FFFFFF00FFFFFF00E9
:10032000FFFFFF00FFFFFF00FFFFFF00FFFFFF00D9
:10033000FFFFFF00FFFFFF00FFFFFF00FFFFFF00C9
:10034000FFFFFF00FFFFFF00FFFFFF00FFFFFF00B9
:10035000FFFFFF00FFFFFF00FFFFFF00FFFFFF00A9
:10036000FFFFFF00FFFFFF00FFFFFF00FFFFFF0099
:10037000FFFFFF00FFFFFF00FFFFFF00FFFFFF0089
:10038000FFFFFF00FFFFFF00FFFFFF00FFFFFF0079
:10039000FFFFFF00FFFFFF00FFFFFF00FFFFFF0069
:1003A000FFFFFF00FFFFFF00FFFFFF00FFFFFF0059
:1003B000FFFFFF00FFFFFF00FFFFFF00FFFFFF0049
:1003C000FFFFFF00FFFFFF00FFFFFF00FFFFFF0039
:1003D000FFFFFF00FFFFFF00FFFFFF00FFFFFF0029
:1003E000FFFFFF00FFFFFF00FFFFFF00FFFFFF0019
:1003F000FFFFFF00FFFFFF00FFFFFF00FFFFFF0009
:10040000AFEC2100E0F221000001880000000000B4
:10041000F26202000000000000002000407088002E
:10042000000020005070880000002000307088001C
:1004300000002000607088000000200070708800BC
:10044000000020000070880000002000207088005C
:1004500000002000C070880000002000D0708800DC
:1004600000002000E070880000002000F07088008C
:10047000F00F20008070880000002000A07088002D
:1004800000002000407188000000200050718800AA
:10049000000020006071880000002000707188005A
:1004A000E0012F000071880000002000207188000A
:1004B00000002000C071880000002000D07188007A
:1004C00000032300B071880000002000E071880064
:1004D00000002000F0718800000024008071880076
:1004E00080032300A0718800000020004072880073
:1004F0000000200050728800000020006072880018
:100500000000200070728800200020000072880027
:10051000100820002072880000002000C0728800AF
:1005200000002000D072880000002300B072880014
:1005300000002000E0728800000222008072880023
:1005400000012100A0728800000020004073880094
:1005500000002000507388003000240030738800B1
:100560000000200060738800000020007073880085
:1005700020082000007388001000200020738800ED
:1005800000002000C0738800F0CF2000D0738800E6
:1005900000002000B073880000002000E073880095
:1005A000F0CF20008073880000002000A073880036
:1005B000000020004074880000002700507488006C
:1005C000F00F200030748800000020006074880064
:1005D00000002700007488000000280020748800B4
:1005E00000002000C074880000002000D074880043
:1005F00000002000B074880000002000E074880033
:10060000000022008074880000002C00A074880084
:1006100010032000203688001005200030368800A6
:10062000D0062000B036880010072000C0368800B1
:100630000030200040348800001020006034880022
:1006400000B02100B034880000D02100C034880000
:1006500010302300103A880020002000203A880043
:10066000A0082000303A880075AEA80075CEA8001A
:1006700000802A0000118800004C22001011880020
:10068000701C20004011880000802A008011880022
:10069000004C22009011880060022000C0118800E8
:1006A00060802A008012880000402000901288009C
:1006B000701C2000C012880060802A00801588000D
:1006C000004C200090158800701C2000C015880088
:1006D000158EA80004CEA900E008210050848800EF
:1006E00060848800A01B2100B08D8800C08D880028
:1006F000E0212100D0908800E09088006015210062
:10070000908A8800A08A8800208F210070C7880006
:1007100080C788000002280080088800504420001C
:1007200060088800DE38EF00E438EF00F0FF2F00AB
:1007300030C7880040C788006A30EF000230EF0001
:100740006988A90069A8A90069C8A8006888A800E4
:1007500068A8A90068C8A8004388A80043A8A90001
:1007600043C8A8001E6202000000000065CEA80079
:100770001E620200000000000004200080630200EE
:100780000000000000032000FE62020000000000E4
:1007900070082000FE6202000000000070002000CF
:1007A000FE6202000000000070022000FE620200F3
:1007B00000000000F0022000FE62020000000000C5
:1007C000F00E2000FE620200000000008002200007
:1007D000FE6202000000000000002000FE62020035
:1007E00000000000400420008063020000000000C0
:1007F00000002000FE620200000000000000200057
:10080000FE62020000000000000F2000FE620200F5
:100810000000000000082000FE620200000000004E
:1008200050022000FE62020000000000000F2000C5
:10083000FE6202000000000000002000FE620200D4
:1008400000000000B0042000FE6202000000000072
:1008500000002000FE6202000000000000002000F6
:10086000FE62020000000000A0052000806302007C
:100870000000000000002000FE62020000000000F6
:10088000B00520008063020000000000100020007E
:10089000FE6202000000000080052000806302006C
:1008A0000000000060052000FE6202000000000061
:1008B0005864020000000000600420008063020011
:1008C0000000000000002000FE62020000000000A6
:1008D00000002000FE62020000000000D0052000A1
:1008E000806302000000000040002000FE62020061
:1008F0000000000070002000FE6202000000000006
:10090000900520008063020000000000C004200069
:100910008063020000000000154EA80015EEA9003B
:1009200015CEA90015AEA8000000000000000000D0
:1009300000000000000000000000000000000000B7
:1009400000000000152EA8008662020000000000D2
:1009500086620200000000008662020000000000C3
:100960008662020000000000C46102000000000076
:1009700086620200000000008662020000000000A3
:100980008662020000000000866202000000000093
:1009900015EEA80015CEA80015AEA80000000000B6
:1009A0000000000000000000000000000000000047
:1009B0000000000000000000152EA8008662020062
:1009C0000000000086620200000000008662020053
:1009D000000000008662020000000000C461020006
:1009E0000000000086620200000000008662020033
:1009F0000000000086620200000000008662020023
:100A00000000000015EEA90015CEA90015AEA90042
:100A100000000000000000000000000000000000D6
:100A2000000000000000000000000000152EA800DB
:100A300086620200000000008662020000000000E2
:100A400086620200000000008662020000000000D2
:100A5000C461020000000000866202000000000085
:100A600086620200000000008662020000000000B2
:100A70008662020000000000156EA9000000000060
:100A80000000000000000000000000000000000066
:100A90000000000000000000800E2000E660020060
:100AA0000000000000002000E660020000000000DE
:100AB00000002000E66002000000000000002000AE
:100AC000E66002000000000000002000E660020076
:100AD0000000000000002000E660020000000000AE
:100AE00000002000E660020000000000000020007E
:100AF000E6600200000000003A6102000000000011
:100B0000156EA800000000000000000000000000BA
:100B100000000000000000000000000000000000D5
:100B2000A10A20000100E1004220AE009E05040061
:100B3000000000000007040000000000156EA9007E
:100B400000000000000000000000000000000000A5
:100B5000000000000000000000000000800E2000E7
:100B6000E66002000000000000002000E6600200D5
:100B70000000000000002000E6600200000000000D
:100B800000082000E66002000000000000002000D5
:100B9000E66002000000000000002000E6600200A5
:100BA0000000000000002000E660020000000000DD
:100BB00000002000E6600200000000003A61020030
:100BC00000000000000278003A610200000000000E
:100BD0004800DD0004004000F08088003A61020017
:100BE00000000000000278003A61020000000000EE
:100BF0004800DD0004004000008188003A610200E6
:100C000000000000000278003A61020000000000CD
:100C10004800DD0004004000608388003A61020063
:100C200000000000000278003A61020000000000AD
:100C30004800DD0004004000708388003A61020033
:100C400000000000000278003A610200000000008D
:100C50004800DD0004004000808388003A61020003
:100C600000000000000278003A610200000000006D
:100C70004800DD0004004000908388003A610200D3
:100C800000000000000278003A610200000000004D
:100C90004800DD0004004000A08388003A610200A3
:100CA00000000000000278003A610200000000002D
:100CB0004800DD00040040000105200081005000D4
:100CC0004220AF0072060400000000003104200042
:100CD000810050004220AF007206040000000000B6
:100CE00000052000B08388003A6102000000000087
:100CF000000278003A610200000000004800DD00B8
:100D000004004000C08388003A6102000000000037
:100D1000000278003A610200000000004800DD0097
:100D200004004000E08088003A61020000000000FA
:100D3000000278003A610200000000004800DD0077
:100D400004004000E08388003A61020000000000D7
:100D5000000278003A610200000000004800DD0057
:100D600004004000F08388003A61020000000000A7
:100D7000000278003A610200000000004800DD0037
:100D80000400400091838000810050004200AF00C9
:100D90000000EB00008488003A61020000000000BF
:100DA000000278003A610200000000004800DD0007
:100DB00004004000909488003A61020000000000A6
:100DC000000278003A610200000000004800DD00E7
:100DD00004004000A0948800156EA80000000000E8
:100DE0000000000000000000000000000000000003
:100DF0000000000000000000620804000000000085
:100E0000156EA900000000000000000000000000B6
:100E100000000000000000000000000000000000D2
:100E2000800E2000E66002000000000000002000AC
:100E3000E66002000000000010002000E6600200F2
:100E40000000000000002000E6600200000000003A
:100E500000002000E660020000000000000020000A
:100E6000E66002000000000000002000E6600200D2
:100E70000000000000002000E6600200000000000A
:100E80003A61020000000000000278003A610200AE
:100E9000000000004800DD0004004000F0808800F1
:100EA0003A61020000000000000278003A6102008E
:100EB000000000004800DD000400400000818800C0
:100EC0003A61020000000000000278003A6102006E
:100ED000000000004800DD0004004000608388003E
:100EE0003A61020000000000000278003A6102004E
:100EF000000000004800DD0004004000708388000E
:100F00003A61020000000000000278003A6102002D
:100F1000000000004800DD000400400080838800DD
:100F20003A61020000000000000278003A6102000D
:100F3000000000004800DD000400400090838800AD
:100F40003A61020000000000000278003A610200ED
:100F5000000000004800DD0004004000A08388007D
:100F60003A61020000000000000278003A610200CD
:100F7000000000004800DD000400400001052000E2
:100F8000810050004220AF00D407040000000000A0
:100F900031042000810050004220AF00D40704003B
:100FA0000000000000052000B08388003A610200C4
:100FB00000000000000278003A610200000000001A
:100FC0004800DD0004004000C08388003A61020050
:100FD00000000000000278003A61020000000000FA
:100FE0004800DD0004004000E08088003A61020013
:100FF00000000000000278003A61020000000000DA
:101000004800DD0004004000E08388003A610200EF
:1010100000000000000278003A61020000000000B9
:101020004800DD0004004000F08388003A610200BF
:1010300000000000000278003A6102000000000099
:101040004800DD00040040009183800081005000D2
:101050004200AF000000EB00008488003A6102000B
:1010600000000000000278003A6102000000000069
:101070004800DD0004004000909488003A610200BE
:1010800000000000000278003A6102000000000049
:101090004800DD0004004000A0948800156EA80000
:1010A0000000000000000000000000000000000040
:1010B00000000000000000000000000062080400C2
:1010C0000000000015EEA80015CEA80015AEA8007F
:1010D0000000000000000000000000000000000010
:1010E000000000000000000000000000156EA900D4
:1010F00000000000000000000000000000000000F0
:10110000000000000000000000000000800E200031
:10111000E66002000000000000002000E66002001F
:101120000000000000002000E66002000000000057
:1011300000002000E6600200000000000000200027
:10114000E66002000000000000002000E6600200EF
:101150000000000000002000E66002000000000027
:1011600000002000E6600200000000003A6102007A
:1011700000000000000278003A6102000000000058
:101180004800DD0004004000B09488003A6102008D
:1011900000000000000278003A6102000000000038
:1011A0004800DD0004004000C0948800156EA800CF
:1011B000000000000000000000000000000000002F
:1011C000000000000000000000000000E6292100EF
:1011D00010002000005B780020032000005B7800F6
:1011E00060838000001B7800A0002000001B7800B6
:1011F00000002000001B7800000A2000001B78007F
:10120000062B210000002000001B78000040260073
:10121000001B7800062D210010002000005B7800E4
:1012200020032000005B780060838000001B7800B2
:10123000A0002000001B780000002000001B7800A8
:10124000000F2000001B7800262E21000000200047
:10125000001B780000402600001B7800263021008B
:1012600010002000005B780060032000005B780025
:1012700060838000001B7800A0002000001B780025
:1012800000002000001B780000142000001B7800E4
:101290004631210000002000001B7800004026009D
:1012A000001B78004633210010002000005B78000E
:1012B00020032000005B780060838000001B780022
:1012C000A0002000001B780000002000001B780018
:1012D00000192000001B7800663421000000200067
:1012E000001B780000402600001B780066362100B5
:1012F00010002000005B780020032000005B7800D5
:1013000060838000001B7800A0002000001B780094
:1013100000002000001B7800001E2000001B780049
:101320008637210000002000001B780000402600C6
:10133000001B78008639210010002000005B780037
:1013400020032000005B780060838000001B780091
:10135000A0002000001B780000002000001B780087
:1013600000232000001B7800A63A21000000200086
:10137000001B780000402600001B7800A63C2100DE
:1013800010002000005B780020032000005B780044
:1013900060838000001B7800A0002000001B780004
:1013A00000002000001B780000282000001B7800AF
:1013B000C63D210000002000001B780000402600F0
:1013C000001B7800C63F210010002000005B780061
:1013D00020032000005B780060838000001B780001
:1013E000A0002000001B780000002000001B7800F7
:1013F000002D2000001B7800E640210000002000A6
:10140000001B780000402600001B7800E642210007
:1014100010002000005B780020032000005B7800B3
:1014200060838000001B7800A0002000001B780073
:1014300000002000001B7800A00A2000001B78009C
:101440000644210000002000001B78000040260018
:10145000001B78000646210010002000005B780089
:1014600020032000005B780060838000001B780070
:10147000A0002000001B780000002000001B780066
:10148000A00F2000001B780026472100000020004C
:10149000001B780000402600001B78002649210030
:1014A00010002000005B780020032000005B780023
:1014B00060838000001B7800A0002000001B7800E3
:1014C00000002000001B7800A0142000001B780002
:1014D000464A210000002000001B78000040260042
:1014E000001B7800464C210010002000005B7800B3
:1014F00020032000005B780060838000001B7800E0
:10150000A0002000001B780000002000001B7800D5
:10151000A0192000001B7800664D2100000020006B
:10152000001B780000402600001B7800664F210059
:1015300010002000005B780020032000005B780092
:1015400060838000001B7800A0002000001B780052
:1015500000002000001B7800A01E2000001B780067
:101560008650210000002000001B7800004026006B
:10157000001B78008652210010002000005B7800DC
:1015800020032000005B780060838000001B78004F
:10159000A0002000001B780000002000001B780045
:1015A000A0232000001B7800A6532100000020008B
:1015B000001B780000402600001B7800A655210083
:1015C00010002000005B780020032000005B780002
:1015D00060838000001B7800A0002000001B7800C2
:1015E00000002000001B7800A0282000001B7800CD
:1015F000C656210000002000001B78000040260095
:10160000001B7800C658210010002000005B780005
:1016100020032000005B780060838000001B7800BE
:10162000A0002000001B780000002000001B7800B4
:10163000A02D2000001B7800E659210000002000AA
:10164000001B780000402600001B7800E65B2100AC
:1016500010002000005B780020032000005B780071
:1016600060838000001B7800A0002000001B780031
:1016700000002000001B7800400B2000001B7800B9
:10168000065D210000002000001B780000402600BD
:10169000001B7800065F210010002000005B78002E
:1016A00020032000005B780060838000001B78002E
:1016B000A0002000001B780000002000001B780024
:1016C00040102000001B7800266021000000200050
:1016D000001B780000402600001B780026622100D5
:1016E00010002000005B780020032000005B7800E1
:1016F00060838000001B7800A0002000001B7800A1
:1017000000002000001B780040152000001B78001E
:101710004663210000002000001B780000402600E6
:10172000001B78004665210010002000005B780057
:1017300020032000005B780060838000001B78009D
:10174000A0002000001B780000002000001B780093
:10175000401A2000001B780066662100000020006F
:10176000001B780000402600001B780066682100FE
:1017700010002000005B780020032000005B780050
:1017800060838000001B7800A0002000001B780010
:1017900000002000001B7800401F2000001B780084
:1017A0008669210000002000001B78000040260010
:1017B000001B7800866B210010002000005B780081
:1017C00020032000005B780060838000001B78000D
:1017D000A0002000001B780000002000001B780003
:1017E00040242000001B7800A66C2100000020008F
:1017F000001B780000402600001B7800A66E210028
:1018000010002000005B780020032000005B7800BF
:1018100060838000001B7800A0002000001B78007F
:1018200000002000001B780040292000001B7800E9
:10183000C66F210000002000001B78000040260039
:10184000001B7800C671210010002000005B7800AA
:1018500020032000005B780060838000001B78007C
:10186000A0002000001B780000002000001B780072
:10187000402E2000001B7800E672210000002000AE
:10188000001B780000402600001B7800E674210051
:1018900010002000005B780020032000005B78002F
:1018A00060838000001B7800A0002000001B7800EF
:1018B00000002000001B7800E00B2000001B7800D7
:1018C0000676210000002000001B78000040260062
:1018D000001B78000678210010002000005B7800D3
:1018E00020032000005B780060838000001B7800EC
:1018F000A0002000001B780000002000001B7800E2
:10190000E0102000001B7800267921000000200054
:10191000001B780000402600001B7800267B210079
:1019200010002000005B780020032000005B78009E
:1019300060838000001B7800A0002000001B78005E
:1019400000002000001B7800E0152000001B78003C
:10195000467C210000002000001B7800004026008B
:10196000001B7800467E210010002000005B7800FC
:1019700020032000005B780060838000001B78005B
:10198000A0002000001B780000002000001B780051
:10199000E01A2000001B7800667F21000000200074
:1019A000001B780000402600001B780066812100A3
:1019B00010002000005B780020032000005B78000E
:1019C00060838000001B7800A0002000001B7800CE
:1019D00000002000001B7800E01F2000001B7800A2
:1019E0008682210000002000001B780000402600B5
:1019F000001B78008684210010002000005B780026
:101A000020032000005B780060838000001B7800CA
:101A1000A0002000001B780000002000001B7800C0
:101A2000E0242000001B7800A68521000000200093
:101A3000001B780000402600001B7800A6872100CC
:101A400010002000005B780020032000005B78007D
:101A500060838000001B7800A0002000001B78003D
:101A600000002000001B7800E0292000001B780007
:101A7000C688210000002000001B780000402600DE
:101A8000001B7800C68A210010002000005B78004F
:101A900020032000005B780060838000001B78003A
:101AA000A0002000001B780000002000001B780030
:101AB000E02E2000001B7800E68B210000002000B3
:101AC000001B780000402600001B78000E6C02000E
:101AD00000000000F00F2000F0938800803E2000FE
:101AE0002084880000002000108188002081880068
:101AF00000002000109488002828A8002848A8008A
:101B00002A28A8002168A8002A48A80020E8A800E0
:101B1000C228A8000000200060C788000230AE0084
:101B200018140400000000000230A900B0072000D3
:101B3000407402000000000010C12E00407402003A
:101B4000000000006083800040740200000000007C
:101B500070838000407402000000000080838000D9
:101B60004074020000000000908380004074020076
:101B700000000000A083800040740200000000000C
:101B8000B08380004074020000000000C083800029
:101B90004074020000000000F080800040740200E9
:101BA000000000000081800040740200000000007E
:101BB000E08080004074020000000000D0838000BC
:101BC0004074020000000000408380004074020066
:101BD00000000000E629210016027800F10F200025
:101BE0000102620041012000068340009641780016
:101BF00001F02F00818161000480710040740200B7
:101C000000000000E629210020022000000343001C
:101C1000160078004074020000000000062D21002C
:101C200016027800F10F200001026200410120003D
:101C3000068340009641780001F02F008181610009
:101C4000048071004074020000000000062D210095
:101C500020022000000343001600780040740200B8
:101C6000000000002630210016027800F10F20004D
:101C70000102620041012000068340009641780085
:101C800001F02F0081816100048071004074020026
:101C90000000000026302100200220000003430045
:101CA0001600780040740200000000004633210056
:101CB00016027800F10F20000102620041012000AD
:101CC000068340009641780001F02F008181610079
:101CD00004807100407402000000000046332100BF
:101CE0002002200000034300160078004074020028
:101CF000000000006636210016027800F10F200077
:101D000001026200410120000683400096417800F4
:101D100001F02F0081816100048071004074020095
:101D2000000000006636210020022000000343006E
:101D3000160078004074020000000000863921007F
:101D400016027800F10F200001026200410120001C
:101D5000068340009641780001F02F0081816100E8
:101D600004807100407402000000000086392100E8
:101D70002002200000034300160078004074020097
:101D800000000000A63C210016027800F10F2000A0
:101D90000102620041012000068340009641780064
:101DA00001F02F0081816100048071004074020005
:101DB00000000000A63C2100200220000003430098
:101DC000160078004074020000000000C63F2100A9
:101DD00016027800F10F200001026200410120008C
:101DE000068340009641780001F02F008181610058
:101DF000048071004074020000000000C63F210012
:101E00002002200000034300160078004074020006
:101E100000000000E642210016027800F10F2000C9
:101E200001026200410120000683400096417800D3
:101E300001F02F0081816100048071004074020074
:101E400000000000E64221002002200000034300C1
:101E500016007800407402000000000006462100D1
:101E600016027800F10F20000102620041012000FB
:101E7000068340009641780001F02F0081816100C7
:101E8000048071004074020000000000064621003A
:101E90002002200000034300160078004074020076
:101EA000000000002649210016027800F10F2000F2
:101EB0000102620041012000068340009641780043
:101EC00001F02F00818161000480710040740200E4
:101ED00000000000264921002002200000034300EA
:101EE000160078004074020000000000464C2100FB
:101EF00016027800F10F200001026200410120006B
:101F0000068340009641780001F02F008181610036
:101F1000048071004074020000000000464C210063
:101F200020022000000343001600780040740200E5
:101F300000000000664F210016027800F10F20001B
:101F400001026200410120000683400096417800B2
:101F500001F02F0081816100048071004074020053
:101F600000000000664F2100200220000003430013
:101F70001600780040740200000000008652210024
:101F800016027800F10F20000102620041012000DA
:101F9000068340009641780001F02F0081816100A6
:101FA000048071004074020000000000865221008D
:101FB0002002200000034300160078004074020055
:101FC00000000000A655210016027800F10F200045
:101FD0000102620041012000068340009641780022
:101FE00001F02F00818161000480710040740200C3
:101FF00000000000A655210020022000000343003D
:10200000160078004074020000000000C65821004D
:1020100016027800F10F2000010262004101200049
:10202000068340009641780001F02F008181610015
:10203000048071004074020000000000C6582100B6
:1020400020022000000343001600780040740200C4
:1020500000000000E65B210016027800F10F20006E
:102060000102620041012000068340009641780091
:1020700001F02F0081816100048071004074020032
:1020800000000000E65B2100200220000003430066
:10209000160078004074020000000000065F210076
:1020A00016027800F10F20000102620041012000B9
:1020B000068340009641780001F02F008181610085
:1020C000048071004074020000000000065F2100DF
:1020D0002002200000034300160078004074020034
:1020E000000000002662210016027800F10F200097
:1020F0000102620041012000068340009641780001
:1021000001F02F00818161000480710040740200A1
:10211000000000002662210020022000000343008E
:10212000160078004074020000000000466521009F
:1021300016027800F10F2000010262004101200028
:10214000068340009641780001F02F0081816100F4
:102150000480710040740200000000004665210008
:1021600020022000000343001600780040740200A3
:10217000000000006668210016027800F10F2000C0
:102180000102620041012000068340009641780070
:1021900001F02F0081816100048071004074020011
:1021A00000000000666821002002200000034300B8
:1021B000160078004074020000000000866B2100C9
:1021C00016027800F10F2000010262004101200098
:1021D000068340009641780001F02F008181610064
:1021E000048071004074020000000000866B210032
:1021F0002002200000034300160078004074020013
:1022000000000000A66E210016027800F10F2000E9
:1022100001026200410120000683400096417800DF
:1022200001F02F0081816100048071004074020080
:1022300000000000A66E21002002200000034300E1
:10224000160078004074020000000000C6712100F2
:1022500016027800F10F2000010262004101200007
:10226000068340009641780001F02F0081816100D3
:10227000048071004074020000000000C67121005B
:102280002002200000034300160078004074020082
:1022900000000000E674210016027800F10F200013
:1022A000010262004101200006834000964178004F
:1022B00001F02F00818161000480710040740200F0
:1022C00000000000E674210020022000000343000B
:1022D000160078004074020000000000067821001B
:1022E00016027800F10F2000010262004101200077
:1022F000068340009641780001F02F008181610043
:102300000480710040740200000000000678210083
:1023100020022000000343001600780040740200F1
:1023200000000000267B210016027800F10F20003B
:1023300001026200410120000683400096417800BE
:1023400001F02F008181610004807100407402005F
:1023500000000000267B2100200220000003430033
:10236000160078004074020000000000467E210044
:1023700016027800F10F20000102620041012000E6
:10238000068340009641780001F02F0081816100B2
:10239000048071004074020000000000467E2100AD
:1023A0002002200000034300160078004074020061
:1023B000000000006681210016027800F10F200065
:1023C000010262004101200006834000964178002E
:1023D00001F02F00818161000480710040740200CF
:1023E000000000006681210020022000000343005D
:1023F000160078004074020000000000868421006E
:1024000016027800F10F2000010262004101200055
:10241000068340009641780001F02F008181610021
:1024200004807100407402000000000086842100D6
:1024300020022000000343001600780040740200D0
:1024400000000000A687210016027800F10F20008E
:10245000010262004101200006834000964178009D
:1024600001F02F008181610004807100407402003E
:1024700000000000A6872100200220000003430086
:10248000160078004074020000000000C68A210097
:1024900016027800F10F20000102620041012000C5
:1024A000068340009641780001F02F008181610091
:1024B000048071004074020000000000C68A210000
:1024C0002002200000034300160078004074020040
:1024D0000000000020808000407402000000000026
:1024E00030808000407402000000000040808000C6
:1024F0004074020000000000508080004074020020
:1025000000000000608080004074020000000000B5
:102510007080800040740200000000008080800015
:1025200040740200000000009080800040740200AF
:1025300000000000A0808000407402000000000045
:10254000B08080004074020000000000C080800065
:102550004074020000000000D0808000407402003F
:1025600000000000D00720004074020000000000BE
:102570000040200061C78000808050004200AE0013
:10258000181404000000000090948000D09488008B
:10259000A0948000E0948800B0948000909488001B
:1025A000C0948000A094880015EEA90015CEA90063
:1025B00015AEA800000000000000000000000000B0
:1025C000000000000000000000000000000000000B
:1025D000067C020000000000156EA900000000004B
:1025E00000000000000000000000000000000000EB
:1025F000000000000000000040082000E66002002B
:1026000000000000A4948000F30720000300620093
:10261000E660020000000000949480004822DE0082
:1026200003006200E6600200000000009494800055
:10263000F30F200003006200E660020000000000CB
:102640000608200054740200000000000002780018
:102650004800DE00F30F200003006000E660020087
:102660000000000003006200E660020000000000BD
:102670000603E9000600E0004220AE002213040039
:10268000000000000000000000000000000000004A
:10269000156EA8000000000000000000000000000F
:1026A000000000000000000000000000000000002A
:1026B0008662020000000000627C02000000000050
:1026C000001020000100200092948000A39480005C
:1026D0000200400083804800B0948800C1948800C4
:1026E000000020009094880000002000A094880042
:1026F00015EEA80015CEA80015AEA8000000000039
:1027000000000000000000000000000000000000C9
:102710000000000000000000067C02000000000035
:10272000156EA9000000000000000000000000007D
:102730000000000000000000000000000000000099
:1027400040082000E66002000000000000002000B9
:10275000E66002000000000000002000E6600200C9
:102760000000000000002000E66002000000000001
:10277000B094800000027800F30F20000300600096
:10278000E6600200000000004822DE000300620054
:10279000E660020000000000C094800000027800A3
:1027A000F30F200003006000E6600200000000005C
:1027B0004822DE0003006200E66002000000000024
:1027C000156EA800000000000000000000000000DE
:1027D00000000000000000000000000000000000F9
:1027E0008662020000000000627C0200000000001F
:1027F00015EEA90015CEA90015AEA9000000000035
:1028000000000000000000000000000000000000C8
:102810000000000000000000D09480009094880028
:10282000E0948000A094880000402000EC38B500BF
:10283000108180000000D000E1072000010060004E
:102840000006010070160400000000001E190400BC
:10285000000000002819040000000000201D0400F2
:1028600000000000624E040000000000E65004007A
:1028700000000000AE150400000000005416040023
:10288000000000008C230400000000002229040046
:10289000000000001053040000000000705304000A
:1028A0000000000002430400000000005047040044
:1028B00000000000D229040000000000EE2A0400FD
:1028C00000000000C230040000000000E2360400F6
:1028D00000000000222C0400000000003E2D040037
:1028E00000000000722E0400000000008E2F040083
:1028F000000000008637040000000000A238040039
:1029000000000000D639040000000000F23A040084
:1029100000000000263C040000000000423D0400CE
:1029200000000000763E040000000000923F04001A
:1029300000000000B240040000000000CE4104008E
:1029400000000000BC47040000000000D84804005C
:1029500000000000604C040000000000244E040051
:10296000000000000C4A040000000000284B040096
:1029700000000000A615040000000000A6150400D9
:1029800000000000A615040000000000A6150400C9
:1029900000000000A615040000000000A6150400B9
:1029A00000000000A615040000000000A6150400A9
:1029B00000000000A615040000000000A615040099
:1029C00000000000A615040000000000A615040089
:1029D00000000000A615040000000000A615040079
:1029E00000000000A615040000000000A615040069
:1029F00000000000A615040000000000A615040059
:102A000000000000A615040000000000A615040048
:102A100000000000A615040000000000A615040038
:102A200000000000A615040000000000A615040028
:102A300000000000A615040000000000A615040018
:102A400000000000A615040000000000A615040008
:102A500000000000A615040000000000A6150400F8
:102A600000000000A615040000000000A6150400E8
:102A700000000000A615040000000000A6150400D8
:102A800000000000A615040000000000A6150400C8
:102A900000000000A615040000000000A6150400B8
:102AA00000000000A615040000000000A6150400A8
:102AB00000000000A615040000000000A615040098
:102AC00000000000A615040000000000A615040088
:102AD00000000000A615040000000000A615040078
:102AE00000000000A615040000000000A615040068
:102AF00000000000A615040000000000A615040058
:102B000000000000A615040000000000A615040047
:102B100000000000A615040000000000A615040037
:102B200000000000A615040000000000A615040027
:102B300000000000A615040000000000A615040017
:102B400000000000A61504000000000000002000A6
:102B5000108188008E0D04000000000058640200FF
:102B600000000000E41120006004200080630200E7
:102B700000000000F30F200003006200FE6202006C
:102B8000000000004822DE0003006200FE62020036
:102B9000000000002004200080630200000000000C
:102BA00030052000FE62020000000000000220004C
:102BB000FE6202000000000040052000FE620200EC
:102BC0000000000000022000FE6202000000000081
:102BD00050052000FE6202000000000000022000FC
:102BE000FE6202000000000020042000FE620200DD
:102BF0000000000084482000600420008063020080
:102C000000000000F30F200003006200FE620200DB
:102C1000000000004822DE0003006200FE620200A5
:102C2000000000002004200080630200000000007B
:102C3000D0042000FE62020000000000100420000A
:102C4000FE6202000000000090042000FE6202000C
:102C500000000000E0042000FE620200000000000E
:102C600000022000FE62020000000000D0042000EC
:102C7000FE6202000000000050042000FE6202001C
:102C800000000000E0042000FE62020000000000DE
:102C900050052000FE620200000000002230EC001F
:102CA0008E0D04000000000040C7800031002000AD
:102CB000010050004220AE006C160400000000002D
:102CC0007E23020000000000200020001081880008
:102CD0008E0D0400000000008E0D040000000000B6
:102CE0005864020000000000641720006004200007
:102CF0008063020000000000F30F20000300620068
:102D0000FE620200000000004822DE0003006200B4
:102D1000FE62020000000000200420008063020028
:102D20000000000010042000FE620200000000000D
:102D300000022000FE62020000000000700420007B
:102D4000FE6202000000000000022000FE6202009D
:102D50000000000020052000FE62020000000000CC
:102D600000022000FE62020000000000900420002B
:102D7000FE6202000000000000022000FE6202006D
:102D80000000000070042000FE620200000000004D
:102D900000022000FE62020000000000500420003B
:102DA000FE6202000000000000022000FE6202003D
:102DB00000000000C0042000FE62020000000000CD
:102DC0004421200060042000806302000000000015
:102DD000F30F200003006200FE620200000000000A
:102DE0004822DE0003006200FE62020000000000D4
:102DF000200420008063020000000000C0042000C6
:102E0000FE6202000000000090042000FE6202004A
:102E10000000000010052000FE620200000000001B
:102E200050052000FE620200000000009004200017
:102E3000FE6202000000000040042000FE6202006A
:102E40000000000000022000FE62020000000000FE
:102E500060042000FE620200000000005004200018
:102E6000FE6202000000000020052000FE62020059
:102E70000000000040052000FE620200000000008B
:102E800090042000FE62020000000000C004200048
:102E9000FE6202000000000090042000FE620200BA
:102EA00000000000A0052000FE62020000000000FB
:102EB00050042000FE6202000000000020052000F7
:102EC000FE62020000000000442620006004200092
:102ED0008063020000000000F30F20000300620086
:102EE000FE620200000000004822DE0003006200D3
:102EF000FE62020000000000200420008063020047
:102F00000000000010042000FE620200000000002B
:102F100000052000FE620200000000000005200005
:102F2000FE62020000000000C0042000FE620200F9
:102F30000000000090042000FE620200000000007B
:102F400030042000FE620200000000001004200097
:102F5000FE6202000000000040052000FE62020048
:102F60000000000090042000FE620200000000004B
:102F7000F0042000FE62020000000000E0042000D7
:102F8000FE6202000000000000022000FE6202005B
:102F90000000000000022000FE62020000000000AD
:102FA00050052000FE62020000000000E004200046
:102FB000FE6202000000000090042000FE62020099
:102FC0000000000040052000FE620200000000003A
:102FD000C42D200060042000806302000000000077
:102FE000F30F200003006200FE62020000000000F8
:102FF0004822DE0003006200FE62020000000000C2
:103000002004200080630200000000007007200000
:10301000FE6202000000000070072000FE62020055
:103020000000000070072000FE62020000000000A7
:10303000E0022000FE6202000000000010062000F6
:10304000FE6202000000000070062000FE62020026
:103050000000000020072000FE62020000000000C7
:1030600090062000FE6202000000000070062000B2
:10307000FE6202000000000050062000FE62020016
:1030800000000000C0062000FE62020000000000F8
:10309000E0022000FE620200000000003006200076
:1030A000FE62020000000000F0062000FE62020046
:1030B00000000000E0022000FE62020000000000AC
:1030C000A0072000FE6202000000000010062000A1
:1030D000FE62020000000000343520006004200081
:1030E0008063020000000000F30F20000300620074
:1030F000FE620200000000004822DE0003006200C1
:10310000FE62020000000000200420008063020034
:103110000000000060052000FE62020000000000C8
:1031200050062000FE620200000000002007200080
:10313000FE6202000000000030072000FE62020074
:103140000000000090062000FE6202000000000067
:10315000F0062000FE62020000000000E0062000F1
:10316000FE6202000000000000022000FE62020079
:1031700000000000A0032000FE620200000000002A
:1031800000022000FE620200000000005004200047
:10319000FE6202000000000030042000FE62020017
:1031A0000000000010032000FE620200000000008A
:1031B00010032000FE620200000000000002200058
:1031C000FE6202000000000020042000FE620200F7
:1031D0000000000050062000FE6202000000000017
:1031E00040072000FE6202000000000010062000E0
:1031F000FE62020000000000B435200060042000E0
:103200008063020000000000F30F20000300620052
:10321000FE620200000000004822DE00030062009F
:10322000FE6202000000000080BB200030838800A6
:103230002230EC008E0D0400000000006610E20059
:103240004220AF002230EC008E0D04000000000090
:103250005864020000000000E41120006004200017
:103260008063020000000000F30F200003006200F2
:10327000FE620200000000004822DE00030062003F
:10328000FE620200000000002004200080630200B3
:1032900000000000D0042000FE62020000000000D8
:1032A00000022000FE620200000000001004200066
:1032B000FE6202000000000000022000FE62020028
:1032C0000000000090042000FE62020000000000E8
:1032D00000022000FE62020000000000E004200066
:1032E000FE6202000000000000022000FE620200F8
:1032F0000000000000022000FE620200000000004A
:1033000000022000FE62020000000000D004200045
:10331000FE6202000000000000022000FE620200C7
:103320000000000050042000FE62020000000000C7
:1033300000022000FE62020000000000E004200005
:10334000FE6202000000000000022000FE62020097
:103350000000000050052000FE6202000000000096
:10336000641420006004200080630200000000005C
:10337000F30F200003006200FE6202000000000064
:103380004822DE0003006200FE620200000000002E
:10339000200420008063020000000000D002200012
:1033A000FE62020000000000D0022000FE62020067
:1033B00000000000D0022000FE62020000000000B9
:1033C000D0022000FE62020000000000D0022000B7
:1033D000FE62020000000000D0022000FE62020037
:1033E00000000000D0022000FE6202000000000089
:1033F000D0022000FE62020000000000D002200087
:10340000FE62020000000000D0022000FE62020006
:1034100000000000D0022000FE6202000000000058
:10342000D0022000FE62020000000000D002200056
:10343000FE62020000000000D0022000FE620200D6
:1034400000000000D0022000FE6202000000000028
:10345000D0022000FE62020000000000D002200026
:10346000FE6202000000000004232000600420002F
:103470008063020000000000F30F200003006200E0
:10348000FE620200000000004822DE00030062002D
:10349000FE620200000000002004200080630200A1
:1034A0000000000040042000FE6202000000000056
:1034B00010042000FE620200000000004005200011
:1034C000FE6202000000000010042000FE62020004
:1034D00000000000842520006004200080630200BA
:1034E00000000000F30F200003006200FE620200F3
:1034F000000000004822DE0003006200FE620200BD
:103500000000000020042000806302000000000092
:10351000D0042000FE620200000000001004200021
:10352000FE62020000000000E0042000FE620200D3
:103530000000000010042000FE62020000000000F5
:1035400070042000FE620200000000005004200011
:10355000FE62020000000000D0042000FE620200B3
:103560000000000050042000FE6202000000000085
:10357000E0042000FE620200000000004005200080
:10358000FE62020000000000843E20006004200073
:103590008063020000000000F30F200003006200BF
:1035A000FE620200000000004822DE00030062000C
:1035B000FE62020000000000200420008063020080
:1035C0000000000030052000FE6202000000000044
:1035D00050042000FE6202000000000040052000B0
:1035E000FE6202000000000040052000FE620200B2
:1035F0000000000090042000FE62020000000000B5
:10360000E0042000FE6202000000000070042000C0
:10361000FE6202000000000030052000FE62020091
:103620000000000074092000600420008063020094
:1036300000000000F30F200003006200FE620200A1
:10364000000000004822DE0003006200FE6202006B
:103650000000000020042000806302000000000041
:1036600000052000FE62020000000000C0042000EF
:10367000FE6202000000000010042000FE62020052
:1036800000000000E0042000FE62020000000000D4
:1036900040052000FE6202000000000090042000AF
:1036A000FE62020000000000D0042000FE62020062
:1036B0000000000070042000FE6202000000000014
:1036C000F40B200060042000806302000000000072
:1036D000F30F200003006200FE6202000000000001
:1036E0004822DE0003006200FE62020000000000CB
:1036F000200420008063020000000000300520004C
:10370000FE6202000000000050042000FE62020081
:103710000000000040052000FE62020000000000E2
:1037200040052000FE62020000000000900420001E
:10373000FE62020000000000E0042000FE620200C1
:103740000000000070042000FE6202000000000083
:1037500030052000FE620200000000000425200069
:10376000600420008063020000000000F30F2000CE
:1037700003006200FE620200000000004822DE003A
:1037800003006200FE62020000000000200420002E
:10379000806302000000000070052000FE6202004D
:1037A00000000000F0042000FE62020000000000A3
:1037B00020052000FE62020000000000B00420008E
:1037C000FE6202000000000090042000FE62020081
:1037D00000000000E0042000FE6202000000000083
:1037E00070042000FE62020000000000B4272000E8
:1037F000600420008063020000000000F30F20003E
:1038000003006200FE620200000000004822DE00A9
:1038100003006200FE62020000000000200420009D
:103820008063020000000000D0042000FE6202005D
:1038300000000000F0042000FE6202000000000012
:1038400040042000FE62020000000000500420003E
:10385000FE620200000000004440200060042000DE
:103860008063020000000000F30F200003006200EC
:10387000FE620200000000004822DE000300620039
:10388000FE620200000000002004200080630200AD
:103890000000000030042000FE6202000000000072
:1038A00010042000FE62020000000000C00420009E
:1038B000FE6202000000000090042000FE62020090
:1038C0000000000020042000FE6202000000000052
:1038D00020052000FE62020000000000100420000D
:1038E000FE6202000000000040052000FE620200AF
:1038F0000000000090042000FE62020000000000B2
:10390000F0042000FE62020000000000E00420003D
:10391000FE6202000000000034432000600420002A
:103920008063020000000000F30F2000030062002B
:10393000FE620200000000004822DE000300620078
:10394000FE620200000000002004200080630200EC
:1039500000000000D0042000FE6202000000000011
:10396000F0042000FE62020000000000400420007D
:10397000FE6202000000000050042000FE6202000F
:1039800000000000844820006004200080630200E2
:1039900000000000F30F200003006200FE6202003E
:1039A000000000004822DE0003006200FE62020008
:1039B00000000000200420008063020000000000DE
:1039C00000052000FE62020000000000F00420005C
:1039D000FE6202000000000070052000FE6202008E
:1039E0000000000050042000FE6202000000000001
:1039F00020052000FE6202000000000000022000FE
:103A0000FE62020000000000F0042000FE620200DE
:103A10000000000060042000FE62020000000000C0
:103A200060042000FE6202000000000080382100D7
:103A3000308388002230EC008E0D0400000000006E
:103A400040C7800031002000010050004220AE003D
:103A5000381D0400000000007E230200000000006A
:103A60002002200010818800B41D04000000000026
:103A700040C7800011002000010050004220AE002D
:103A8000501D0400000000007E2302000000000022
:103A90004000200010818800B41D040000000000D8
:103AA00040C7800021002000010050004220AE00ED
:103AB000641D0400000000006000200010818800E8
:103AC000B41D04000000000040C7800091002000E9
:103AD000010050004220AE00781D040000000000EC
:103AE0008000200010818800B41D04000000000048
:103AF00040C7800081002000010050004220AE003D
:103B00008C1D040000000000A0002000108188002F
:103B1000B41D04000000000040C7800071002000B8
:103B2000010050004220AE00A41D0400000000006F
:103B30007E23020000000000C000200010818800E9
:103B4000B41D0400000000006610E2004220AE0038
:103B5000B41D040000000000A000200010818800B7
:103B6000B41D0400000000008E0D040000000000E1
:103B70005864020000000000840720006004200058
:103B80008063020000000000F30F200003006200C9
:103B9000FE620200000000004822DE000300620016
:103BA000FE6202000000000020042000806302008A
:103BB0000000000010042000FE620200000000006F
:103BC00000072000FE620200000000000007200045
:103BD000FE62020000000000C0062000FE6202003B
:103BE0000000000090062000FE62020000000000BD
:103BF0000423200060042000806302000000000015
:103C0000F30F200003006200FE62020000000000CB
:103C10004822DE0003006200FE6202000000000095
:103C20002004200080630200000000004004200007
:103C3000FE6202000000000050062000FE6202004A
:103C400000000000E0062000FE620200000000000C
:103C500030072000FE6202000000000090062000F5
:103C6000FE62020000000000843E2000600420008C
:103C70008063020000000000F30F200003006200D8
:103C8000FE620200000000004822DE000300620025
:103C9000FE62020000000000200420008063020099
:103CA0000000000020052000FE620200000000006D
:103CB000F0062000FE6202000000000070072000F5
:103CC000FE62020000000000F0022000FE6202001E
:103CD0000000000080042000FE62020000000000DE
:103CE000B44820006004200080630200000000004F
:103CF000F30F200003006200FE62020000000000DB
:103D00004822DE0003006200FE62020000000000A4
:103D100020042000806302000000000054492000BD
:103D2000600420008063020000000000F30F200008
:103D300003006200FE620200000000004822DE0074
:103D400003006200FE620200000000002004200068
:103D50008063020000000000044A2000600420008C
:103D60008063020000000000F30F200003006200E7
:103D7000FE620200000000004822DE000300620034
:103D8000FE620200000000002004200080630200A8
:103D900000000000A44A20006004200080630200AC
:103DA00000000000F30F200003006200FE6202002A
:103DB000000000004822DE0003006200FE620200F4
:103DC00000000000200420008063020000000000CA
:103DD000F440200060042000806302000000000026
:103DE000F30F200003006200FE62020000000000EA
:103DF0004822DE0003006200FE62020000000000B4
:103E00002004200080630200000000003005200034
:103E1000FE6202000000000000072000FE620200B7
:103E20000000000050062000FE62020000000000BA
:103E300050062000FE620200000000004006200044
:103E4000FE620200000000007425200060042000D3
:103E50008063020000000000F30F200003006200F6
:103E6000FE620200000000004822DE000300620043
:103E7000FE620200000000002004200080630200B7
:103E80000000000030042000FE620200000000007C
:103E900010062000FE62020000000000C0062000A4
:103EA000FE6202000000000090062000FE62020098
:103EB0000000000020062000FE620200000000005A
:103EC000F40920006004200080630200000000006C
:103ED000F30F200003006200FE62020000000000F9
:103EE0004822DE0003006200FE62020000000000C3
:103EF0002004200080630200000000003005200044
:103F0000FE6202000000000000072000FE620200C6
:103F10000000000010062000FE6202000000000009
:103F200020072000FE620200000000005006200072
:103F3000FE62020000000000B4482000600420007F
:103F40008063020000000000F30F20000300620005
:103F5000FE620200000000004822DE000300620052
:103F6000FE62020000000000D00520008063020015
:103F70000000000040002000FE620200000000007F
:103F800070002000FE62020000000000900520008A
:103F9000806302000000000070052000FE62020045
:103FA000000000002230EC008E0D04000000000034
:103FB000E082800080818800B66B02000000000073
:103FC0000483800060042000806302000000000081
:103FD000F30F200003006200FE62020000000000F8
:103FE0004822DE0003006200FE62020000000000C2
:103FF000200420008063020000000000A0828000F6
:104000000103200001004000FE62020000000000E9
:10401000B08280000103200001004000FE62020027
:1040200000000000C0828000010320000100400069
:10403000FE62020000000000D08280000103200028
:1040400001004000FE6202000000000004838000C6
:1040500010838000000242006004200080630200A0
:1040600000000000F30F200003006200FE62020067
:10407000000000004822DE0003006200FE62020031
:1040800000000000A0828000DE220200000000008C
:10409000A08288006230EC00B0828000DE22020044
:1040A00000000000B08288006230EC00C082800016
:1040B000DE22020000000000C08288006230EC00B6
:1040C000D0828000DE22020000000000D082880042
:1040D000D4828000A0002000C18280000101B800CD
:1040E0000402410040062000B18280000101B800B6
:1040F00004024100803E2000A18280000101B8003E
:1041000004024100E482880000000600E082800092
:1041100080818800B66B02000000000004838000EC
:10412000600420008063020000000000F30F200004
:1041300003006200FE620200000000004822DE0070
:1041400003006200FE620200000000002004200064
:104150008063020000000000C08280000103200094
:1041600001004000FE62020000000000D0828000DA
:104170000103200001004000FE6202000000000078
:10418000048380001083800000024200600420004D
:104190008063020000000000F30F200003006200B3
:1041A000FE620200000000004822DE000300620000
:1041B000FE62020000000000C0828000DE220200D9
:1041C00000000000C08288006230EC00D0828000D5
:1041D000DE22020000000000D0828800D48280002D
:1041E000A0002000C18280000101B800040241004B
:1041F000E482880000000600E08280008081880060
:10420000B66B020000000000048380006004200000
:104210008063020000000000F30F20000300620032
:10422000FE620200000000004822DE00030062007F
:10423000FE620200000000002004200080630200F3
:1042400000000000B0828000010320000100400057
:10425000FE62020000000000C08280000103200016
:1042600001004000FE62020000000000D0828000D9
:104270000103200001004000FE6202000000000077
:10428000048380001083800000024200600420004C
:104290008063020000000000F30F200003006200B2
:1042A000FE620200000000004822DE0003006200FF
:1042B000FE62020000000000B0828000DE220200E8
:1042C00000000000B08288006230EC00C0828000F4
:1042D000DE22020000000000C08288006230EC0094
:1042E000D0828000DE22020000000000D082880020
:1042F000D4828000A0002000C18280000101B800AB
:104300000402410040062000B18280000101B80093
:1043100004024100E482880000000600E082800080
:1043200080818800B66B02000000000004838000DA
:10433000600420008063020000000000F30F2000F2
:1043400003006200FE620200000000004822DE005E
:1043500003006200FE620200000000002004200052
:104360008063020000000000A082800001032000A2
:1043700001004000FE62020000000000B0828000E8
:104380000103200001004000FE6202000000000066
:10439000C08280000103200001004000FE62020094
:1043A00000000000D08280000103200001004000D6
:1043B000FE62020000000000048380001083800081
:1043C0000002420060042000806302000000000040
:1043D000F30F200003006200FE62020000000000F4
:1043E0004822DE0003006200FE62020000000000BE
:1043F000A0828000DE22020000000000A08288006F
:104400006230EC00B0828000DE220200000000007A
:10441000B08288006230EC00C0828000DE220200A0
:1044200000000000C08288006230EC00D082800072
:10443000DE22020000000000D0828800D4828000CA
:10444000A0002000C18280000101B80004024100E8
:1044500040062000B18280000101B8000402410042
:10446000803E2000A18280000101B80004024100CA
:10447000E482880000000600E082800080818800DD
:10448000B66B02000000000004838000600420007E
:104490008063020000000000F30F200003006200B0
:1044A000FE620200000000004822DE0003006200FD
:1044B000FE62020000000000200420008063020071
:1044C00000000000A08280000103200001004000E5
:1044D000FE62020000000000E0022000FE62020016
:1044E00000000000B08280000103200001004000B5
:1044F000FE62020000000000C08280000103200074
:1045000001004000FE620200000000000483800001
:1045100010838000000242006004200080630200DB
:1045200000000000F30F200003006200FE620200A2
:10453000000000004822DE0003006200FE6202006C
:1045400000000000A0828000DE22020000000000C7
:10455000A08288006230EC006230EC00B082800003
:10456000DE22020000000000B08288006230EC0011
:10457000C0828000DE22020000000000C0828800AD
:10458000D4828000A0002000C18280000101B80018
:104590000402410040062000B18280000101B80001
:1045A00004024100803E2000A18280000101B80089
:1045B00004024100E4828800000006002083880095
:1045C0000483800010838000000242006004200009
:1045D0008063020000000000F30F2000030062006F
:1045E000FE620200000000004822DE0003006200BC
:1045F000FE62020000000000200420008063020030
:104600000000000020838000010320000100400022
:10461000FE6202000000000004838000108380001E
:1046200000024200600420008063020000000000DD
:10463000F30F200003006200FE6202000000000091
:104640004822DE0003006200FE620200000000005B
:1046500040C7800041002000010050004220AE0011
:1046600048230400000000006430EC002083800038
:10467000A1002000810050004200AF006430EF0034
:104680007E23020000000000E02204000000000081
:1046900040C7800051002000010050004220AE00C1
:1046A0006A230400000000006430ED0020838000D5
:1046B000A100200092002000810050004200AF00C5
:1046C000228388007E23020000000000E022040014
:1046D0000000000040C78000610020000100500081
:1046E0004220AE0028230400000000007E230200C8
:1046F00000000000208380000000060040C780000A
:10470000F1FF2F00010050004220AE007E23040084
:1047100000000000000006005864020000000000D5
:10472000B407200060042000806302000000000045
:10473000F30F200003006200FE6202000000000090
:104740004822DE0003006200FE620200000000005A
:10475000200420008063020000000000000520000B
:10476000FE6202000000000000022000FE62020063
:1047700000000000C0042000FE62020000000000F3
:1047800000022000FE620200000000001004200071
:10479000FE6202000000000000022000FE62020033
:1047A00000000000E0042000FE62020000000000A3
:1047B00000022000FE620200000000004005200010
:1047C000FE6202000000000000022000FE62020003
:1047D0000000000090042000FE62020000000000C3
:1047E00000022000FE62020000000000E004200041
:1047F000FE6202000000000000022000FE620200D3
:104800000000000070042000FE62020000000000B2
:1048100000022000FE6202000000000000022000F2
:10482000FE6202000000000000022000FE620200A2
:104830000000000030052000FE62020000000000C1
:1048400000022000FE620200000000005004200070
:10485000FE6202000000000000022000FE62020072
:104860000000000040052000FE6202000000000081
:1048700000022000FE62020000000000400520004F
:10488000FE6202000000000000022000FE62020042
:104890000000000090042000FE6202000000000002
:1048A00000022000FE62020000000000E004200080
:1048B000FE6202000000000000022000FE62020012
:1048C0000000000070042000FE62020000000000F2
:1048D00000022000FE6202000000000030052000FF
:1048E000FE62020000000000340A20006004200084
:1048F0008063020000000000F30F2000030062004C
:10490000FE620200000000004822DE000300620098
:10491000FE6202000000000020042000806302000C
:1049200000000000D0022000FE6202000000000033
:10493000D0022000FE62020000000000D002200031
:10494000FE62020000000000D0022000FE620200B1
:1049500000000000D0022000FE6202000000000003
:10496000D0022000FE62020000000000D002200001
:10497000FE62020000000000D0022000FE62020081
:1049800000000000D0022000FE62020000000000D3
:10499000D0022000FE62020000000000D0022000D1
:1049A000FE62020000000000D0022000FE62020051
:1049B00000000000D0022000FE62020000000000A3
:1049C000D0022000FE62020000000000D0022000A1
:1049D000FE62020000000000D0022000FE62020021
:1049E00000000000D0022000FE6202000000000073
:1049F000D0022000FE62020000000000D002200071
:104A0000FE62020000000000D0022000FE620200F0
:104A100000000000D0022000FE6202000000000042
:104A2000D0022000FE62020000000000D002200040
:104A3000FE62020000000000D0022000FE620200C0
:104A400000000000D0022000FE6202000000000012
:104A5000D0022000FE62020000000000D002200010
:104A6000FE62020000000000D0022000FE62020090
:104A700000000000D0022000FE62020000000000E2
:104A8000D0022000FE62020000000000D0022000E0
:104A9000FE62020000000000D0022000FE62020060
:104AA00000000000D0022000FE62020000000000B2
:104AB0000423200060042000806302000000000046
:104AC000F30F200003006200FE62020000000000FD
:104AD0004822DE0003006200FE62020000000000C7
:104AE000200420008063020000000000708380002A
:104AF00080818800B66B020000000000B082800058
:104B00000103200001004000FE62020000000000DE
:104B1000C08280000103200001004000FE6202000C
:104B200000000000D082800001032000010040004E
:104B3000FE6202000000000000022000FE6202008F
:104B400000000000C0042000FE620200000000001F
:104B500010042000FE62020000000000E0042000BB
:104B6000FE6202000000000040042000FE6202001D
:104B70000000000000022000FE62020000000000B1
:104B8000E0042000FE62020000000000500520004A
:104B9000FE62020000000000D0042000FE6202005D
:104BA0000000000020042000FE620200000000005F
:104BB00050042000FE6202000000000020052000DA
:104BC000FE62020000000000843E2000600420001D
:104BD0008063020000000000F30F20000300620069
:104BE000FE620200000000004822DE0003006200B6
:104BF000FE6202000000000020042000806302002A
:104C00000000000090042000FE620200000000008E
:104C1000D0042000FE620200000000000005200019
:104C2000FE62020000000000C0042000FE620200DC
:104C30000000000050042000FE620200000000009E
:104C4000D0042000FE62020000000000500420009A
:104C5000FE62020000000000E0042000FE6202008C
:104C60000000000040052000FE620200000000007D
:104C70000441200060042000806302000000000066
:104C8000F30F200003006200FE620200000000003B
:104C90004822DE0003006200FE6202000000000005
:104CA0002004200080630200000000003005200086
:104CB000FE6202000000000050042000FE620200BC
:104CC0000000000040052000FE620200000000001D
:104CD00040052000FE620200000000009004200059
:104CE000FE62020000000000E0042000FE620200FC
:104CF0000000000070042000FE62020000000000BE
:104D000030052000FE620200000000008424200024
:104D1000600420008063020000000000F30F200008
:104D200003006200FE620200000000004822DE0074
:104D300003006200FE620200000000002004200068
:104D4000806302000000000060042000FE62020098
:104D50000000000050042000FE620200000000007D
:104D600020052000FE620200000000004005200037
:104D7000FE6202000000000090042000FE620200BB
:104D800000000000C0042000FE62020000000000DD
:104D900090042000FE6202000000000030052000A8
:104DA000FE6202000000000050042000FE620200CB
:104DB0000000000020052000FE620200000000004C
:104DC00064272000600420008063020000000000CF
:104DD000F30F200003006200FE62020000000000EA
:104DE0004822DE0003006200FE62020000000000B4
:104DF000200420008063020000000000B0062000B4
:104E0000FE6202000000000070062000FE62020048
:104E100000000000F0022000FE620200000000001E
:104E200080062000FE620200000000000002200058
:104E3000FE62020000000000608380008081880024
:104E4000B66B020000000000A08280000103200079
:104E500001004000FE62020000000000B0828000FD
:104E60000103200001004000FE620200000000007B
:104E7000C08280000103200001004000FE620200A9
:104E800000000000D08280000103200001004000EB
:104E9000FE620200000000000440200060042000C8
:104EA0008063020000000000F30F20000300620096
:104EB000FE620200000000004822DE0003006200E3
:104EC000FE62020000000000200420008063020057
:104ED0000000000060042000FE62020000000000EC
:104EE00050042000FE6202000000000020052000A7
:104EF000FE6202000000000040052000FE62020089
:104F00000000000090042000FE620200000000008B
:104F1000C0042000FE620200000000009004200097
:104F2000FE6202000000000030052000FE62020068
:104F30000000000050042000FE620200000000009B
:104F400020052000FE620200000000000443200053
:104F5000600420008063020000000000F30F2000C6
:104F600003006200FE620200000000004822DE0032
:104F700003006200FE620200000000002004200026
:104F8000806302000000000030052000FE62020085
:104F90000000000070042000FE620200000000001B
:104FA00000022000FE62020000000000F08080008D
:104FB00080818800B66B020000000000A0828000A3
:104FC0000103200001004000FE620200000000001A
:104FD000E0022000FE62020000000000B0828000BB
:104FE0000103200001004000FE62020000000000FA
:104FF000C08280000103200001004000FE62020028
:10500000000000008448200060042000806302004B
:1050100000000000F30F200003006200FE620200A7
:10502000000000004822DE0003006200FE62020071
:105030000000000020042000806302000000000047
:10504000D0042000FE6202000000000010042000D6
:10505000FE6202000000000090042000FE620200D8
:1050600000000000E0042000FE62020000000000DA
:1050700000022000FE62020000000000D0042000B8
:10508000FE6202000000000050042000FE620200E8
:1050900000000000E0042000FE62020000000000AA
:1050A00050052000FE62020000000000444920007C
:1050B000600420008063020000000000F30F200065
:1050C00003006200FE620200000000004822DE00D1
:1050D00003006200FE6202000000000020042000C5
:1050E000806302000000000060042000FE620200F5
:1050F0000000000090042000FE620200000000009A
:1051000020052000FE6202000000000030052000A3
:10511000FE6202000000000040052000FE62020066
:105120000000000000022000FE62020000000000FB
:1051300030052000FE620200000000005004200044
:10514000FE62020000000000C0042000FE620200B7
:105150000000000050042000FE6202000000000079
:1051600030042000FE620200000000004005200024
:10517000FE6202000000000000022000FE62020049
:105180000000000090042000FE6202000000000009
:1051900040052000FE6202000000000050042000D4
:1051A000FE62020000000000D0042000FE62020047
:1051B0000000000000022000FE620200000000006B
:1051C00040052000FE62020000000000F004200004
:1051D000FE6202000000000000022000FE620200E9
:1051E0000000000010042000FE6202000000000029
:1051F00040042000FE62020000000000A004200025
:10520000FE6202000000000050052000FE62020065
:105210000000000030052000FE62020000000000D7
:1052200040052000FE620200000000000071220024
:105230003083880090002000108188008E0D0400CB
:105240000000000040C78000310020000100500035
:105250004220AE005E290400000000007E23020010
:105260000000000000712200808188000000200002
:105270009081880000002000A0818800A083800029
:10528000B081880000002000C0818800000020005C
:10529000D0818800787302000000000080818000C7
:1052A00000818800B27C0200000000002000200085
:1052B00010818800CE2904000000000040C7800053
:1052C00011002000010050004220AE0076290400A9
:1052D000000000007E23020000000000E00020002B
:1052E00010818800CE2904000000000040C7800023
:1052F00021002000010050004220AE008E29040051
:10530000000000007E2302000000000000012000D9
:1053100010818800CE2904000000000040C78000F2
:1053200081002000010050004220AE00A6290400A8
:10533000000000007E230200000000002001200089
:1053400010818800CE2904000000000040C78000C2
:1053500071002000010050004220AE00BE29040070
:10536000000000007E230200000000004001200039
:1053700010818800CE290400000000006610E200C1
:105380004220AE00CE2904000000000020002000D2
:1053900010818800CE290400000000008E0D04005A
:1053A00000000000844820006004200080630200A8
:1053B00000000000F30F200003006200FE62020004
:1053C000000000004822DE0003006200FE620200CE
:1053D00000000000200420008063020000000000A4
:1053E00000022000FE620200000000000002200017
:1053F000FE6202000000000000022000FE620200C7
:105400000000000000022000FE6202000000000018
:1054100000022000FE6202000000000000022000E6
:10542000FE6202000000000000022000FE62020096
:105430000000000000022000FE62020000000000E8
:1054400000022000FE62020000000000444920002B
:10545000600420008063020000000000F30F2000C1
:1054600003006200FE620200000000004822DE002D
:1054700003006200FE620200000000002004200021
:10548000806302000000000000022000FE620200B3
:105490000000000000022000FE6202000000000088
:1054A00050052000FE620200000000000005200000
:1054B000FE6202000000000000022000FE62020006
:1054C0000000000000022000FE6202000000000058
:1054D00000022000FE620200000000000002200026
:1054E000FE6202000000000000022000FE620200D6
:1054F0000000000000022000FE6202000000000028
:1055000000022000FE6202000000000000022000F5
:10551000FE6202000000000040042000FE62020063
:1055200000000000F0042000FE6202000000000005
:1055300070052000FE62020000000000E004200070
:10554000FE6202000000000000022000FE62020075
:105550000000000000022000FE62020000000000C7
:1055600000022000FE620200000000000002200095
:10557000FE6202000000000000022000FE62020045
:105580000000000000022000FE6202000000000097
:1055900030052000FE6202000000000040052000EF
:1055A000FE62020000000000F0042000FE62020023
:1055B0000000000020052000FE6202000000000044
:1055C00050042000FE62020000000000F0002000F5
:1055D000108188008E0D04000000000070838000A0
:1055E000E082880000232000008388000000200063
:1055F00010838800FC20020000000000E082800090
:1056000070838800844820006004200080630200CA
:1056100000000000F30F200003006200FE620200A1
:10562000000000004822DE0003006200FE6202006B
:105630000000000020042000806302000000000041
:10564000D0042000FE6202000000000010042000D0
:10565000FE6202000000000090042000FE620200D2
:1056600000000000E0042000FE62020000000000D4
:1056700000022000FE62020000000000D0042000B2
:10568000FE6202000000000050042000FE620200E2
:1056900000000000E0042000FE62020000000000A4
:1056A00050052000FE620200000000004449200076
:1056B000600420008063020000000000F30F20005F
:1056C00003006200FE620200000000004822DE00CB
:1056D00003006200FE6202000000000020042000BF
:1056E000806302000000000060042000FE620200EF
:1056F0000000000090042000FE6202000000000094
:1057000020052000FE62020000000000300520009D
:10571000FE6202000000000040052000FE62020060
:105720000000000000022000FE62020000000000F5
:1057300030052000FE62020000000000500420003E
:10574000FE62020000000000C0042000FE620200B1
:105750000000000050042000FE6202000000000073
:1057600030042000FE62020000000000400520001E
:10577000FE6202000000000000022000FE62020043
:105780000000000090042000FE6202000000000003
:1057900040052000FE6202000000000050042000CE
:1057A000FE62020000000000D0042000FE62020041
:1057B0000000000000022000FE6202000000000065
:1057C00040052000FE62020000000000F0042000FE
:1057D000FE6202000000000000022000FE620200E3
:1057E0000000000010042000FE6202000000000023
:1057F00040042000FE62020000000000A00420001F
:10580000FE6202000000000050052000FE6202005F
:105810000000000030052000FE62020000000000D1
:1058200040052000FE62020000000000007122001E
:105830003083880090002000108188008E0D0400C5
:105840000000000084482000600420008063020003
:1058500000000000F30F200003006200FE6202005F
:10586000000000004822DE0003006200FE62020029
:1058700000000000200420008063020000000000FF
:1058800000022000FE620200000000000002200072
:10589000FE6202000000000000022000FE62020022
:1058A0000000000000022000FE6202000000000074
:1058B00000022000FE620200000000000002200042
:1058C000FE6202000000000000022000FE620200F2
:1058D0000000000000022000FE6202000000000044
:1058E00000022000FE620200000000004449200087
:1058F000600420008063020000000000F30F20001D
:1059000003006200FE620200000000004822DE0088
:1059100003006200FE62020000000000200420007C
:10592000806302000000000000022000FE6202000E
:105930000000000000022000FE62020000000000E3
:1059400050052000FE62020000000000000520005B
:10595000FE6202000000000000022000FE62020061
:105960000000000000022000FE62020000000000B3
:1059700000022000FE620200000000000002200081
:10598000FE6202000000000000022000FE62020031
:105990000000000000022000FE6202000000000083
:1059A00000022000FE620200000000000002200051
:1059B000FE6202000000000040042000FE620200BF
:1059C00000000000F0042000FE6202000000000061
:1059D00070052000FE62020000000000E0042000CC
:1059E000FE6202000000000000022000FE620200D1
:1059F0000000000000022000FE6202000000000023
:105A000000022000FE6202000000000000022000F0
:105A1000FE6202000000000000022000FE620200A0
:105A20000000000000022000FE62020000000000F2
:105A300030052000FE62020000000000400520004A
:105A4000FE62020000000000F0042000FE6202007E
:105A50000000000020052000FE620200000000009F
:105A600050042000FE62020000000000300120000F
:105A7000108188008E0D040000000000608380000B
:105A8000E0828800B027200000838800000020000A
:105A9000108388008E21020000000000E082800058
:105AA0006083880084482000600420008063020036
:105AB00000000000F30F200003006200FE620200FD
:105AC000000000004822DE0003006200FE620200C7
:105AD000000000002004200080630200000000009D
:105AE000D0042000FE62020000000000100420002C
:105AF000FE6202000000000090042000FE6202002E
:105B000000000000E0042000FE620200000000002F
:105B100000022000FE62020000000000D00420000D
:105B2000FE6202000000000050042000FE6202003D
:105B300000000000E0042000FE62020000000000FF
:105B400050052000FE6202000000000044492000D1
:105B5000600420008063020000000000F30F2000BA
:105B600003006200FE620200000000004822DE0026
:105B700003006200FE62020000000000200420001A
:105B8000806302000000000060042000FE6202004A
:105B90000000000090042000FE62020000000000EF
:105BA00020052000FE6202000000000030052000F9
:105BB000FE6202000000000040052000FE620200BC
:105BC0000000000000022000FE6202000000000051
:105BD00030052000FE62020000000000500420009A
:105BE000FE62020000000000C0042000FE6202000D
:105BF0000000000050042000FE62020000000000CF
:105C000030042000FE620200000000004005200079
:105C1000FE6202000000000000022000FE6202009E
:105C20000000000090042000FE620200000000005E
:105C300040052000FE620200000000005004200029
:105C4000FE62020000000000D0042000FE6202009C
:105C50000000000000022000FE62020000000000C0
:105C600040052000FE62020000000000F004200059
:105C7000FE6202000000000000022000FE6202003E
:105C80000000000010042000FE620200000000007E
:105C900040042000FE62020000000000A00420007A
:105CA000FE6202000000000050052000FE620200BB
:105CB0000000000030052000FE620200000000002D
:105CC00040052000FE62020000000000007122007A
:105CD0003083880090002000108188008E0D040021
:105CE000000000008448200060042000806302005F
:105CF00000000000F30F200003006200FE620200BB
:105D0000000000004822DE0003006200FE62020084
:105D1000000000002004200080630200000000005A
:105D200000022000FE6202000000000000022000CD
:105D3000FE6202000000000000022000FE6202007D
:105D40000000000000022000FE62020000000000CF
:105D500000022000FE62020000000000000220009D
:105D6000FE6202000000000000022000FE6202004D
:105D70000000000000022000FE620200000000009F
:105D800000022000FE6202000000000044492000E2
:105D9000600420008063020000000000F30F200078
:105DA00003006200FE620200000000004822DE00E4
:105DB00003006200FE6202000000000020042000D8
:105DC000806302000000000000022000FE6202006A
:105DD0000000000000022000FE620200000000003F
:105DE00050052000FE6202000000000000052000B7
:105DF000FE6202000000000000022000FE620200BD
:105E00000000000000022000FE620200000000000E
:105E100000022000FE6202000000000000022000DC
:105E2000FE6202000000000000022000FE6202008C
:105E30000000000000022000FE62020000000000DE
:105E400000022000FE6202000000000000022000AC
:105E5000FE6202000000000040042000FE6202001A
:105E600000000000F0042000FE62020000000000BC
:105E700070052000FE62020000000000E004200027
:105E8000FE6202000000000000022000FE6202002C
:105E90000000000000022000FE620200000000007E
:105EA00000022000FE62020000000000000220004C
:105EB000FE6202000000000000022000FE620200FC
:105EC0000000000000022000FE620200000000004E
:105ED00030052000FE6202000000000040052000A6
:105EE000FE62020000000000F0042000FE620200DA
:105EF0000000000020052000FE62020000000000FB
:105F000050042000FE62020000000000500120004A
:105F1000108188008E0D040000000000F0808000D9
:105F2000E0828800304320000083880000002000C9
:105F3000108388003C22020000000000E082800004
:105F4000F080880084482000600420008063020004
:105F500000000000F30F200003006200FE62020058
:105F6000000000004822DE0003006200FE62020022
:105F700000000000200420008063020000000000F8
:105F8000D0042000FE620200000000001004200087
:105F9000FE6202000000000090042000FE62020089
:105FA00000000000E0042000FE620200000000008B
:105FB00000022000FE62020000000000D004200069
:105FC000FE6202000000000050042000FE62020099
:105FD00000000000E0042000FE620200000000005B
:105FE00050052000FE62020000000000444920002D
:105FF000600420008063020000000000F30F200016
:1060000003006200FE620200000000004822DE0081
:1060100003006200FE620200000000002004200075
:10602000806302000000000060042000FE620200A5
:106030000000000090042000FE620200000000004A
:1060400020052000FE620200000000003005200054
:10605000FE6202000000000040052000FE62020017
:106060000000000000022000FE62020000000000AC
:1060700030052000FE6202000000000050042000F5
:10608000FE62020000000000C0042000FE62020068
:106090000000000050042000FE620200000000002A
:1060A00030042000FE6202000000000040052000D5
:1060B000FE6202000000000000022000FE620200FA
:1060C0000000000090042000FE62020000000000BA
:1060D00040052000FE620200000000005004200085
:1060E000FE62020000000000D0042000FE620200F8
:1060F0000000000000022000FE620200000000001C
:1061000040052000FE62020000000000F0042000B4
:10611000FE6202000000000000022000FE62020099
:106120000000000010042000FE62020000000000D9
:1061300040042000FE62020000000000A0042000D5
:10614000FE6202000000000050052000FE62020016
:106150000000000030052000FE6202000000000088
:1061600040052000FE6202000000000000712200D5
:106170003083880090002000108188008E0D04007C
:10618000000000005864020000000000B408200075
:10619000600420008063020000000000F30F200074
:1061A00003006200FE620200000000004822DE00E0
:1061B00003006200FE6202000000000020042000D4
:1061C000806302000000000090042000FE620200D4
:1061D0000000000000022000FE620200000000003B
:1061E000D0042000FE620200000000000002200037
:1061F000FE6202000000000000052000FE620200B6
:106200000000000000022000FE620200000000000A
:10621000C0042000FE620200000000000002200016
:10622000FE6202000000000050042000FE62020036
:106230000000000000022000FE62020000000000DA
:10624000D0042000FE6202000000000000022000D6
:10625000FE6202000000000050042000FE62020006
:106260000000000000022000FE62020000000000AA
:10627000E0042000FE620200000000000002200096
:10628000FE6202000000000040052000FE620200E5
:1062900000000000340B2000600420008063020036
:1062A00000000000F30F200003006200FE62020005
:1062B000000000004822DE0003006200FE620200CF
:1062C00000000000200420008063020000000000A5
:1062D000D0022000FE62020000000000D002200078
:1062E000FE62020000000000D0022000FE620200F8
:1062F00000000000D0022000FE620200000000004A
:10630000D0022000FE62020000000000D002200047
:10631000FE62020000000000D0022000FE620200C7
:1063200000000000D0022000FE6202000000000019
:10633000D0022000FE62020000000000D002200017
:10634000FE62020000000000D0022000FE62020097
:1063500000000000D0022000FE62020000000000E9
:10636000D0022000FE62020000000000D0022000E7
:10637000FE62020000000000D0022000FE62020067
:1063800000000000D0022000FE62020000000000B9
:10639000D0022000FE620200000000004410200035
:1063A000600420008063020000000000F30F200062
:1063B00003006200FE620200000000004822DE00CE
:1063C00003006200FE6202000000000020042000C2
:1063D000806302000000000030052000FE62020021
:1063E0000000000000022000FE6202000000000029
:1063F00050042000FE6202000000000000022000A5
:10640000FE6202000000000040052000FE62020063
:106410000000000000022000FE62020000000000F8
:1064200040052000FE620200000000000002200083
:10643000FE6202000000000090042000FE620200E4
:106440000000000000022000FE62020000000000C8
:10645000E0042000FE6202000000000000022000B4
:10646000FE6202000000000070042000FE620200D4
:106470000000000000022000FE6202000000000098
:1064800030052000FE62020000000000C41220005F
:10649000600420008063020000000000F30F200071
:1064A00003006200FE620200000000004822DE00DD
:1064B00003006200FE6202000000000020042000D1
:1064C0008063020000000000D0022000FE62020093
:1064D00000000000D0022000FE6202000000000068
:1064E000D0022000FE62020000000000D002200066
:1064F000FE62020000000000D0022000FE620200E6
:1065000000000000D0022000FE6202000000000037
:10651000D0022000FE62020000000000D002200035
:10652000FE62020000000000D0022000FE620200B5
:1065300000000000D0022000FE6202000000000007
:10654000D0022000FE62020000000000D002200005
:10655000FE62020000000000D0022000FE62020085
:1065600000000000D0022000FE62020000000000D7
:10657000D0022000FE62020000000000840720001C
:10658000600420008063020000000000F30F200080
:1065900003006200FE620200000000004822DE00EC
:1065A00003006200FE6202000000000020042000E0
:1065B00080630200000000008083800080818800EA
:1065C000B66B020000000000C082800001032000C2
:1065D00001004000FE62020000000000D082800046
:1065E0000103200001004000FE62020000000000E4
:1065F00000022000FE620200000000009004200063
:10660000FE62020000000000E0022000FE620200C4
:106610000000000040042000FE62020000000000B4
:10662000E0022000FE6202000000000000022000E4
:10663000FE62020000000000E0042000FE62020092
:1066400000000000F0062000FE62020000000000D2
:10665000042320006004200080630200000000008A
:10666000F30F200003006200FE6202000000000041
:106670004822DE0003006200FE620200000000000B
:10668000200420008063020000000000908380004E
:1066900080818800B66B020000000000C08280008C
:1066A0000103200001004000FE6202000000000023
:1066B000D08280000103200001004000FE62020041
:1066C0000000000000022000FE6202000000000046
:1066D000E0042000FE62020000000000F00620003E
:1066E000FE6202000000000000022000FE620200C4
:1066F00000000000F0042000FE6202000000000024
:1067000060042000FE620200000000000002200081
:10671000FE6202000000000020052000FE62020070
:1067200000000000F0042000FE62020000000000F3
:1067300070052000FE62020000000000300520000D
:10674000FE62020000000000843E20006004200081
:106750008063020000000000F30F200003006200CD
:10676000FE620200000000004822DE00030062001A
:10677000FE6202000000000020042000806302008E
:1067800000000000A083800080818800B66B0200BA
:1067900000000000B08280000103200001004000E2
:1067A000FE62020000000000C082800001032000A1
:1067B00001004000FE62020000000000D082800064
:1067C0000103200001004000FE6202000000000002
:1067D00000022000FE6202000000000020052000F0
:1067E000FE62020000000000F0042000FE620200D1
:1067F0000000000070052000FE62020000000000A2
:1068000000022000FE62020000000000700520006F
:10681000FE6202000000000090042000FE62020000
:106820000000000040042000FE62020000000000A2
:1068300040052000FE6202000000000080042000ED
:10684000FE6202000000000000022000FE62020062
:106850000000000030062000FE6202000000000080
:10686000D0062000FE620200000000001424200078
:10687000600420008063020000000000F30F20008D
:1068800003006200FE620200000000004822DE00F9
:1068900003006200FE6202000000000020042000ED
:1068A000806302000000000000052000FE6202007C
:1068B00000000000C0042000FE6202000000000092
:1068C00010042000FE62020000000000E00420002E
:1068D000FE6202000000000040052000FE6202008F
:1068E0000000000050042000FE62020000000000D2
:1068F00020052000FE6202000000000000022000CF
:10690000FE62020000000000F0022000FE620200B1
:106910000000000000022000FE62020000000000F3
:1069200030042000FE62020000000000500520003C
:10693000FE62020000000000C0042000FE620200AF
:106940000000000040052000FE6202000000000080
:1069500090042000FE62020000000000600520009C
:10696000FE6202000000000010042000FE6202002F
:106970000000000040052000FE6202000000000050
:10698000F0042000FE62020000000000200520004C
:10699000FE6202000000000000022000FE62020011
:1069A00000000000B0838000FE62020000000000D2
:1069B000D43F20006004200080630200000000003B
:1069C000F30F200003006200FE62020000000000DE
:1069D0004822DE0003006200FE62020000000000A8
:1069E0002004200080630200000000004005200019
:1069F000FE6202000000000010042000FE6202009F
:106A000000000000E0042000FE6202000000000020
:106A1000B0042000FE62020000000000000220001E
:106A2000FE6202000000000030042000FE6202004E
:106A30000000000010042000FE62020000000000C0
:106A400000052000FE62020000000000100420008B
:106A5000FE6202000000000030042000FE6202001E
:106A60000000000090042000FE6202000000000010
:106A700040052000FE62020000000000900520009A
:106A8000FE6202000000000000022000FE62020020
:106A900000000000C4422000600420008063020067
:106AA00000000000F30F200003006200FE620200FD
:106AB000000000004822DE0003006200FE620200C7
:106AC000000000002004200080630200000000009D
:106AD000C0042000FE6202000000000090042000BC
:106AE000FE6202000000000040052000FE6202007D
:106AF0000000000020052000FE62020000000000EF
:106B000050042000FE62020000000000300520005A
:106B1000FE6202000000000000022000FE6202008F
:106B200000000000C083800080818800B66B0200F6
:106B300000000000A082800001032000010040004E
:106B4000FE62020000000000B0828000010320000D
:106B500001004000FE62020000000000C0828000D0
:106B60000103200001004000FE620200000000005E
:106B7000D08280000103200001004000FE6202007C
:106B800000000000844820006004200080630200B0
:106B900000000000F30F200003006200FE6202000C
:106BA000000000004822DE0003006200FE620200D6
:106BB00000000000200420008063020000000000AC
:106BC00000022000FE62020000000000000220001F
:106BD000FE6202000000000000022000FE620200CF
:106BE0000000000020042000FE62020000000000FF
:106BF00010042000FE6202000000000030042000AB
:106C0000FE62020000000000B0042000FE620200EC
:106C10000000000000022000FE62020000000000F0
:106C200000022000FE620200000000004449200033
:106C3000600420008063020000000000F30F2000C9
:106C400003006200FE620200000000004822DE0035
:106C500003006200FE620200000000002004200029
:106C6000806302000000000060042000FE62020059
:106C70000000000090042000FE62020000000000FE
:106C800020052000FE620200000000003005200008
:106C9000FE6202000000000040052000FE620200CB
:106CA0000000000000022000FE6202000000000060
:106CB00030052000FE6202000000000050042000A9
:106CC000FE62020000000000C0042000FE6202001C
:106CD0000000000050042000FE62020000000000DE
:106CE00030042000FE620200000000004005200089
:106CF000FE6202000000000000022000FE620200AE
:106D00000000000090042000FE620200000000006D
:106D100040052000FE620200000000005004200038
:106D2000FE62020000000000D0042000FE620200AB
:106D30000000000000022000FE62020000000000CF
:106D400040052000FE62020000000000F004200068
:106D5000FE6202000000000000022000FE6202004D
:106D60000000000010042000FE620200000000008D
:106D700040042000FE62020000000000A004200089
:106D8000FE6202000000000050052000FE620200CA
:106D90000000000030052000FE620200000000003C
:106DA00040052000FE620200000000000071220089
:106DB0003083880010012000108188008E0D0400AF
:106DC0000000000040C7800031002000010050009A
:106DD0004220AE00FA360400000000007E230200CC
:106DE000000000008000200010818800823704002D
:106DF0000000000040C7800001002000010050009A
:106E00004220AE0012370400000000007E23020082
:106E1000000000006001200010818800823704001B
:106E20000000000040C78000110020000100500059
:106E30004220AE002A370400000000007E2302003A
:106E400000000000800120001081880082370400CB
:106E50000000000040C78000210020000100500019
:106E60004220AE0042370400000000007E230200F2
:106E700000000000A001200010818800823704007B
:106E80000000000040C78000810020000100500089
:106E90004220AE005A370400000000007E230200AA
:106EA00000000000C001200010818800823704002B
:106EB0000000000040C78000710020000100500069
:106EC0004220AE0072370400000000007E23020062
:106ED00000000000E00120001081880082370400DB
:106EE000000000006610E2004220AE00823704007D
:106EF000000000008000200010818800823704001C
:106F0000000000008E0D04000000000084482000F6
:106F1000600420008063020000000000F30F2000E6
:106F200003006200FE620200000000004822DE0052
:106F300003006200FE620200000000002004200046
:106F4000806302000000000000022000FE620200D8
:106F50000000000000022000FE62020000000000AD
:106F600000022000FE62020000000000000220007B
:106F7000FE6202000000000000022000FE6202002B
:106F80000000000000022000FE620200000000007D
:106F900000022000FE62020000000000000220004B
:106FA000FE6202000000000000022000FE620200FB
:106FB00000000000444920006004200080630200BB
:106FC00000000000F30F200003006200FE620200D8
:106FD000000000004822DE0003006200FE620200A2
:106FE0000000000020042000806302000000000078
:106FF00000022000FE6202000000000000022000EB
:10700000FE6202000000000050052000FE62020047
:107010000000000000052000FE62020000000000E9
:1070200000022000FE6202000000000000022000BA
:10703000FE6202000000000000022000FE6202006A
:107040000000000000022000FE62020000000000BC
:1070500000022000FE62020000000000000220008A
:10706000FE6202000000000000022000FE6202003A
:107070000000000000022000FE620200000000008C
:1070800040042000FE62020000000000F004200026
:10709000FE6202000000000070052000FE62020097
:1070A00000000000E0042000FE620200000000007A
:1070B00000022000FE62020000000000000220002A
:1070C000FE6202000000000000022000FE620200DA
:1070D0000000000000022000FE620200000000002C
:1070E00000022000FE6202000000000000022000FA
:1070F000FE6202000000000030052000FE62020077
:107100000000000040052000FE62020000000000B8
:10711000F0042000FE6202000000000020052000B4
:10712000FE6202000000000050042000FE62020027
:107130000000000070012000108188008E0D040006
:107140000000000080838000E0828800800720002B
:107150000083880000002000108388008620020041
:1071600000000000E08280008083880084482000C6
:10717000600420008063020000000000F30F200084
:1071800003006200FE620200000000004822DE00F0
:1071900003006200FE6202000000000020042000E4
:1071A000806302000000000000022000FE62020076
:1071B0000000000000022000FE620200000000004B
:1071C00000022000FE6202000000000020042000F7
:1071D000FE6202000000000010042000FE620200B7
:1071E0000000000030042000FE62020000000000E9
:1071F000B0042000FE620200000000000002200037
:10720000FE6202000000000000022000FE62020098
:107210000000000044492000600420008063020058
:1072200000000000F30F200003006200FE62020075
:10723000000000004822DE0003006200FE6202003F
:107240000000000020042000806302000000000015
:1072500060042000FE620200000000009004200094
:10726000FE6202000000000020052000FE62020015
:107270000000000030052000FE6202000000000057
:1072800040052000FE620200000000000002200015
:10729000FE6202000000000030052000FE620200D5
:1072A0000000000050042000FE6202000000000008
:1072B000C0042000FE620200000000005004200014
:1072C000FE6202000000000030042000FE620200A6
:1072D0000000000040052000FE62020000000000E7
:1072E00000022000FE620200000000009004200066
:1072F000FE6202000000000040052000FE62020065
:107300000000000050042000FE62020000000000A7
:10731000D0042000FE6202000000000000022000F5
:10732000FE6202000000000040052000FE62020034
:1073300000000000F0042000FE62020000000000D7
:1073400000022000FE620200000000001004200085
:10735000FE6202000000000040042000FE62020005
:1073600000000000A0042000FE62020000000000F7
:1073700050052000FE6202000000000030052000E1
:10738000FE6202000000000040052000FE620200D4
:1073900000000000007122003083880010012000EE
:1073A000108188008E0D0400000000008448200039
:1073B000600420008063020000000000F30F200042
:1073C00003006200FE620200000000004822DE00AE
:1073D00003006200FE6202000000000020042000A2
:1073E000806302000000000000022000FE62020034
:1073F0000000000000022000FE6202000000000009
:1074000000022000FE6202000000000000022000D6
:10741000FE6202000000000000022000FE62020086
:107420000000000000022000FE62020000000000D8
:1074300000022000FE6202000000000000022000A6
:10744000FE6202000000000000022000FE62020056
:107450000000000044492000600420008063020016
:1074600000000000F30F200003006200FE62020033
:10747000000000004822DE0003006200FE620200FD
:1074800000000000200420008063020000000000D3
:1074900000022000FE620200000000000002200046
:1074A000FE6202000000000050052000FE620200A3
:1074B0000000000000052000FE6202000000000045
:1074C00000022000FE620200000000000002200016
:1074D000FE6202000000000000022000FE620200C6
:1074E0000000000000022000FE6202000000000018
:1074F00000022000FE6202000000000000022000E6
:10750000FE6202000000000000022000FE62020095
:107510000000000000022000FE62020000000000E7
:1075200040042000FE62020000000000F004200081
:10753000FE6202000000000070052000FE620200F2
:1075400000000000E0042000FE62020000000000D5
:1075500000022000FE620200000000000002200085
:10756000FE6202000000000000022000FE62020035
:107570000000000000022000FE6202000000000087
:1075800000022000FE620200000000000002200055
:10759000FE6202000000000030052000FE620200D2
:1075A0000000000040052000FE6202000000000014
:1075B000F0042000FE620200000000002005200010
:1075C000FE6202000000000050042000FE62020083
:1075D0000000000090012000108188008E0D040042
:1075E0000000000090838000E082880000232000DB
:1075F000008388000000200010838800862002009D
:1076000000000000E0828000908388008448200011
:10761000600420008063020000000000F30F2000DF
:1076200003006200FE620200000000004822DE004B
:1076300003006200FE62020000000000200420003F
:10764000806302000000000000022000FE620200D1
:107650000000000000022000FE62020000000000A6
:1076600000022000FE620200000000002004200052
:10767000FE6202000000000010042000FE62020012
:107680000000000030042000FE6202000000000044
:10769000B0042000FE620200000000000002200092
:1076A000FE6202000000000000022000FE620200F4
:1076B00000000000444920006004200080630200B4
:1076C00000000000F30F200003006200FE620200D1
:1076D000000000004822DE0003006200FE6202009B
:1076E0000000000020042000806302000000000071
:1076F00060042000FE6202000000000090042000F0
:10770000FE6202000000000020052000FE62020070
:107710000000000030052000FE62020000000000B2
:1077200040052000FE620200000000000002200070
:10773000FE6202000000000030052000FE62020030
:107740000000000050042000FE6202000000000063
:10775000C0042000FE62020000000000500420006F
:10776000FE6202000000000030042000FE62020001
:107770000000000040052000FE6202000000000042
:1077800000022000FE6202000000000090042000C1
:10779000FE6202000000000040052000FE620200C0
:1077A0000000000050042000FE6202000000000003
:1077B000D0042000FE620200000000000002200051
:1077C000FE6202000000000040052000FE62020090
:1077D00000000000F0042000FE6202000000000033
:1077E00000022000FE6202000000000010042000E1
:1077F000FE6202000000000040042000FE62020061
:1078000000000000A0042000FE6202000000000052
:1078100050052000FE62020000000000300520003C
:10782000FE6202000000000040052000FE6202002F
:107830000000000000712200308388001001200049
:10784000108188008E0D0400000000008448200094
:10785000600420008063020000000000F30F20009D
:1078600003006200FE620200000000004822DE0009
:1078700003006200FE6202000000000020042000FD
:10788000806302000000000000022000FE6202008F
:107890000000000000022000FE6202000000000064
:1078A00000022000FE620200000000000002200032
:1078B000FE6202000000000000022000FE620200E2
:1078C0000000000000022000FE6202000000000034
:1078D00000022000FE620200000000000002200002
:1078E000FE6202000000000000022000FE620200B2
:1078F0000000000044492000600420008063020072
:1079000000000000F30F200003006200FE6202008E
:10791000000000004822DE0003006200FE62020058
:10792000000000002004200080630200000000002E
:1079300000022000FE6202000000000000022000A1
:10794000FE6202000000000050052000FE620200FE
:107950000000000000052000FE62020000000000A0
:1079600000022000FE620200000000000002200071
:10797000FE6202000000000000022000FE62020021
:107980000000000000022000FE6202000000000073
:1079900000022000FE620200000000000002200041
:1079A000FE6202000000000000022000FE620200F1
:1079B0000000000000022000FE6202000000000043
:1079C00040042000FE62020000000000F0042000DD
:1079D000FE6202000000000070052000FE6202004E
:1079E00000000000E0042000FE6202000000000031
:1079F00000022000FE6202000000000000022000E1
:107A0000FE6202000000000000022000FE62020090
:107A10000000000000022000FE62020000000000E2
:107A200000022000FE6202000000000000022000B0
:107A3000FE6202000000000030052000FE6202002D
:107A40000000000040052000FE620200000000006F
:107A5000F0042000FE62020000000000200520006B
:107A6000FE6202000000000050042000FE620200DE
:107A700000000000B0012000108188008E0D04007D
:107A800000000000A0838000E0828800803E20008B
:107A9000008388000000200010838800FC20020082
:107AA00000000000E0828000A0838800844820005D
:107AB000600420008063020000000000F30F20003B
:107AC00003006200FE620200000000004822DE00A7
:107AD00003006200FE62020000000000200420009B
:107AE000806302000000000000022000FE6202002D
:107AF0000000000000022000FE6202000000000002
:107B000000022000FE6202000000000020042000AD
:107B1000FE6202000000000010042000FE6202006D
:107B20000000000030042000FE620200000000009F
:107B3000B0042000FE6202000000000000022000ED
:107B4000FE6202000000000000022000FE6202004F
:107B5000000000004449200060042000806302000F
:107B600000000000F30F200003006200FE6202002C
:107B7000000000004822DE0003006200FE620200F6
:107B800000000000200420008063020000000000CC
:107B900060042000FE62020000000000900420004B
:107BA000FE6202000000000020052000FE620200CC
:107BB0000000000030052000FE620200000000000E
:107BC00040052000FE6202000000000000022000CC
:107BD000FE6202000000000030052000FE6202008C
:107BE0000000000050042000FE62020000000000BF
:107BF000C0042000FE6202000000000050042000CB
:107C0000FE6202000000000030042000FE6202005C
:107C10000000000040052000FE620200000000009D
:107C200000022000FE62020000000000900420001C
:107C3000FE6202000000000040052000FE6202001B
:107C40000000000050042000FE620200000000005E
:107C5000D0042000FE6202000000000000022000AC
:107C6000FE6202000000000040052000FE620200EB
:107C700000000000F0042000FE620200000000008E
:107C800000022000FE62020000000000100420003C
:107C9000FE6202000000000040042000FE620200BC
:107CA00000000000A0042000FE62020000000000AE
:107CB00050052000FE620200000000003005200098
:107CC000FE6202000000000040052000FE6202008B
:107CD00000000000007122003083880010012000A5
:107CE000108188008E0D04000000000084482000F0
:107CF000600420008063020000000000F30F2000F9
:107D000003006200FE620200000000004822DE0064
:107D100003006200FE620200000000002004200058
:107D2000806302000000000000022000FE620200EA
:107D30000000000000022000FE62020000000000BF
:107D400000022000FE62020000000000000220008D
:107D5000FE6202000000000000022000FE6202003D
:107D60000000000000022000FE620200000000008F
:107D700000022000FE62020000000000000220005D
:107D8000FE6202000000000000022000FE6202000D
:107D900000000000444920006004200080630200CD
:107DA00000000000F30F200003006200FE620200EA
:107DB000000000004822DE0003006200FE620200B4
:107DC000000000002004200080630200000000008A
:107DD00000022000FE6202000000000000022000FD
:107DE000FE6202000000000050052000FE6202005A
:107DF0000000000000052000FE62020000000000FC
:107E000000022000FE6202000000000000022000CC
:107E1000FE6202000000000000022000FE6202007C
:107E20000000000000022000FE62020000000000CE
:107E300000022000FE62020000000000000220009C
:107E4000FE6202000000000000022000FE6202004C
:107E50000000000000022000FE620200000000009E
:107E600040042000FE62020000000000F004200038
:107E7000FE6202000000000070052000FE620200A9
:107E800000000000E0042000FE620200000000008C
:107E900000022000FE62020000000000000220003C
:107EA000FE6202000000000000022000FE620200EC
:107EB0000000000000022000FE620200000000003E
:107EC00000022000FE62020000000000000220000C
:107ED000FE6202000000000030052000FE62020089
:107EE0000000000040052000FE62020000000000CB
:107EF000F0042000FE6202000000000020052000C7
:107F0000FE6202000000000050042000FE62020039
:107F100000000000D0012000108188008E0D0400B8
:107F200000000000844820006004200080630200FC
:107F300000000000F30F200003006200FE62020058
:107F4000000000004822DE0003006200FE62020022
:107F500000000000200420008063020000000000F8
:107F600000022000FE62020000000000000220006B
:107F7000FE6202000000000000022000FE6202001B
:107F80000000000020042000FE620200000000004B
:107F900010042000FE6202000000000030042000F7
:107FA000FE62020000000000B0042000FE62020039
:107FB0000000000000022000FE620200000000003D
:107FC00000022000FE620200000000004449200080
:107FD000600420008063020000000000F30F200016
:107FE00003006200FE620200000000004822DE0082
:107FF00003006200FE620200000000002004200076
:10800000806302000000000060042000FE620200A5
:108010000000000090042000FE620200000000004A
:1080200020052000FE620200000000003005200054
:10803000FE6202000000000040052000FE62020017
:108040000000000000022000FE62020000000000AC
:1080500030052000FE6202000000000050042000F5
:10806000FE62020000000000C0042000FE62020068
:108070000000000050042000FE620200000000002A
:1080800030042000FE6202000000000040052000D5
:10809000FE6202000000000000022000FE620200FA
:1080A0000000000090042000FE62020000000000BA
:1080B00040052000FE620200000000005004200085
:1080C000FE62020000000000D0042000FE620200F8
:1080D0000000000000022000FE620200000000001C
:1080E00040052000FE62020000000000F0042000B5
:1080F000FE6202000000000000022000FE6202009A
:108100000000000010042000FE62020000000000D9
:1081100040042000FE62020000000000A0042000D5
:10812000FE6202000000000050052000FE62020016
:108130000000000030052000FE6202000000000088
:1081400040052000FE6202000000000000712200D5
:108150003083880010012000108188008E0D0400FB
:1081600000000000844820006004200080630200BA
:1081700000000000F30F200003006200FE62020016
:10818000000000004822DE0003006200FE620200E0
:1081900000000000200420008063020000000000B6
:1081A00000022000FE620200000000000002200029
:1081B000FE6202000000000000022000FE620200D9
:1081C0000000000000022000FE620200000000002B
:1081D00000022000FE6202000000000000022000F9
:1081E000FE6202000000000000022000FE620200A9
:1081F0000000000000022000FE62020000000000FB
:1082000000022000FE62020000000000444920003D
:10821000600420008063020000000000F30F2000D3
:1082200003006200FE620200000000004822DE003F
:1082300003006200FE620200000000002004200033
:10824000806302000000000000022000FE620200C5
:108250000000000000022000FE620200000000009A
:1082600050052000FE620200000000000005200012
:10827000FE6202000000000000022000FE62020018
:108280000000000000022000FE620200000000006A
:1082900000022000FE620200000000000002200038
:1082A000FE6202000000000000022000FE620200E8
:1082B0000000000000022000FE620200000000003A
:1082C00000022000FE620200000000000002200008
:1082D000FE6202000000000040042000FE62020076
:1082E00000000000F0042000FE6202000000000018
:1082F00070052000FE62020000000000E004200083
:10830000FE6202000000000000022000FE62020087
:108310000000000000022000FE62020000000000D9
:1083200000022000FE6202000000000000022000A7
:10833000FE6202000000000000022000FE62020057
:108340000000000000022000FE62020000000000A9
:1083500030052000FE620200000000004005200001
:10836000FE62020000000000F0042000FE62020035
:108370000000000020052000FE6202000000000056
:1083800050042000FE62020000000000F001200006
:10839000108188008E0D040000000000C083800062
:1083A000E082880030432000008388000000200025
:1083B000108388008E21020000000000E08280000F
:1083C000C08388008448200060042000806302008D
:1083D00000000000F30F200003006200FE620200B4
:1083E000000000004822DE0003006200FE6202007E
:1083F0000000000020042000806302000000000054
:1084000000022000FE6202000000000000022000C6
:10841000FE6202000000000000022000FE62020076
:108420000000000020042000FE62020000000000A6
:1084300010042000FE620200000000003004200052
:10844000FE62020000000000B0042000FE62020094
:108450000000000000022000FE6202000000000098
:1084600000022000FE6202000000000044492000DB
:10847000600420008063020000000000F30F200071
:1084800003006200FE620200000000004822DE00DD
:1084900003006200FE6202000000000020042000D1
:1084A000806302000000000060042000FE62020001
:1084B0000000000090042000FE62020000000000A6
:1084C00020052000FE6202000000000030052000B0
:1084D000FE6202000000000040052000FE62020073
:1084E0000000000000022000FE6202000000000008
:1084F00030052000FE620200000000005004200051
:10850000FE62020000000000C0042000FE620200C3
:108510000000000050042000FE6202000000000085
:1085200030042000FE620200000000004005200030
:10853000FE6202000000000000022000FE62020055
:108540000000000090042000FE6202000000000015
:1085500040052000FE6202000000000050042000E0
:10856000FE62020000000000D0042000FE62020053
:108570000000000000022000FE6202000000000077
:1085800040052000FE62020000000000F004200010
:10859000FE6202000000000000022000FE620200F5
:1085A0000000000010042000FE6202000000000035
:1085B00040042000FE62020000000000A004200031
:1085C000FE6202000000000050052000FE62020072
:1085D0000000000030052000FE62020000000000E4
:1085E00040052000FE620200000000000071220031
:1085F0003083880010012000108188008E0D040057
:10860000000000005864020000000000B4072000D1
:10861000600420008063020000000000F30F2000CF
:1086200003006200FE620200000000004822DE003B
:1086300003006200FE62020000000000200420002F
:10864000806302000000000030042000FE6202008F
:108650000000000000022000FE6202000000000096
:1086600010042000FE620200000000000002200052
:10867000FE62020000000000C0042000FE62020052
:108680000000000000022000FE6202000000000066
:1086900090042000FE6202000000000000022000A2
:1086A000FE6202000000000020042000FE620200C2
:1086B0000000000000022000FE6202000000000036
:1086C00020052000FE6202000000000000022000E1
:1086D000FE6202000000000010042000FE620200A2
:1086E0000000000000022000FE6202000000000006
:1086F00040052000FE620200000000000002200091
:10870000FE6202000000000090042000FE620200F1
:108710000000000000022000FE62020000000000D5
:10872000F0042000FE6202000000000000022000B1
:10873000FE62020000000000E0042000FE62020071
:1087400000000000340A2000600420008063020062
:1087500000000000F30F200003006200FE62020030
:10876000000000004822DE0003006200FE620200FA
:1087700000000000200420008063020000000000D0
:10878000D0022000FE62020000000000D0022000A3
:10879000FE62020000000000D0022000FE62020023
:1087A00000000000D0022000FE6202000000000075
:1087B000D0022000FE62020000000000D002200073
:1087C000FE62020000000000D0022000FE620200F3
:1087D00000000000D0022000FE6202000000000045
:1087E000D0022000FE62020000000000D002200043
:1087F000FE62020000000000D0022000FE620200C3
:1088000000000000D0022000FE6202000000000014
:10881000D0022000FE62020000000000D002200012
:10882000FE62020000000000D0022000FE62020092
:1088300000000000D0022000FE62020000000000E4
:10884000D0022000FE62020000000000D0022000E2
:10885000FE62020000000000D0022000FE62020062
:1088600000000000D0022000FE62020000000000B4
:10887000D0022000FE62020000000000042320005D
:10888000600420008063020000000000F30F20005D
:1088900003006200FE620200000000004822DE00C9
:1088A00003006200FE6202000000000020042000BD
:1088B000806302000000000020052000FE6202002C
:1088C0000000000050062000FE62020000000000D0
:1088D00030072000FE620200000000005006200069
:1088E000FE6202000000000040072000FE6202005D
:1088F0000000000084252000600420008063020046
:1089000000000000F30F200003006200FE6202007E
:10891000000000004822DE0003006200FE62020048
:10892000000000002004200080630200000000001E
:10893000F0042000FE62020000000000400620005B
:10894000FE62020000000000F0062000FE6202004D
:1089500000000000D0062000FE62020000000000BF
:1089600050062000FE6202000000000040072000C8
:10897000FE6202000000000050062000FE620200BD
:108980000000000020072000FE620200000000003E
:10899000D424200060042000806302000000000056
:1089A000F30F200003006200FE62020000000000DE
:1089B0004822DE0003006200FE62020000000000A8
:1089C0002004200080630200000000003005200029
:1089D000FE6202000000000000052000FE620200AE
:1089E0000000000050042000FE62020000000000B1
:1089F00050042000FE62020000000000400420003D
:108A0000FE62020000000000242720006004200015
:108A10008063020000000000F30F200003006200EA
:108A2000FE620200000000004822DE000300620037
:108A3000FE620200000000002004200080630200AB
:108A400000000000D0062000FE62020000000000CE
:108A5000D0062000FE62020000000000F0022000AC
:108A6000FE6202000000000000072000FE6202001B
:108A70000000000050072000FE620200000000001D
:108A8000C0062000FE620200000000003007200047
:108A9000FE6202000000000050062000FE6202009C
:108AA0000000000000022000FE6202000000000042
:108AB000E080800080818800B66B0200000000002A
:108AC000A08280000103200001004000FE6202003D
:108AD00000000000B082800001032000010040007F
:108AE000FE62020000000000C0828000010320003E
:108AF00001004000FE62020000000000D082800001
:108B00000103200001004000FE620200000000009E
:108B10005440200060042000806302000000000038
:108B2000F30F200003006200FE620200000000005C
:108B30004822DE0003006200FE6202000000000026
:108B400020042000806302000000000030052000A7
:108B5000FE6202000000000000052000FE6202002C
:108B60000000000050042000FE620200000000002F
:108B700050042000FE6202000000000040042000BB
:108B8000FE62020000000000D442200060042000C9
:108B90008063020000000000F30F20000300620069
:108BA000FE620200000000004822DE0003006200B6
:108BB000FE6202000000000020042000806302002A
:108BC0000000000030052000FE62020000000000EE
:108BD000C0062000FE620200000000001006200017
:108BE000FE6202000000000060072000FE6202003A
:108BF0000000000050062000FE620200000000009D
:108C000000022000FE6202000000000000022000BE
:108C1000FE6202000000000000022000FE6202006E
:108C200000000000008480000000E80080818800CF
:108C3000B66B020000000000C0828000010320002B
:108C400001004000FE62020000000000D0828000AF
:108C50000103200001004000FE620200000000004D
:108C600084482000600420008063020000000000AF
:108C7000F30F200003006200FE620200000000000B
:108C80004822DE0003006200FE62020000000000D5
:108C9000200420008063020000000000D0042000B7
:108CA000FE6202000000000010042000FE620200CC
:108CB0000000000090042000FE620200000000009E
:108CC000E0042000FE62020000000000000220001C
:108CD000FE62020000000000D0042000FE620200DC
:108CE0000000000050042000FE62020000000000AE
:108CF000E0042000FE620200000000005005200099
:108D0000FE620200000000004449200060042000D0
:108D10008063020000000000F30F200003006200E7
:108D2000FE620200000000004822DE000300620034
:108D3000FE620200000000002004200080630200A8
:108D40000000000060042000FE620200000000003D
:108D500090042000FE6202000000000020052000B8
:108D6000FE6202000000000030052000FE620200EA
:108D70000000000040052000FE620200000000002C
:108D800000022000FE62020000000000300520000A
:108D9000FE6202000000000050042000FE6202009B
:108DA00000000000C0042000FE620200000000007D
:108DB00050042000FE620200000000003004200089
:108DC000FE6202000000000040052000FE6202007A
:108DD0000000000000022000FE620200000000000F
:108DE00090042000FE620200000000004005200008
:108DF000FE6202000000000050042000FE6202003B
:108E000000000000D0042000FE620200000000000C
:108E100000022000FE620200000000004005200069
:108E2000FE62020000000000F0042000FE6202006A
:108E30000000000000022000FE62020000000000AE
:108E400010042000FE620200000000004004200028
:108E5000FE62020000000000A0042000FE6202008A
:108E60000000000050052000FE620200000000002B
:108E700030052000FE6202000000000040052000D6
:108E8000FE620200000000000071220030838800B2
:108E9000D0002000108188008E0D0400000000002A
:108EA00040C7800031002000010050004220AE0089
:108EB0006C470400000000007E2302000000000058
:108EC000B27C020000000000200020001081880019
:108ED000B84704000000000040C780008100200067
:108EE000010050004220AE00844704000000000052
:108EF0007E23020000000000000220001081880094
:108F0000B84704000000000040C7800011002000A6
:108F1000010050004220AE00A04704000000000005
:108F20007E230200000000007C30EF007E30EF0066
:108F3000B27C020000000000B847040000000000FE
:108F400040C7800071002000010050004220AE00A8
:108F5000B8470400000000007E230200000000006B
:108F60004002200010818800B84704000000000083
:108F70008E0D0400000000008448200060042000E2
:108F80008063020000000000F30F20000300620075
:108F9000FE620200000000004822DE0003006200C2
:108FA000FE62020000000000200420008063020036
:108FB0000000000000022000FE620200000000002D
:108FC00000022000FE6202000000000000022000FB
:108FD000FE6202000000000000022000FE620200AB
:108FE0000000000000022000FE62020000000000FD
:108FF00000022000FE6202000000000000022000CB
:10900000FE6202000000000000022000FE6202007A
:109010000000000000022000FE62020000000000CC
:10902000444920006004200080630200000000002A
:10903000F30F200003006200FE6202000000000047
:109040004822DE0003006200FE6202000000000011
:1090500020042000806302000000000000022000C5
:10906000FE6202000000000000022000FE6202001A
:109070000000000050052000FE6202000000000019
:1090800000052000FE620200000000000002200037
:10909000FE6202000000000000022000FE620200EA
:1090A0000000000000022000FE620200000000003C
:1090B00000022000FE62020000000000000220000A
:1090C000FE6202000000000000022000FE620200BA
:1090D0000000000000022000FE620200000000000C
:1090E00000022000FE620200000000004004200098
:1090F000FE62020000000000F0042000FE62020098
:109100000000000070052000FE6202000000000068
:10911000E0042000FE6202000000000000022000C7
:10912000FE6202000000000000022000FE62020059
:109130000000000000022000FE62020000000000AB
:1091400000022000FE620200000000000002200079
:10915000FE6202000000000000022000FE62020029
:109160000000000030052000FE6202000000000048
:1091700040052000FE62020000000000F004200014
:10918000FE6202000000000020052000FE620200D6
:109190000000000050042000FE62020000000000F9
:1091A00010022000108188008E0D040000000000D5
:1091B000E0808000E0828800B027200000838800E3
:1091C00000002000108388008E21020000000000B3
:1091D000E0828000E0808800844820006004200055
:1091E0008063020000000000F30F20000300620013
:1091F000FE620200000000004822DE000300620060
:10920000FE620200000000002004200080630200D3
:1092100000000000D0042000FE62020000000000F8
:1092200010042000FE6202000000000090042000F4
:10923000FE62020000000000E0042000FE62020066
:109240000000000000022000FE620200000000009A
:10925000D0042000FE620200000000005004200044
:10926000FE62020000000000E0042000FE62020036
:109270000000000050052000FE6202000000000017
:1092800044492000600420008063020000000000C8
:10929000F30F200003006200FE62020000000000E5
:1092A0004822DE0003006200FE62020000000000AF
:1092B0002004200080630200000000006004200001
:1092C000FE6202000000000090042000FE62020026
:1092D0000000000020052000FE62020000000000E7
:1092E00030052000FE620200000000004005200062
:1092F000FE6202000000000000022000FE62020088
:109300000000000030052000FE62020000000000A6
:1093100050042000FE62020000000000C004200093
:10932000FE6202000000000050042000FE62020005
:109330000000000030042000FE6202000000000077
:1093400040052000FE620200000000000002200034
:10935000FE6202000000000090042000FE62020095
:109360000000000040052000FE6202000000000036
:1093700050042000FE62020000000000D004200023
:10938000FE6202000000000000022000FE620200F7
:109390000000000040052000FE6202000000000006
:1093A000F0042000FE620200000000000002200025
:1093B000FE6202000000000010042000FE620200B5
:1093C0000000000040042000FE62020000000000D7
:1093D000A0042000FE6202000000000050052000F2
:1093E000FE6202000000000030052000FE62020064
:1093F0000000000040052000FE62020000000000A6
:109400000071220030838800D00020001081880085
:109410008E0D04000000000084482000600420003D
:109420008063020000000000F30F200003006200D0
:10943000FE620200000000004822DE00030062001D
:10944000FE62020000000000200420008063020091
:109450000000000000022000FE6202000000000088
:1094600000022000FE620200000000000002200056
:10947000FE6202000000000000022000FE62020006
:109480000000000000022000FE6202000000000058
:1094900000022000FE620200000000000002200026
:1094A000FE6202000000000000022000FE620200D6
:1094B0000000000000022000FE6202000000000028
:1094C0004449200060042000806302000000000086
:1094D000F30F200003006200FE62020000000000A3
:1094E0004822DE0003006200FE620200000000006D
:1094F0002004200080630200000000000002200021
:10950000FE6202000000000000022000FE62020075
:109510000000000050052000FE6202000000000074
:1095200000052000FE620200000000000002200092
:10953000FE6202000000000000022000FE62020045
:109540000000000000022000FE6202000000000097
:1095500000022000FE620200000000000002200065
:10956000FE6202000000000000022000FE62020015
:109570000000000000022000FE6202000000000067
:1095800000022000FE6202000000000040042000F3
:10959000FE62020000000000F0042000FE620200F3
:1095A0000000000070052000FE62020000000000C4
:1095B000E0042000FE620200000000000002200023
:1095C000FE6202000000000000022000FE620200B5
:1095D0000000000000022000FE6202000000000007
:1095E00000022000FE6202000000000000022000D5
:1095F000FE6202000000000000022000FE62020085
:109600000000000030052000FE62020000000000A3
:1096100040052000FE62020000000000F00420006F
:10962000FE6202000000000020052000FE62020031
:109630000000000050042000FE6202000000000054
:1096400050022000108188008E0D040000000000F0
:10965000008480000000E800E08288005043200081
:10966000008388000000200010838800862002000C
:1096700000000000E08280000000E9000084880013
:109680008448200060042000806302000000000085
:10969000F30F200003006200FE62020000000000E1
:1096A0004822DE0003006200FE62020000000000AB
:1096B000200420008063020000000000D00420008D
:1096C000FE6202000000000010042000FE620200A2
:1096D0000000000090042000FE6202000000000074
:1096E000E0042000FE6202000000000000022000F2
:1096F000FE62020000000000D0042000FE620200B2
:109700000000000050042000FE6202000000000083
:10971000E0042000FE62020000000000500520006E
:10972000FE620200000000004449200060042000A6
:109730008063020000000000F30F200003006200BD
:10974000FE620200000000004822DE00030062000A
:10975000FE6202000000000020042000806302007E
:109760000000000060042000FE6202000000000013
:1097700090042000FE62020000000000200520008E
:10978000FE6202000000000030052000FE620200C0
:109790000000000040052000FE6202000000000002
:1097A00000022000FE6202000000000030052000E0
:1097B000FE6202000000000050042000FE62020071
:1097C00000000000C0042000FE6202000000000053
:1097D00050042000FE62020000000000300420005F
:1097E000FE6202000000000040052000FE62020050
:1097F0000000000000022000FE62020000000000E5
:1098000090042000FE6202000000000040052000DD
:10981000FE6202000000000050042000FE62020010
:1098200000000000D0042000FE62020000000000E2
:1098300000022000FE62020000000000400520003F
:10984000FE62020000000000F0042000FE62020040
:109850000000000000022000FE6202000000000084
:1098600010042000FE6202000000000040042000FE
:10987000FE62020000000000A0042000FE62020060
:109880000000000050052000FE6202000000000001
:1098900030052000FE6202000000000040052000AC
:1098A000FE62020000000000007122003083880088
:1098B000D0002000108188008E0D04000000000000
:1098C0005864020000000000E41120006004200041
:1098D0008063020000000000F30F2000030062001C
:1098E000FE620200000000004822DE000300620069
:1098F000FE620200000000002004200080630200DD
:109900000000000000052000FE62020000000000D0
:1099100000022000FE62020000000000F0042000AF
:10992000FE6202000000000000022000FE62020051
:109930000000000070052000FE6202000000000030
:1099400000022000FE62020000000000500420001F
:10995000FE6202000000000000022000FE62020021
:109960000000000020052000FE6202000000000050
:1099700000022000FE620200000000000002200041
:10998000FE6202000000000000022000FE620200F1
:1099900000000000F0042000FE6202000000000051
:1099A00000022000FE6202000000000060042000AF
:1099B000FE6202000000000000022000FE620200C1
:1099C0000000000060042000FE62020000000000B1
:1099D0006414200060042000806302000000000086
:1099E000F30F200003006200FE620200000000008E
:1099F0004822DE0003006200FE6202000000000058
:109A0000200420008063020000000000D00220003B
:109A1000FE62020000000000D0022000FE62020090
:109A200000000000D0022000FE62020000000000E2
:109A3000D0022000FE62020000000000D0022000E0
:109A4000FE62020000000000D0022000FE62020060
:109A500000000000D0022000FE62020000000000B2
:109A6000D0022000FE62020000000000D0022000B0
:109A7000FE62020000000000D0022000FE62020030
:109A800000000000D0022000FE6202000000000082
:109A9000D0022000FE62020000000000D002200080
:109AA000FE62020000000000D0022000FE62020000
:109AB00000000000D0022000FE6202000000000052
:109AC000D0022000FE62020000000000D002200050
:109AD000FE62020000000000042320006004200059
:109AE0008063020000000000F30F2000030062000A
:109AF000FE620200000000004822DE000300620057
:109B0000FE620200000000002004200080630200CA
:109B10000000000000052000FE62020000000000BE
:109B2000F0042000FE62020000000000700520002A
:109B3000FE6202000000000050042000FE620200ED
:109B40000000000020052000FE620200000000006E
:109B500000022000FE62020000000000F00420006D
:109B6000FE6202000000000060042000FE620200AD
:109B70000000000060042000FE62020000000000FF
:109B80001425200060042000806302000000000013
:109B9000F30F200003006200FE62020000000000DC
:109BA0004822DE0003006200FE62020000000000A6
:109BB0002004200080630200000000003004200028
:109BC000FE6202000000000010042000FE6202009D
:109BD00000000000E0042000FE620200000000001F
:109BE00030042000FE62020000000000500420004B
:109BF000FE62020000000000C0042000FE620200BD
:109C00000000000064252000600420008063020042
:109C100000000000F30F200003006200FE6202005B
:109C2000000000004822DE0003006200FE62020025
:109C30000000000080382100308388002230EC00D2
:109C40008E0D04000000000040C7800011002000BD
:109C5000010050004220AE00364E0400000000001B
:109C600075AEA900B41D04000000000040C78000CC
:109C700081002000010050004220AE004E4E040042
:109C8000000000007E2302000000000020002000F1
:109C900010818800B41D0400000000006610E2007E
:109CA0004220AE005E4E04000000000020002000B4
:109CB000108188005E4E0400000000008E0D04003C
:109CC000000000005864020000000000D4112000D1
:109CD000600420008063020000000000F30F2000F9
:109CE00003006200FE620200000000004822DE0065
:109CF00003006200FE620200000000002004200059
:109D0000806302000000000040042000FE620200A8
:109D10000000000000022000FE62020000000000BF
:109D200010042000FE62020000000000000220007B
:109D3000FE6202000000000040052000FE620200FA
:109D40000000000000022000FE620200000000008F
:109D500010042000FE62020000000000000220004B
:109D6000FE6202000000000000022000FE6202000D
:109D70000000000000022000FE620200000000005F
:109D8000D0042000FE62020000000000000220005B
:109D9000FE6202000000000010042000FE620200CB
:109DA0000000000000022000FE620200000000002F
:109DB000E0042000FE62020000000000000220001B
:109DC000FE6202000000000010042000FE6202009B
:109DD0000000000000022000FE62020000000000FF
:109DE00070042000FE62020000000000000220005B
:109DF000FE6202000000000050042000FE6202002B
:109E00000000000000022000FE62020000000000CE
:109E1000D0042000FE6202000000000000022000CA
:109E2000FE6202000000000050042000FE620200FA
:109E30000000000000022000FE620200000000009E
:109E4000E0042000FE62020000000000000220008A
:109E5000FE6202000000000040052000FE620200D9
:109E60000000000054142000600420008063020001
:109E700000000000F30F200003006200FE620200F9
:109E8000000000004822DE0003006200FE620200C3
:109E90000000000020042000806302000000000099
:109EA000D0022000FE62020000000000D00220006C
:109EB000FE62020000000000D0022000FE620200EC
:109EC00000000000D0022000FE620200000000003E
:109ED000D0022000FE62020000000000D00220003C
:109EE000FE62020000000000D0022000FE620200BC
:109EF00000000000D0022000FE620200000000000E
:109F0000D0022000FE62020000000000D00220000B
:109F1000FE62020000000000D0022000FE6202008B
:109F200000000000D0022000FE62020000000000DD
:109F3000D0022000FE62020000000000D0022000DB
:109F4000FE62020000000000D0022000FE6202005B
:109F500000000000D0022000FE62020000000000AD
:109F6000D0022000FE62020000000000D0022000AB
:109F7000FE62020000000000D0022000FE6202002B
:109F800000000000D0022000FE620200000000007D
:109F9000D0022000FE62020000000000D00220007B
:109FA000FE62020000000000D0022000FE620200FB
:109FB00000000000D0022000FE620200000000004D
:109FC000D0022000FE62020000000000D00220004B
:109FD000FE62020000000000D0022000FE620200CB
:109FE00000000000D0022000FE620200000000001D
:109FF000D0022000FE6202000000000004232000C6
:10A00000600420008063020000000000F30F2000C5
:10A0100003006200FE620200000000004822DE0031
:10A0200003006200FE620200000000002004200025
:10A03000806302000000000030042000FE62020085
:10A0400000000000C0042000FE62020000000000CA
:10A0500050042000FE6202000000000010042000F6
:10A06000FE6202000000000020052000FE620200E7
:10A0700000000000342520006004200080630200FE
:10A0800000000000F30F200003006200FE620200E7
:10A09000000000004822DE0003006200FE620200B1
:10A0A0000000000020042000806302000000000087
:10A0B00030052000FE620200000000005004200075
:10A0C000FE62020000000000E0042000FE620200C8
:10A0D0000000000040042000FE62020000000000BA
:10A0E000B4402000600420008063020000000000F3
:10A0F000F30F200003006200FE6202000000000077
:10A100004822DE0003006200FE6202000000000040
:10A1100020042000806302000000000040042000B2
:10A12000FE6202000000000050052000FE620200F6
:10A1300000000000D0042000FE62020000000000C9
:10A1400000052000FE62020000000000844820009C
:10A15000600420008063020000000000F30F200074
:10A1600003006200FE620200000000004822DE00E0
:10A1700003006200FE6202000000000020042000D4
:10A18000806302000000000020042000FE62020044
:10A190000000000010042000FE6202000000000029
:10A1A00030042000FE62020000000000B004200025
:10A1B000FE62020000000000803821003083880029
:10A1C0002230EC008E0D04000000000040C780002B
:10A1D00031002000010050004220AE00FE5004007B
:10A1E000000000007E23020000000000200020008C
:10A1F000108188000C5304000000000040C780005C
:10A2000011002000010050004220AE002251040045
:10A210000000000000002000B09488000000200032
:10A22000C094880080C7800070C7880000002000AC
:10A2300060C7880080382100308388000C530400F8
:10A240000000000040C78000810020000100500095
:10A250004220AE000C520400000000007E230200E9
:10A260000000000050042000C47102000000000043
:10A2700020042000C4710200000000000003200040
:10A28000C47102000000000080032000C4710200BD
:10A2900000000000C0042000C471020000000000A3
:10A2A000F0062000C47102000000000070062000CB
:10A2B000C471020000000000E0032000C47102002D
:10A2C0000000000090948000D0948800A09480004A
:10A2D000E094880000002000909488000000200096
:10A2E000A094880015EEA90015CEA90015AEA8000F
:10A2F000000000000000000000000000000000005E
:10A30000000000000000000000000000156EA90021
:10A31000000000000000000000000000000000003D
:10A32000000000000000000000000000800E20007F
:10A33000E66002000000000000002000E66002006D
:10A340000000000000002000E660020000000000A5
:10A3500000002000E6600200000000000000200075
:10A36000E66002000000000000002000E66002003D
:10A370000000000000002000E66002000000000075
:10A3800000002000E6600200000000003A610200C8
:10A39000000000007E82020000000000100020008B
:10A3A0009232B4000000200094B2B4009094800077
:10A3B000A1948000B2948000C394800000005100FA
:10A3C000818059004200AF00C65104000000000027
:10A3D000D094800090948800E0948000A09488003D
:10A3E00015EEA90015CEA90015AEA90000000000C9
:10A3F000000000000000000000000000000000005D
:10A400000000000000000000803821003083880038
:10A410000C5304000000000040C7800071002000C1
:10A42000010050004220AE00FC5204000000000079
:10A430007E2302000000000050042000C4710200CE
:10A440000000000020042000C47102000000000091
:10A4500000032000C47102000000000080032000FF
:10A46000C47102000000000040042000C47102001A
:10A470000000000050072000C4710200000000002E
:10A48000D0062000C4710200000000000007200078
:10A49000C471020000000000E0032000C47102004B
:10A4A0000000000090948000D0948800A094800068
:10A4B000E0948800000020009094880000002000B4
:10A4C000A094880015EEA90015CEA90015AEA8002D
:10A4D000000000000000000000000000000000007C
:10A4E000000000000000000000000000156EA90040
:10A4F000000000000000000000000000000000005C
:10A50000000000000000000000000000800E20009D
:10A51000E66002000000000000002000E66002008B
:10A520000000000000002000E660020000000000C3
:10A5300000002000E6600200000000000000200093
:10A54000E66002000000000000002000E66002005B
:10A550000000000000002000E66002000000000093
:10A5600000002000E6600200000000003A610200E6
:10A57000000000007E8202000000000010002000A9
:10A580009232B4000000200094B2B4009094800095
:10A59000A1948000F2FF2F00F30020000000510082
:10A5A000818059004200AF00B65204000000000054
:10A5B000D094800090948800E0948000A09488005B
:10A5C00015EEA90015CEA90015AEA90000000000E7
:10A5D000000000000000000000000000000000007B
:10A5E0000000000000000000803821003083880057
:10A5F0000C530400000000006610E2004220AE0090
:10A600000C5304000000000020002000108188008E
:10A610000C530400000000008E0D04000000000038
:10A6200058640200000000008448200060042000FC
:10A630008063020000000000F30F200003006200AE
:10A64000FE620200000000004822DE0003006200FB
:10A65000FE6202000000000020042000806302006F
:10A6600000000000D0042000FE6202000000000094
:10A6700010042000FE620200000000009004200090
:10A68000FE62020000000000E0042000FE62020002
:10A690000000000000022000FE6202000000000036
:10A6A000D0042000FE6202000000000050042000E0
:10A6B000FE62020000000000E0042000FE620200D2
:10A6C0000000000050052000FE62020000000000B3
:10A6D000B0002000108188008E0D040000000000F2
:10A6E00040C7800031002000010050004220AE0031
:10A6F000C8540400000000007E2302000000000097
:10A70000062B210000002000001B780000402600DE
:10A71000001B7800262E210000002000001B78007E
:10A7200000402600001B7800463121000000200078
:10A73000001B780000402600001B780066342100D2
:10A7400000002000001B780000402600001B78005D
:10A750008637210000002000001B78000040260002
:10A76000001B7800A63A210000002000001B7800A2
:10A7700000402600001B7800C63D2100000020009C
:10A78000001B780000402600001B7800E6402100F6
:10A7900000002000001B780000402600001B78000D
:10A7A0000644210000002000001B78000040260025
:10A7B000001B78002647210000002000001B7800C5
:10A7C00000402600001B7800464A210000002000BF
:10A7D000001B780000402600001B7800664D210019
:10A7E00000002000001B780000402600001B7800BD
:10A7F0008650210000002000001B78000040260049
:10A80000001B7800A653210000002000001B7800E8
:10A8100000402600001B7800C656210000002000E2
:10A82000001B780000402600001B7800E65921003C
:10A8300000002000001B780000402600001B78006C
:10A84000065D210000002000001B7800004026006B
:10A85000001B78002660210000002000001B78000B
:10A8600000402600001B7800466321000000200005
:10A87000001B780000402600001B7800666621005F
:10A8800000002000001B780000402600001B78001C
:10A890008669210000002000001B7800004026008F
:10A8A000001B7800A66C210000002000001B78002F
:10A8B00000402600001B7800C66F21000000200029
:10A8C000001B780000402600001B7800E672210083
:10A8D00000002000001B780000402600001B7800CC
:10A8E0000676210000002000001B780000402600B2
:10A8F000001B78002679210000002000001B780052
:10A9000000402600001B7800467C2100000020004B
:10A91000001B780000402600001B7800667F2100A5
:10A9200000002000001B780000402600001B78007B
:10A930008682210000002000001B780000402600D5
:10A94000001B7800A685210000002000001B780075
:10A9500000402600001B7800C6882100000020006F
:10A96000001B780000402600001B7800E68B2100C9
:10A9700000002000001B780000402600001B78002B
:10A980002000200010818800485F040000000000C3
:10A99000030220007E32EC00F093800001022000D0
:10A9A000810050004200AE00E654040000000000A8
:10A9B0008E64020000000000BA6402000000000083
:10A9C0007EB2EF00485F040000000000E62921008D
:10A9D000F0938000210320000100B8000003430031
:10A9E0000694880016407800F10020000100600005
:10A9F00011002000810050004220AE002A550400C2
:10AA000000000000F09380000000E80091838000C7
:10AA1000808050004200AE002A5504000000000073
:10AA20001660A600B2550400000000001650A700F2
:10AA30000E560400000000001640A0001650A600AC
:10AA40001C560400000000001640A1000E56040031
:10AA50000000000006948000810020000683400072
:10AA6000160278000000200000024200600420006E
:10AA70008063020000000000F30F2000030062006A
:10AA8000FE620200000000004822DE0003006200B7
:10AA9000FE6202000000000020042000806302002B
:10AAA00000000000AC82020000000000069480005C
:10AAB0001660A70086550400000000000002200078
:10AAC000FE6202000000000000022000FE620200A0
:10AAD0000000000000022000FE62020000000000F2
:10AAE00000022000FE6202000000000000022000C0
:10AAF000FE6202000000000000022000FE62020070
:10AB000000000000AE55040000000000C00320005B
:10AB1000FE6202000000000040042000FE6202000D
:10AB20000000000050042000FE620200000000004F
:10AB300060042000FE62020000000000E00320002C
:10AB4000FE6202000000000000022000FE6202001F
:10AB500000000000AE550400000000000E56040086
:10AB600000000000008480007E12E3004220AF005D
:10AB70000210A80006948000810020000683400097
:10AB8000160278000000200000024200600420004D
:10AB90008063020000000000F30F20000300620049
:10ABA000FE620200000000004822DE000300620096
:10ABB000FE6202000000000020042000806302000A
:10ABC00000000000AC82020000000000C003200072
:10ABD000FE6202000000000030042000FE6202005D
:10ABE00000000000F0042000FE62020000000000EF
:10ABF000D0042000FE62020000000000E0032000FC
:10AC0000FE6202000000000000022000FE6202005E
:10AC1000000000000E560400000000008301E9005F
:10AC20000300E0004220AE00CA540400000000000F
:10AC3000485F0400000000000210AF00C25704008B
:10AC400000000000008480007E12E3004220AE007D
:10AC5000445C040000000000009480001084880020
:10AC60000694800081022000068340003640780070
:10AC7000F10F2000010060000250AE009056040069
:10AC800000000000418480004084880001005000E2
:10AC9000F10F2000010060000000E0004220AF0042
:10ACA0009256040000000000808188003230EF00DE
:10ACB0003430EF00E0808000B08188003830EF0051
:10ACC0003A30EF000E730200000000008081800027
:10ACD00091818000E2838000F383800002004000C5
:10ACE00083804800F29F2C00A3B923000202500089
:10ACF000838258004200AE00845604000000000029
:10AD00000200780083007800E0838800F1838800E7
:10AD1000B27C020000000000925604000000000017
:10AD2000408488000250A80070A72200808188001B
:10AD3000300120009081880000002000A081880060
:10AD4000E0808000B08188003830EF003A30EF00BA
:10AD50000E730200000000000694800051022000E3
:10AD60000683400036407800F10F200001006000AB
:10AD7000B6407800C808DD0002F02F008280600035
:10AD800001007000B081880036407800F10F20008B
:10AD900001006000C08188000694800051022000FC
:10ADA0000683400036407800F10F2000010060006B
:10ADB000B6407800C808DD0002F02F0082806000F5
:10ADC00081007000B0818000810050004220AE0000
:10ADD000AC5604000000000036417800F10F20005E
:10ADE00001016100C1818000010151004220AE00DB
:10ADF000AC560400000000003A30EF00F2FF2F00D4
:10AE00000201500032002000028158004200AE00D2
:10AE10001457040000000000F0FF2F00B0818800EC
:10AE2000F0FF2F00C081880078730200000000004E
:10AE300080818000D0838800069480004102200039
:10AE400006834000364078000030A7007A30EF00DB
:10AE5000E444200060042000806302000000000041
:10AE6000F30F200003006200FE62020000000000F9
:10AE70004822DE0003006200FE62020000000000C3
:10AE80002004200080630200000000003005200044
:10AE9000FE6202000000000000072000FE620200C7
:10AEA0000000000050062000FE62020000000000CA
:10AEB00050062000FE620200000000004006200054
:10AEC000FE62020000000000A0032000FE620200FB
:10AED0000000000000022000FE62020000000000EE
:10AEE000D083800080818800B66B020000000000E3
:10AEF000908280000103200001004000FE620200F9
:10AF000000000000A082800001032000010040003A
:10AF1000FE62020000000000E0022000FE6202006B
:10AF200000000000B082800001032000010040000A
:10AF3000FE62020000000000C082800001032000C9
:10AF400001004000FE62020000000000B006200088
:10AF5000FE62020000000000D0062000FE62020037
:10AF600000000000F0022000FE620200000000006D
:10AF700080062000FE620200000000004E5804001F
:10AF8000000000007A30EF00008480007E12E300B1
:10AF90004220AF000210A900E44420006004200019
:10AFA0008063020000000000F30F20000300620035
:10AFB000FE620200000000004822DE000300620082
:10AFC000FE620200000000002004200080630200F6
:10AFD0000000000030052000FE62020000000000BA
:10AFE00000072000FE620200000000005006200062
:10AFF000FE6202000000000050062000FE62020017
:10B000000000000040062000FE6202000000000078
:10B01000A0032000FE6202000000000000022000E9
:10B02000FE62020000000000C0032000FE62020079
:10B030000000000030042000FE620200000000005A
:10B04000F0042000FE62020000000000D004200096
:10B05000FE62020000000000E0032000FE62020029
:10B060000000000000022000FE620200000000005C
:10B0700000022000FE62020000000000000220002A
:10B08000FE6202000000000000022000FE620200DA
:10B09000000000004E58040000000000E083800023
:10B0A000F1838000F29F2C00A3B92300020250001C
:10B0B000838258004200AE00645804000000000083
:10B0C00002007800830078008081880091818800E8
:10B0D000D46A020000000000F43F20006004200059
:10B0E0008063020000000000F30F200003006200F4
:10B0F000FE620200000000004822DE000300620041
:10B10000FE620200000000002004200080630200B4
:10B110000000000040052000FE6202000000000068
:10B1200020072000FE6202000000000090062000C0
:10B13000FE6202000000000000072000FE62020024
:10B1400000000000A0032000FE62020000000000DA
:10B1500000022000FE620200000000005082800019
:10B160000103200001004000FE6202000000000018
:10B17000608280000103200001004000FE620200A6
:10B1800000000000708280000103200001004000E8
:10B19000FE62020000000000E0022000FE620200E9
:10B1A00000000000808280000103200001004000B8
:10B1B000FE62020000000000908280000103200077
:10B1C00001004000FE62020000000000A08280003A
:10B1D0000103200001004000FE62020000000000A8
:10B1E000B0062000FE62020000000000D006200031
:10B1F000FE62020000000000803821007A10E200A8
:10B200004220AF0050C7880080162000808188004F
:10B21000000020009081880000002000A0818800AC
:10B2200000818000B081880000002000C08188007B
:10B2300000002000D08188000E7302000000000092
:10B24000F0808000B081880000002000C08188006C
:10B2500000002000D08188000E7302000000000072
:10B260008081800010828800908180002082880088
:10B27000A08180003082880000A62E008081880096
:10B28000000020009081880000002000A08188003C
:10B29000D0838000B081880000002000C081880039
:10B2A000D08188000E7302000000000080818000C1
:10B2B000E081880090818000F0818800A08180007A
:10B2C0000082880060838000B08188000000200038
:10B2D000C0818800D08188000E7302000000000049
:10B2E00010828000B081880020828000C0818800A8
:10B2F00020828000C0818800787302000000000076
:10B3000080818000408388000694800081002000B6
:10B3100006834000040020006004200080630200D7
:10B3200000000000F30F200003006200FE62020034
:10B33000000000004822DE0003006200FE620200FE
:10B3400000000000200420008063020000000000D4
:10B3500000022000FE620200000000000002200047
:10B36000FE6202000000000000022000FE620200F7
:10B370000000000000022000FE6202000000000049
:10B3800000022000FE620200000000000002200017
:10B39000FE6202000000000000022000FE620200C7
:10B3A0000000000000022000FE6202000000000019
:10B3B00000022000FE6202000000000060838000A6
:10B3C00080818800B66B020000000000908280003F
:10B3D0000103200001004000FE62020000000000A6
:10B3E000A08280000103200001004000FE620200F4
:10B3F00000000000B0828000010320000100400036
:10B40000FE62020000000000C082800001032000F4
:10B4100001004000FE62020000000000D0828000B7
:10B420000103200001004000FE6202000000000055
:10B43000B0062000FE62020000000000700620003E
:10B44000FE62020000000000F0022000FE62020026
:10B450000000000080062000FE62020000000000E4
:10B4600000022000FE620200000000000002200036
:10B47000FE6202000000000000022000FE620200E6
:10B480000000000000022000FE6202000000000038
:10B490000694800021012000068340003640780099
:10B4A000F20F20000200600096407800C808DD001E
:10B4B00002F02F008280600001007000808188000F
:10B4C000B66B0200000000009082800001032000A3
:10B4D00001004000FE62020000000000A082800027
:10B4E0000103200001004000FE6202000000000095
:10B4F000B08280000103200001004000FE620200D3
:10B5000000000000C0828000010320000100400014
:10B51000FE62020000000000D082800001032000D3
:10B5200001004000FE62020000000000D006200082
:10B53000FE62020000000000C0062000FE62020061
:10B5400000000000F0022000FE6202000000000087
:10B55000D0062000FE620200000000000002200071
:10B56000FE6202000000000000022000FE620200F5
:10B5700000000000A0032000FE62020000000000A6
:10B5800040052000FE6202000000000010062000BE
:10B59000FE6202000000000020072000FE620200A0
:10B5A0000000000070062000FE62020000000000A3
:10B5B00050062000FE62020000000000400720004C
:10B5C000FE6202000000000006948000810020005E
:10B5D00006834000043720006004200080630200DE
:10B5E00000000000F30F200003006200FE62020072
:10B5F000000000004822DE0003006200FE6202003C
:10B600000000000020042000806302000000000011
:10B6100040052000FE62020000000000100620002D
:10B62000FE6202000000000020072000FE6202000F
:10B630000000000070062000FE6202000000000012
:10B6400050062000FE6202000000000040072000BB
:10B65000FE62020000000000A0032000FE62020063
:10B660000000000000022000FE6202000000000056
:10B6700000022000FE6202000000000060838000E3
:10B6800080818800B66B020000000000908280007C
:10B690000103200001004000FE62020000000000E3
:10B6A000A08280000103200001004000FE62020031
:10B6B00000000000B0828000010320000100400073
:10B6C000FE62020000000000C08280000103200032
:10B6D00001004000FE62020000000000D0828000F5
:10B6E0000103200001004000FE6202000000000093
:10B6F000B0062000FE62020000000000700620007C
:10B70000FE62020000000000F0022000FE62020063
:10B710000000000080062000FE6202000000000021
:10B7200000022000FE620200000000000002200073
:10B73000FE6202000000000000022000FE62020023
:10B740000000000000022000FE6202000000000075
:10B7500006948000210120000683400036407800D6
:10B76000F20F20000200600096407800C808DD005B
:10B7700002F02F008280600001007000808188004C
:10B78000B66B0200000000009082800001032000E0
:10B7900001004000FE62020000000000A082800064
:10B7A0000103200001004000FE62020000000000D2
:10B7B000B08280000103200001004000FE62020010
:10B7C00000000000C0828000010320000100400052
:10B7D000FE62020000000000D08280000103200011
:10B7E00001004000FE62020000000000D0062000C0
:10B7F000FE62020000000000C0062000FE6202009F
:10B8000000000000F0022000FE62020000000000C4
:10B81000D0062000FE6202000000000000022000AE
:10B82000FE6202000000000000022000FE62020032
:10B8300000000000A0032000FE62020000000000E3
:10B8400040052000FE6202000000000010062000FB
:10B85000FE6202000000000020072000FE620200DD
:10B860000000000070062000FE62020000000000E0
:10B8700050062000FE620200000000004007200089
:10B88000FE62020000000000D08380000694800069
:10B8900041012000068340000000E000110020006C
:10B8A0004220AF0001002000014B78000694800088
:10B8B000200120000003430040838000F10F20009E
:10B8C00001006000005B7800408380004800DE00DB
:10B8D00001006000005B78000694800020022000D8
:10B8E0000003430016007800F1FF2F008100600084
:10B8F0004220AF00B05C04000000000000F0A70090
:10B90000B05C04000000000080818800000020007E
:10B9100090818800A081880010828000B08188001A
:10B9200020828000C081880030828000D081880021
:10B930000E73020000000000E0818000B0818800EA
:10B94000F0818000C081880000828000D081880062
:10B950007873020000000000B85C040000000000E2
:10B960000000200080818800B85C04000000000016
:10B970000694800060002000000343008081800066
:10B98000000B780006948000808180006183800035
:10B99000010150004200AF00D25C04000000000032
:10B9A0000201EA0032848800608380008081880080
:10B9B0000000200090818800A0818800A000200065
:10B9C000B081880000002000C0818800D0818800FC
:10B9D0000E7302000000000040062000B0818800C5
:10B9E00000002000C0818800D081880078730200A8
:10B9F000000000008081800031848000010150003F
:10BA00001670A1004200AE001670A00006948000DF
:10BA1000810020000683400016027800000020000C
:10BA20000002420060042000806302000000000069
:10BA3000F30F200003006200FE620200000000001D
:10BA40004822DE0003006200FE62020000000000E7
:10BA5000200420008063020000000000AC8202008D
:10BA600000000000069480001670A6006E5D0400C1
:10BA70000000000006948000410120000683400081
:10BA80001600A6006E5D0400000000006B30AE00E2
:10BA90006E5D04000000000000022000FE62020053
:10BAA0000000000000022000FE6202000000000012
:10BAB00000022000FE6202000000000000022000E0
:10BAC000FE6202000000000000022000FE62020090
:10BAD00000000000C05D040000000000069480002B
:10BAE0006000200000034300160078008081880079
:10BAF0000594800000032000008042001000A70091
:10BB00001C74020000000000B66B02000000000080
:10BB1000908280000103200001004000FE620200CC
:10BB200000000000A082800001032000010040000E
:10BB3000FE62020000000000B082800001032000CD
:10BB400001004000FE62020000000000C082800090
:10BB50000103200001004000FE620200000000001E
:10BB6000D08280000103200001004000FE6202003C
:10BB70000000000000022000FE6202000000000041
:10BB8000069480001640A100C43E200060042000FE
:10BB90008063020000000000F30F20000300620039
:10BBA000FE620200000000004822DE000300620086
:10BBB000FE620200000000002004200080630200FA
:10BBC0000000000040052000FE62020000000000AE
:10BBD00090062000FE62020000000000D006200057
:10BBE000FE6202000000000050062000FE6202001B
:10BBF00000000000A0032000FE6202000000000020
:10BC000000022000FE62020000000000218080008F
:10BC10004808DE00FE620200000000002080800074
:10BC2000FE62020000000000A0032000FE6202008D
:10BC300000000000318080004808DE00FE62020043
:10BC40000000000030808000FE6202000000000062
:10BC5000A0032000FE62020000000000418080007E
:10BC60004808DE00FE620200000000004080800004
:10BC7000FE62020000000000444120006004200039
:10BC80008063020000000000F30F20000300620048
:10BC9000FE620200000000004822DE000300620095
:10BCA000FE62020000000000200420008063020009
:10BCB00000000000C0042000FE620200000000003E
:10BCC00010062000FE620200000000004007200075
:10BCD000FE62020000000000E0022000FE6202009E
:10BCE00000000000A0032000FE620200000000002F
:10BCF00000022000FE62020000000000518080006F
:10BD00004808DE00FE620200000000005080800053
:10BD1000FE62020000000000F00D2000FE62020042
:10BD200000000000618080004808DE00FE62020022
:10BD30000000000060808000FE6202000000000041
:10BD400020022000FE6202000000000071808000DE
:10BD50004808DE00FE6202000000000070808000E3
:10BD6000FE6202000000000070022000FE6202007D
:10BD700000000000818080004808DE00FE620200B2
:10BD800000000000C4432000600420008063020023
:10BD900000000000F30F200003006200FE620200BA
:10BDA000000000004822DE0003006200FE62020084
:10BDB000000000002004200080630200000000005A
:10BDC000C0042000FE62020000000000F006200017
:10BDD000FE62020000000000E0062000FE62020099
:10BDE0000000000070062000FE620200000000005B
:10BDF000A0032000FE62020000000000908080008E
:10BE0000FE62020000000000A18080004808DE0001
:10BE1000FE62020000000000A0808000FE620200BE
:10BE200000000000F00D2000FE6202000000000093
:10BE3000B18080004808DE00FE62020000000000C1
:10BE4000B0808000FE62020000000000200220009E
:10BE5000FE62020000000000C18080004808DE0091
:10BE6000FE62020000000000C0808000FE6202004E
:10BE70000000000070022000FE62020000000000CE
:10BE8000D18080004808DE00FE6202000000000051
:10BE90008E0D040000000000154EA800152EA8000D
:10BEA00015AEA80015CEA90015EEA80000000000F0
:10BEB0000000000000000000C4610200000000005B
:10BEC000000000000000000000000000156EA90046
:10BED0000000000000000000000000000000000062
:10BEE000000000000000000000000000800E2000A4
:10BEF000E66002000000000000002000E660020092
:10BF00000000000000002000E660020000000000C9
:10BF100000002000E6600200000000000000200099
:10BF2000E66002000000000000002000E660020061
:10BF30000000000000002000E66002000000000099
:10BF400000002000E6600200000000000810200051
:10BF500009002D003A61020000000000800C78000A
:10BF60008984E8000804E9000800E0004220AE00EF
:10BF7000AA5F0400000000000000000000000000B4
:10BF800000000000156EA800000000000000000086
:10BF900000000000000000000000000000000000A1
:10BFA000000000008662020000000000156EA9007B
:10BFB0000000000000000000000000000000000081
:10BFC0000000000000000000000000001008200039
:10BFD000E66002000000000000002000E6600200B1
:10BFE0000000000000002000E660020000000000E9
:10BFF00000002000E660020000000000156EA800AE
:10C000000000000000000000000000000000000030
:10C010000000000000000000000000008662020036
:10C02000000000008662020000000000866202003C
:10C03000000000008662020000000000156EA900EA
:10C0400000000000000000000000000000000000F0
:10C050000000000000000000000000004008200078
:10C06000E66002000000000000002000E660020020
:10C070000000000000002000E66002000000000058
:10C0800000002000E6600200000000000810200010
:10C090007000200008004000E66002000000000080
:10C0A0000804E9000800E0004220AE0048600400F7
:10C0B00000000000156EA800000000000000000055
:10C0C0000000000000000000000000000000000070
:10C0D000000000008662020000000000156EA9004A
:10C0E0000000000000000000000000000000000050
:10C0F0000000000000000000000000008008200098
:10C10000E66002000000000000002000E66002007F
:10C110000000000000002000E660020000000000B7
:10C1200000002000E660020000000000F0808000B7
:10C13000E66002000000000000818000E66002006E
:10C140000000000060838000E66002000000000044
:10C1500070838000E66002000000000080838000A1
:10C16000E66002000000000090838000E6600200AC
:10C1700000000000A0838000E660020000000000D4
:10C18000B0838000E660020000000000C0838000F1
:10C19000E660020000000000156EA800000000002C
:10C1A000000000000000000000000000000000008F
:10C1B000000000000000000000000000000000007F
:10C1C000000000008E0D040000000000810020002F
:10C1D000000000000000000000000000000000005F
:10C1E000000000000000000000000000548EA900C4
:10C1F000000000000000000000000000000000003F
:10C200000000000000000000000000000000D0005E
:10C210000080A60035EEA9000080A70035EEA8003A
:10C22000000000000000000000000000000000000E
:10C23000000000000000000000000000548EA80074
:10C2400000000000000000000000000000000000EE
:10C250000000000000000000000000008100E90074
:10C260000100E0004220AE00E86004000000000091
:10C2700000000600000020008100200000000000F7
:10C2800000000000000000000000000000000000AE
:10C290000000000000000000548EA9000000000013
:10C2A000000000000000000000000000000000008E
:10C2B000000000000000000000000000000000007E
:10C2C00000000000000000000000D00033CEAF00EE
:10C2D0000000A00033CEAE000000A100000000006E
:10C2E000000000000000000000000000000000004E
:10C2F0000000000000000000548EA80000000000B4
:10C30000000000000000000000000000000000002D
:10C3100000000000000000008100E9000100E000D2
:10C320004220AE003E610400000000000000060054
:10C33000156EA900000000000000000000000000D1
:10C3400000000000000000000000000000000000ED
:10C35000700D2000E6600200000000003A6102005B
:10C3600000000000156EA8000000000000000000A2
:10C3700000000000000000000000000000000000BD
:10C3800000000000000006009861020000000000AC
:10C390000070A600C4610400000000000000A700B7
:10C3A0001A62040000000000156EA90000000000E1
:10C3B000000000000000000000000000000000007D
:10C3C0000000000000000000D0032000E660020032
:10C3D00000000000A0022000E66002000000000053
:10C3E00000082000E660020000000000600A200053
:10C3F000E660020000000000156EA80000000000CA
:10C40000000000000000000000000000000000002C
:10C410000000000000000000986102000000000021
:10C420000070A6000C620400000000000C62040012
:10C430000000000000000600FFFF37005C62020001
:10C4400000000000942EAA005C62020000000000C0
:10C45000942EAA005C62020000000000942EAA0044
:10C460005C62020000000000942EAA005C620200E0
:10C4700000000000942EAA005C6202000000000090
:10C48000942EAA005C62020000000000942EAA0014
:10C490005C62020000000000942EAA005C620200B0
:10C4A00000000000942EAA005C6202000000000060
:10C4B000942EAA0000000600866202000000000020
:10C4C0008662020000000000866202000000000098
:10C4D0008662020000000000866202000000000088
:10C4E0008662020000000000866202000000000078
:10C4F0008662020000000000866202000000000068
:10C50000866202000000000000000600B062020027
:10C5100000000000B062020000000000B0620200F3
:10C5200000000000B062020000000000B0620200E3
:10C5300000000000B062020000000000B0620200D3
:10C5400000000000B062020000000000B0620200C3
:10C5500000000000B06202000000000000000600C1
:10C5600002022000220888000021EF00524420002F
:10C57000120888000068A90002022800220888002A
:10C580000068AE00C0620400000000000000060069
:10C59000D862020000000000C10220008100680093
:10C5A0004220AE00C8620400000000000000060047
:10C5B0002202AE00D8620400000000002682BF0004
:10C5C000F10F20000100600034A2B7002222AE006B
:10C5D000EE620400000000002222A9000000060014
:10C5E000004006000000EB00000778000C00090086
:10C5F000002F78000007EB0000000600F10F20007C
:10C60000810060000500FC0000F02F00842EB600C1
:10C6100001007800842EB700000000000000000038
:10C62000000000000000000000000000000000000A
:10C63000000000000000000000000000348EA9008F
:10C6400000000000000000000000000000000000EA
:10C6500000000000000000000000000000000000DA
:10C660000000000034AEA90000000000000000003F
:10C6700000000000000000000000000000000000BA
:10C6800000000000000000000000000035AEA9001E
:10C69000000000000000000000000000000000009A
:10C6A000000000000000000000000000000000008A
:10C6B000000000000000000000000000000000007A
:10C6C000000000000000000035AEA80000000000DF
:10C6D000000000000000000000000000000000005A
:10C6E000000000000000000000000000000000004A
:10C6F00034AEA8000E640200000000000000060036
:10C70000F10F2000810060000500FC0000F02F0008
:10C71000842EB60001007800842EB70000000000CF
:10C720000000000000000000000000000000000009
:10C7300000000000000000000000000000000000F9
:10C74000348EA8000000000000000000000000007F
:10C7500000000000000000000000000000000000D9
:10C76000000000000000000034AEA900000000003E
:10C7700000000000000000000000000000000000B9
:10C7800000000000000000000000000000000000A9
:10C790000000000000000000000000000000000099
:10C7A000000000000000000035AEA90000000000FD
:10C7B0000000000000000000000000000000000079
:10C7C0000000000000000000000000000000000069
:10C7D0000000000000000000000000000000000059
:10C7E0000000000035AEA8000000000000000000BE
:10C7F0000000000000000000000000000000000039
:10C8000000000000000000000000000034AEA8009E
:10C810000E6402000000000000000600000000009E
:10C820000000000000000000000000000000000008
:10C8300000000000000000000000000000000000F8
:10C8400000000000000000000000000000000000E8
:10C8500000000000000000000000000000000000D8
:10C8600000000000000000000000000000000000C8
:10C8700000000000000000000000000000000000B8
:10C8800000000000000000000000000000000000A8
:10C890000000000000000000000000000000000098
:10C8A000000000000000000000000600000006007C
:10C8B00062640200000000008E64020000000000BC
:10C8C00000000600600420008063020000000000F9
:10C8D00000002000FE6202000000000000002000B6
:10C8E000FE620200000000002004200080630200BD
:10C8F00000000000084B200000022000FE62020041
:10C90000000000000804E9000800E0004220AE003A
:10C910007C640400000000000000060060042000A9
:10C92000806302000000000000082000FE62020098
:10C930000000000050022000FE6202000000000023
:10C94000200420008063020000000000085822003C
:10C9500000002000FE620200000000000804E90060
:10C960000800E0004220AE00A864040000000000BF
:10C9700000000600040020007269020000000000B0
:10C98000E40020008063020000000000B0062000E8
:10C99000FE6202000000000070062000FE6202003D
:10C9A00000000000F0022000FE6202000000000013
:10C9B00080062000FE62020000000000240120002A
:10C9C0000069020000000000A40120008063020052
:10C9D00000000000D0062000FE62020000000000FF
:10C9E000C0062000FE62020000000000F0022000ED
:10C9F000FE62020000000000D0062000FE6202007D
:10CA00000000000000022000FE62020000000000A2
:10CA100000022000FE62020000000000A0032000CF
:10CA2000FE6202000000000040052000FE620200DD
:10CA30000000000010062000FE620200000000005E
:10CA400020072000FE6202000000000070062000A7
:10CA5000FE6202000000000050062000FE6202009C
:10CA60000000000040072000FE62020000000000FD
:10CA700084022000C6690200000000008407200034
:10CA8000C669020000000000840C2000C669020094
:10CA90000000000084112000C669020000000000B0
:10CAA00084162000C669020000000000841B2000DC
:10CAB000C66902000000000084202000C669020050
:10CAC0000000000084252000C6690200000000006C
:10CAD000842A2000C669020000000000842F200084
:10CAE000C66902000000000084342000C66902000C
:10CAF0000000000084392000C66902000000000028
:10CB0000043C2000C669020000000000044620002A
:10CB1000C669020000000000040520006004200037
:10CB20008063020000000000F30F20000300620099
:10CB3000FE620200000000004822DE0003006200E6
:10CB4000FE6202000000000020042000806302005A
:10CB50000000000020052000FE620200000000002E
:10CB6000F0062000FE6202000000000070072000B6
:10CB7000FE6202000000000000022000FE620200CF
:10CB80000000000000022000FE6202000000000021
:10CB9000B0062000FE6202000000000070062000C7
:10CBA000FE62020000000000F0022000FE620200AF
:10CBB0000000000080062000FE620200000000006D
:10CBC00000022000FE62020000000000200520009C
:10CBD000FE62020000000000F0062000FE6202007B
:10CBE0000000000070072000FE620200000000004C
:10CBF00000022000FE62020000000000000220008F
:10CC0000FE62020000000000B0062000FE6202008A
:10CC10000000000070062000FE620200000000001C
:10CC2000F0022000FE6202000000000080062000EA
:10CC3000FE6202000000000000022000FE6202000E
:10CC40000000000020052000FE620200000000003D
:10CC5000F0062000FE6202000000000070072000C5
:10CC6000FE6202000000000000022000FE620200DE
:10CC70000000000000022000FE6202000000000030
:10CC8000B0062000FE6202000000000070062000D6
:10CC9000FE62020000000000F0022000FE620200BE
:10CCA0000000000080062000FE620200000000007C
:10CCB00000022000FE6202000000000020052000AB
:10CCC000FE62020000000000F0062000FE6202008A
:10CCD0000000000070072000FE620200000000005B
:10CCE00000022000FE62020000000000000220009E
:10CCF000FE62020000000000B0062000FE6202009A
:10CD00000000000070062000FE620200000000002B
:10CD1000F0022000FE6202000000000080062000F9
:10CD2000FE6202000000000000022000FE6202001D
:10CD30000000000004322000600420008063020034
:10CD400000000000F30F200003006200FE620200FA
:10CD5000000000004822DE0003006200FE620200C4
:10CD6000000000002004200080630200000000009A
:10CD700020052000FE62020000000000F0062000F6
:10CD8000FE6202000000000070072000FE62020048
:10CD90000000000000022000FE620200000000000F
:10CDA00000022000FE62020000000000B006200029
:10CDB000FE6202000000000070062000FE62020019
:10CDC00000000000F0022000FE62020000000000EF
:10CDD00080062000FE620200000000000002200029
:10CDE000FE6202000000000020052000FE6202003A
:10CDF00000000000F0062000FE62020000000000BB
:10CE000070072000FE620200000000000002200007
:10CE1000FE6202000000000000022000FE6202002C
:10CE200000000000B0062000FE62020000000000CA
:10CE300070062000FE62020000000000F0022000E8
:10CE4000FE6202000000000080062000FE62020078
:10CE50000000000000022000FE620200000000004E
:10CE600020052000FE62020000000000F006200005
:10CE7000FE6202000000000070072000FE62020057
:10CE80000000000000022000FE620200000000001E
:10CE900000022000FE62020000000000B006200038
:10CEA000FE6202000000000070062000FE62020028
:10CEB00000000000F0022000FE62020000000000FE
:10CEC00080062000FE620200000000000002200038
:10CED000FE6202000000000020052000FE62020049
:10CEE00000000000F0062000FE62020000000000CA
:10CEF00070072000FE620200000000000002200017
:10CF0000FE6202000000000000022000FE6202003B
:10CF100000000000B0062000FE62020000000000D9
:10CF200070062000FE62020000000000F0022000F7
:10CF3000FE6202000000000080062000FE62020087
:10CF40000000000000022000FE620200000000005D
:10CF50000432200080630200000000004005200031
:10CF6000FE6202000000000010062000FE620200C7
:10CF70000000000020072000FE6202000000000008
:10CF800070062000FE620200000000005006200033
:10CF9000FE6202000000000040072000FE62020066
:10CFA00000000000A0032000FE620200000000005C
:10CFB00000022000FE6202000000000000022000CB
:10CFC000FE62020000000000E432200080630200E4
:10CFD00000000000B0062000FE6202000000000019
:10CFE00070062000FE62020000000000F002200037
:10CFF000FE6202000000000080062000FE620200C7
:10D00000000000002433200000690200000000003E
:10D01000A43320008063020000000000D00620003E
:10D02000FE62020000000000C0062000FE62020056
:10D0300000000000F0022000FE620200000000007C
:10D04000D0062000FE620200000000000002200066
:10D05000FE6202000000000000022000FE620200EA
:10D0600000000000A0032000FE620200000000009B
:10D0700040052000FE6202000000000010062000B3
:10D08000FE6202000000000020072000FE62020095
:10D090000000000070062000FE6202000000000098
:10D0A00050062000FE620200000000004007200041
:10D0B000FE62020000000000B43F2000A6680200EB
:10D0C0000000000054422000D06802000000000070
:10D0D000366902000000000036690200000000000E
:10D0E0003669020000000000D4442000826802007B
:10D0F00000000000E44520008268020000000000FB
:10D1000000000600600420008063020000000000B0
:10D11000F30F200003006200FE6202000000000026
:10D120004822DE0003006200FE62020000000000F0
:10D1300020042000806302000000000000022000A4
:10D14000FE620200000000000000060060042000F3
:10D150008063020000000000F30F20000300620063
:10D16000FE620200000000004822DE0003006200B0
:10D17000FE62020000000000200420008063020024
:10D180000000000000022000FE620200000000001B
:10D1900000022000FE620200000000000000060005
:10D1A000600420008063020000000000F30F2000F4
:10D1B00003006200FE620200000000004822DE0060
:10D1C00003006200FE620200000000002004200054
:10D1D000806302000000000000022000FE620200E6
:10D1E0000000000000022000FE62020000000000BB
:10D1F00000022000FE6202000000000000000600A5
:10D20000600420008063020000000000F30F200093
:10D2100003006200FE620200000000004822DE00FF
:10D2200003006200FE6202000000000020042000F3
:10D23000806302000000000000022000FE62020085
:10D240000000000000022000FE620200000000005A
:10D2500000022000FE620200000000000002200028
:10D26000FE620200000000000000060060042000D2
:10D270008063020000000000F30F20000300620042
:10D28000FE620200000000004822DE00030062008F
:10D29000FE62020000000000200420008063020003
:10D2A0000000000000022000FE62020000000000FA
:10D2B00000022000FE6202000000000000022000C8
:10D2C000FE6202000000000000022000FE62020078
:10D2D0000000000000022000FE62020000000000CA
:10D2E00000000600600420008063020000000000CF
:10D2F000F30F200003006200FE6202000000000045
:10D300004822DE0003006200FE620200000000000E
:10D3100020042000806302000000000000022000C2
:10D32000FE6202000000000000022000FE62020017
:10D330000000000000022000FE6202000000000069
:10D3400000022000FE620200000000000002200037
:10D35000FE6202000000000000022000FE620200E7
:10D360000000000000022000FE6202000000000039
:10D3700000022000FE620200000000000002200007
:10D38000FE620200000000000000060060042000B1
:10D390008063020000000000F30F20000300620021
:10D3A000FE620200000000004822DE00030062006E
:10D3B000FE620200000000002004200080630200E2
:10D3C0000000000000022000FE62020000000000D9
:10D3D00000022000FE6202000000000000022000A7
:10D3E000FE6202000000000000022000FE62020057
:10D3F0000000000000022000FE62020000000000A9
:10D4000000022000FE620200000000000002200076
:10D41000FE6202000000000000022000FE62020026
:10D420000000000000022000FE6202000000000078
:10D4300000022000FE620200000000000002200046
:10D44000FE6202000000000000022000FE620200F6
:10D450000000000000022000FE6202000000000048
:10D4600000022000FE620200000000000002200016
:10D47000FE6202000000000000022000FE620200C6
:10D480000000000000022000FE6202000000000018
:10D4900000022000FE6202000000000000022000E6
:10D4A000FE6202000000000000022000FE62020096
:10D4B0000000000000022000FE62020000000000E8
:10D4C00000022000FE6202000000000000022000B6
:10D4D000FE6202000000000000022000FE62020066
:10D4E0000000000000022000FE62020000000000B8
:10D4F00000022000FE620200000000000002200086
:10D50000FE6202000000000000022000FE62020035
:10D510000000000000022000FE6202000000000087
:10D5200000022000FE620200000000000002200055
:10D53000FE6202000000000000022000FE62020005
:10D540000000000000022000FE6202000000000057
:10D5500000022000FE620200000000000002200025
:10D56000FE6202000000000000022000FE620200D5
:10D570000000000000022000FE6202000000000027
:10D5800000022000FE6202000000000000022000F5
:10D59000FE6202000000000000022000FE620200A5
:10D5A00000000000000006004830EF004A30EF00A5
:10D5B0004C30EF004E30EF005030EF005230EF00B3
:10D5C0005430EF005630EF005830EF005A30EF0083
:10D5D000808180009181800002A02C00A3B92300EB
:10D5E00002025000838258004200AE00046B040027
:10D5F0000000000004007800850078004830EC004E
:10D60000F06A04000000000002102E00535F2000AA
:10D6100002025000838258004200AE001C6B0400DE
:10D620000000000004007800850078004A30EC001B
:10D63000086B040000000000026829008309200034
:10D6400002025000838258004200AE00346B040096
:10D650000000000004007800850078004C30EC00E9
:10D66000206B04000000000002242400F3002000CE
:10D6700002025000838258004200AE004C6B04004E
:10D680000000000004007800850078004E30EC00B7
:10D69000386B040000000000026A2800130020001C
:10D6A00002025000838258004200AE00646B040006
:10D6B0000000000004007800850078005030EC0085
:10D6C000506B0400000000000271220003002000E3
:10D6D00002025000838258004200AE007C6B0400BE
:10D6E0000000000004007800850078005230EC0053
:10D6F000686B040000000000823E2000020250001F
:10D700004200AE008E6B04000000000004007800B0
:10D710005430EC007E6B0400000000004206200044
:10D72000020250004200AE00A06B040000000000A6
:10D73000040078005630EC00906B040000000000FC
:10D74000A2002000020250004200AE00B26B0400B2
:10D7500000000000040078005830EC00A26B0400C8
:10D7600000000000D0828800000006005230EF0068
:10D770005430EF005630EF005830EF005A30EF00D1
:10D780008081800001712200010150004200AE0042
:10D79000D46B040000000000020078005230EC005E
:10D7A000C46B040000000000813E20000101500015
:10D7B0004200AE00E66B04000000000002007800AA
:10D7C0005430EC00D66B040000000000410620003D
:10D7D000010150004200AE00F86B040000000000A0
:10D7E000020078005630EC00E86B040000000000F6
:10D7F000A1002000010150004200AE000A6C0400AC
:10D8000000000000020078005830EC00FA6B0400C1
:10D8100000000000D082880000000600168480000E
:10D820002100200006834000F20F2000020160006A
:10D83000025B7800C800DE00F20F20000281600069
:10D84000025B7800062D21002100200006834000A5
:10D85000F20F200002016000025B7800C800DE00C9
:10D86000F20F200002816000025B78002630210068
:10D870002100200006834000F20F2000020160001A
:10D88000025B7800C800DE00F20F20000281600019
:10D89000025B78004633210021002000068340000F
:10D8A000F20F200002016000025B7800C800DE0079
:10D8B000F20F200002816000025B780066362100D2
:10D8C0002100200006834000F20F200002016000CA
:10D8D000025B7800C800DE00F20F200002816000C9
:10D8E000025B780086392100210020000683400079
:10D8F000F20F200002016000025B7800C800DE0029
:10D90000F20F200002816000025B7800A63C21003B
:10D910002100200006834000F20F20000201600079
:10D92000025B7800C800DE00F20F20000281600078
:10D93000025B7800C63F21002100200006834000E2
:10D94000F20F200002016000025B7800C800DE00D8
:10D95000F20F200002816000025B7800E6422100A5
:10D960002100200006834000F20F20000201600029
:10D97000025B7800C800DE00F20F20000281600028
:10D98000025B78000646210021002000068340004B
:10D99000F20F200002016000025B7800C800DE0088
:10D9A000F20F200002816000025B7800264921000E
:10D9B0002100200006834000F20F200002016000D9
:10D9C000025B7800C800DE00F20F200002816000D8
:10D9D000025B7800464C21002100200006834000B5
:10D9E000F20F200002016000025B7800C800DE0038
:10D9F000F20F200002816000025B7800664F210078
:10DA00002100200006834000F20F20000201600088
:10DA1000025B7800C800DE00F20F20000281600087
:10DA2000025B78008652210021002000068340001E
:10DA3000F20F200002016000025B7800C800DE00E7
:10DA4000F20F200002816000025B7800A6552100E1
:10DA50002100200006834000F20F20000201600038
:10DA6000025B7800C800DE00F20F20000281600037
:10DA7000025B7800C6582100210020000683400088
:10DA8000F20F200002016000025B7800C800DE0097
:10DA9000F20F200002816000025B7800E65B21004B
:10DAA0002100200006834000F20F200002016000E8
:10DAB000025B7800C800DE00F20F200002816000E7
:10DAC000025B7800065F21002100200006834000F1
:10DAD000F20F200002016000025B7800C800DE0047
:10DAE000F20F200002816000025B780026622100B4
:10DAF0002100200006834000F20F20000201600098
:10DB0000025B7800C800DE00F20F20000281600096
:10DB1000025B78004665210021002000068340005A
:10DB2000F20F200002016000025B7800C800DE00F6
:10DB3000F20F200002816000025B7800666821001D
:10DB40002100200006834000F20F20000201600047
:10DB5000025B7800C800DE00F20F20000281600046
:10DB6000025B7800866B21002100200006834000C4
:10DB7000F20F200002016000025B7800C800DE00A6
:10DB8000F20F200002816000025B7800A66E210087
:10DB90002100200006834000F20F200002016000F7
:10DBA000025B7800C800DE00F20F200002816000F6
:10DBB000025B7800C671210021002000068340002E
:10DBC000F20F200002016000025B7800C800DE0056
:10DBD000F20F200002816000025B7800E6742100F1
:10DBE0002100200006834000F20F200002016000A7
:10DBF000025B7800C800DE00F20F200002816000A6
:10DC0000025B780006782100210020000683400096
:10DC1000F20F200002016000025B7800C800DE0005
:10DC2000F20F200002816000025B7800267B210059
:10DC30002100200006834000F20F20000201600056
:10DC4000025B7800C800DE00F20F20000281600055
:10DC5000025B7800467E2100210020000683400000
:10DC6000F20F200002016000025B7800C800DE00B5
:10DC7000F20F200002816000025B780066812100C3
:10DC80002100200006834000F20F20000201600006
:10DC9000025B7800C800DE00F20F20000281600005
:10DCA000025B78008684210021002000068340006A
:10DCB000F20F200002016000025B7800C800DE0065
:10DCC000F20F200002816000025B7800A68721002D
:10DCD0002100200006834000F20F200002016000B6
:10DCE000025B7800C800DE00F20F200002816000B5
:10DCF000025B7800C68A21002100200006834000D4
:10DD0000F20F200002016000025B7800C800DE0014
:10DD1000F20F200002816000025B78000000060024
:10DD20004200F800801F7800811F7800821F780071
:10DD3000508480000080E80022152100020150007C
:10DD400001003A00E0082100618480008100500059
:10DD50004220AF00BA6E04000000000031118000C4
:10DD60000168A9000108780050848800BE6E040094
:10DD700000000000311180000168A90020818000AE
:10DD80000000D000E2032000020060000006010055
:10DD9000546F040000000000646F040000000000E5
:10DDA0007A6F040000000000906F04000000000083
:10DDB000A66F040000000000BC6F0400000000001B
:10DDC000D26F040000000000E86F040000000000B3
:10DDD000F26F040000000000FE6F0400000000006D
:10DDE000087004000000000014700400000000002F
:10DDF0001E700400000000002A70040000000000F3
:10DE00003E700400000000004870040000000000A4
:10DE100054700400000000005E7004000000000068
:10DE20006A70040000000000707004000000000030
:10DE30007A700400000000008670040000000000FA
:10DE40009A70040000000000A470040000000000AC
:10DE5000BA70040000000000C4700400000000005C
:10DE6000CE70040000000000DA7004000000000022
:10DE7000E470040000000000F070040000000000E6
:10DE8000F6700400000000000071040000000000B3
:10DE90000C7104000000000020710400000000006C
:10DEA0002A71040000000000420220000281680084
:10DEB0004220AE00606F0400000000002430EC003F
:10DEC000407104000000000072042000028168001C
:10DED0004220AE00746F0400000000002430EC000B
:10DEE000766F0400000000002430EF004071040051
:10DEF0000000000002052000028168004220AE0000
:10DF00008A6F0400000000002430EC008C6F0400D5
:10DF1000000000002430EF00407104000000000009
:10DF200072042000028168004220AE00A06F04004D
:10DF3000000000002430EC00A26F0400000000008C
:10DF40002430EF0040710400000000007204200043
:10DF5000028168004220AE00B66F0400000000009D
:10DF60002430EC00B86F0400000000002430EF0003
:10DF700040710400000000001204200002816800CB
:10DF80004220AE00CC6F0400000000002430EC0002
:10DF9000CE6F0400000000002430EF004071040048
:10DFA00000000000C2022000028168004220AE0092
:10DFB000E26F0400000000002430EC00E46F040075
:10DFC000000000002430EF00407104000000000059
:10DFD000C808DD00218088002430EC004071040076
:10DFE00000000000208080008100700021808800F7
:10DFF0002430EC004071040000000000C808DD007F
:10E00000318088002430EC004071040000000000E2
:10E010003080800081007000318088002430EC0066
:10E020004071040000000000C808DD004180880045
:10E030002430EC00407104000000000040808000AB
:10E0400081007000418088002430EC0040710400A1
:10E0500000000000C2022000028168004220AE00E1
:10E060003A700400000000002430EC003A70040014
:10E07000000000004071040000000000C808DD003E
:10E08000518088002430EC00407104000000000042
:10E090005080800081007000518088002430EC00A6
:10E0A0004071040000000000C808DD0061808800A5
:10E0B0002430EC004071040000000000608080000B
:10E0C00081007000618088002430EC004071040001
:10E0D000000000002430EC0040710400000000004B
:10E0E000C808DD00718088002430EC004071040015
:10E0F0000000000070808000810070007180880046
:10E100002430EC004071040000000000C202200036
:10E11000028168004220AE009670040000000000FA
:10E120002430EC00967004000000000040710400F0
:10E1300000000000C808DD00818088002430EC0069
:10E140004071040000000000C2022000028168004B
:10E150004220AE00B4700400000000002430EC0047
:10E16000B6700400000000002430EF00407104008D
:10E1700000000000C808DD00918088002430EC0019
:10E180004071040000000000C808DD00A180880084
:10E190002430EC004071040000000000A0808000EA
:10E1A00081007000A18088002430EC0040710400E0
:10E1B00000000000C808DD00B18088002430EC00B9
:10E1C0004071040000000000B080800081007000F9
:10E1D000B18088002430EC00407104000000000091
:10E1E0002430EC004071040000000000C808DD008D
:10E1F000C18088002430EC00407104000000000061
:10E20000C080800081007000C18088002430EC0054
:10E210004071040000000000C2022000028168007A
:10E220004220AE001C710400000000002430EC000D
:10E230001C71040000000000407104000000000098
:10E24000C808DD00D18088002430EC004071040053
:10E2500000000000C2022000028168004220AE00DF
:10E260003A710400000000002430EF003C7104000B
:10E27000000000002430EF004071040000000000A6
:10E280004F017800CF0078004F0078004200F9007D
:10E29000004006004200F800801F7800811F7800CF
:10E2A000821F780002720200000000004F01780017
:10E2B000CF0078004F0078004200F90000400600CF
:10E2C0002222A9000828A900004006003222A90045
:10E2D0000848A900004006004200F800801F7800AE
:10E2E000811F7800821F7800687202000000000021
:10E2F0004F017800CF0078004F0078004200F9000D
:10E30000004006004200F800801F7800811F78005E
:10E31000821F780034720200000000004F01780074
:10E32000CF0078004F0078004200F900004006005E
:10E330005222A9000A28A90000400600908A800005
:10E34000A08A8800A18A8000010050004220AE000F
:10E350009E7104000000000000000600D1908000C3
:10E36000800878008180E800E227210002815000C7
:10E3700001003A00E1212100D1908800158EA9000A
:10E380002A68A80000000600B18D80008100E80026
:10E39000922121000281500001003A00A11B2100BE
:10E3A000C28D8000028150004220AF00D071040075
:10E3B0000000000080487800B18D880023E8A800A4
:10E3C00000000600A18A8000908A800001005000B1
:10E3D0004200A9004220AF000072040000000000CB
:10E3E0008180E800621B21000281500001003A0098
:10E3F0006115210011007800A18A88004200A80060
:10E4000000000600C18D8000B08D8000010050002A
:10E410004220AF002A720400000000003322AF0047
:10E4200032720400000000001140780034E2B700AE
:10E430008100E800922121000281500001003A0091
:10E44000A11B2100C18D8800956EAA006672040090
:10E45000000000003302AE00327204000000000031
:10E4600023E8A90000000600E1908000D090800021
:10E47000010050004220AF005C7204000000000068
:10E480005322AF0066720400000000001100780003
:10E49000A01288008180E800E2272100028150005C
:10E4A00001003A00E1212100E1908800958EAA0048
:10E4B00066720400000000005302AE0066720400A1
:10E4C000000000002A68A900158EA80000000600C0
:10E4D0002A68AF009072040000000000908A80005B
:10E4E0000080E800621B21000201500001003A0098
:10E4F00060152100A18A8000810050004220AF00F9
:10E500009072040000000000B11280000A48A900C7
:10E5100001087800908A88009472040000000000CE
:10E52000B11280000A48A9000000060000000000A7
:10E5300000000000000000000000000096720400CF
:10E5400000000000000000000000000000000000CB
:10E5500000000000A27204000000000000000000A3
:10E56000000000000000000000000000AE72040087
:10E57000000000000000000000000000000000009B
:10E5800000000000BA72040000000000000000005B
:10E59000000000000000000000000000C67204003F
:10E5A000000000000000000000000000000000006B
:10E5B00000000000D2720400000000000000000013
:10E5C000000000000000000000000000DE720400F7
:10E5D000000000000000000000000000000000003B
:10E5E00000000000EA7204000000000000000000CB
:10E5F000000000000000000000000000F6720400AF
:10E60000000000000000000000000000000000000A
:10E61000000000000002040000000000801F7800DD
:10E62000811F7800821F7800831F7800841F780084
:10E63000851F7800861F7800881F7800891F780062
:10E640008A1F78008181800092818000A3818000F0
:10E65000B4818000C5818000D68180000004EB0079
:10E660008004EB000005EB00040CB80088818800F2
:10E67000998188003430EF000414B8000800780055
:10E680003230B4000900780034B0B400041CB80083
:10E69000080078003430B400050CB8000800780099
:10E6A0003230B4000900780034B0B4000514B8006A
:10E6B000080078003430B400060CB8000800780078
:10E6C0003430B4004F057800CF0478004F04780050
:10E6D0004F037800CF0278004F027800CF01780016
:10E6E0004F017800CF0078004F007800000006004E
:10E6F000801F7800811F7800821F7800841F7800B7
:10E70000851F7800861F7800881F7800891F780091
:10E710008A1F7800000320007081880080818000BB
:10E7200091818000A2818000B4818000C581800039
:10E73000D68180000004EB008004EB000005EB00B4
:10E740004200A9002C10AF004200A8000080D200B7
:10E750008180D2000281D2000884D2008984D20054
:10E760000A85D2000404540085845C0006055D001F
:10E770002C10A9004200AF002C10A80003003100AB
:10E780000404440085844C0006054D002E30ED0045
:10E790002E10E2004220AE00A07304000000000032
:10E7A0004200A9002C10AF004200A8000080D20057
:10E7B0008180D2000281D20080818800918188000E
:10E7C000A28188004F057800CF0478004F047800BC
:10E7D0004F037800CF0278004F0278004F01780095
:10E7E000CF0078004F00780000000600000006000F
:10E7F000801F7800B08180003030B400C08180007C
:10E8000032B0B400D081800034B0B4004F00780042
:10E8100000000600801F7800B08180003030B50015
:10E82000C081800032B0B500D081800034B0B50026
:10E830004F00780000000600000006001000A10054
:10E84000B00720004074020000000000F093800038
:10E850004074020000000000C0022000407402006A
:10E860000000000016007800407402000000000064
:10E87000D0072000407402000000000000000600E5
:10E8800071C78000800878008180E800A2EC210038
:10E890000281500001003A00218F210071C78800D9
:10E8A000ECB8EC000000060081C780001100780081
:10E8B0008180E800A2EC21000281500001003A00B2
:10E8C000218F210081C788000000060005EEA80006
:10E8D000801F7800811F7800821F7800831F7800D6
:10E8E000841F7800851F7800861F78006A30EC004E
:10E8F0008430ED008410E2004220AE00AE740400CB
:10E9000000000000803E200020848800AE740400D7
:10E910000000000003022000E2292100030078002B
:10E920000000E900210320000100B80000014100BF
:10E930001260A600A4740400000000000003200080
:10E94000000141001200A0008301E9000300E00083
:10E950004220AE008C74040000000000F0C680006D
:10E960000000D000E101200001006000000601006D
:10E97000F8740400000000000A75040000000000A4
:10E980002E75040000000000527504000000000015
:10E990007C75040000000000F87404000000000012
:10E9A000F874040000000000F87404000000000087
:10E9B000F874040000000000F87404000000000077
:10E9C000F874040000000000F87404000000000067
:10E9D000F874040000000000F87404000000000057
:10E9E000F874040000000000F87404000000000047
:10E9F000E038EF00E2B8EF00850EA800852EA900F0
:10EA0000854EA900856EA900DE38EC003E76040034
:10EA10000000000000C78000838EAE0010C7880091
:10EA20000000E80083AEAE0010C788000000E800D8
:10EA300083CEAE0010C788000000E80000C7880041
:10EA4000850EA900852EA800854EA900856EA90017
:10EA5000DE38EC003E7604000000000000C78000B5
:10EA6000838EAE0010C788000000E80083AEAE00C1
:10EA700010C788000000E80083CEAE0010C78800F1
:10EA80000000E80000C78800850EA900852EA900B7
:10EA9000854EA800856EA900DE38EC003E760400A5
:10EAA0000000000000C78000838EAE0010C7880001
:10EAB0000000E80083AEAE0010C788000000E80048
:10EAC00083CEAE0010C788000000E80000C78800B1
:10EAD000850EA90000000000852EA900000000009E
:10EAE000854EA90000000000856EA800DE38EC000D
:10EAF0003E7604000000000000C78000838EAE0058
:10EB000010C788000000E800DE38EF0010C7800062
:10EB100031C78000010150004220AF009C75040005
:10EB20000000000030C78800A000200020C7880037
:10EB30003E76040000000000E418E2004220AF002E
:10EB40003A76040000000000E438ED00E418E2002A
:10EB50004220AE003A760400000000004200DD00D2
:10EB6000C103200001006000000601002000200019
:10EB700040C788003A760400000000001000200022
:10EB800040C788003A760400000000000000200022
:10EB900040C788003A7604000000000030002000E2
:10EBA00040C788003A7604000000000040002000C2
:10EBB00040C788003A7604000000000050002000A2
:10EBC00040C788003A760400000000008000200062
:10EBD00040C788003A760400000000007000200062
:10EBE00040C788003A760400000000006000200062
:10EBF00040C788003A760400000000009000200022
:10EC000040C788003A7604000000000000000000C1
:10EC100000000000000000000000000000000000F4
:10EC200000000000000000000000000000000000E4
:10EC300000000000000000000000000000000000D4
:10EC400000000000000000000000000000000000C4
:10EC500000000000000000000000000000000000B4
:10EC6000000000000000000000000000F0FF2F0086
:10EC700040C788003E760400000000006610E200F5
:10EC80004220AE006630ED0010818000B10020000F
:10EC9000010050004220AF005A760400000000003E
:10ECA0000230A9008038210050C788006A7604002D
:10ECB00000000000EA38ED00EA18E2004220AE0051
:10ECC0006A760400000000008038210050C78800E8
:10ECD0000230A800109480000000D000E103200062
:10ECE00001006000000601000C7704000000000035
:10ECF0001877040000000000767704000000000090
:10ED0000DC7704000000000012780400000000001E
:10ED100048780400000000009E7804000000000015
:10ED2000B8780400000000002C7904000000000006
:10ED300062790400000000009A79040000000000DD
:10ED4000DC79040000000000387A040000000000B4
:10ED5000567A040000000000A87A040000000000B9
:10ED6000127B040000000000487B0400000000004B
:10ED70007E7B040000000000D47B04000000000043
:10ED80000C770400000000000C7704000000000075
:10ED90000C770400000000000C7704000000000065
:10EDA0000C770400000000000C7704000000000055
:10EDB0000C770400000000000C7704000000000045
:10EDC0000C770400000000000C7704000000000035
:10EDD0000C770400000000000C7704000000000025
:10EDE0000C770400000000000C7704000000000015
:10EDF0000C770400000000000C7704000000000005
:10EE00000C770400000000000C77040000000000F4
:10EE10000C7704000000000084B2EF0090B2EF0015
:10EE20001000200010948800F27B04000000000015
:10EE3000030220008432EC002094800001022000B4
:10EE4000010050004200AE003277040000000000D4
:10EE500084B2EF00D0002000109488007277040084
:10EE600000000000E22921002094800021032000FE
:10EE70000100B8000001410032948800124078007F
:10EE8000F1002000010060004220AF006077040024
:10EE9000000000001260A60060770400000000007F
:10EEA0001240A70060770400000000001250A0008C
:10EEB00020002000109488007277040000000000F9
:10EEC0008301E9000300E0004220AE001A7704004D
:10EED00000000000D0002000109488007277040029
:10EEE00000000000F27B0400000000003694800067
:10EEF0009E71020000000000209480000000E800E5
:10EF00000110200001007000AE710200000000003E
:10EF10000002EB00564078004400DE00F1002000C3
:10EF2000010060008002780004024000AE7102001F
:10EF3000000000008502E8001000200004024000EC
:10EF4000AE7102000000000000002000040240003A
:10EF5000AE71020000000000369480002001200005
:10EF6000000343003640780004024000AE71020006
:10EF7000000000008502E9000500E0004220AE002C
:10EF8000B2770400000000000480EA00F10F2000C6
:10EF900001006000AE7102000000000036948000A5
:10EFA0002003200050948800300020001094880036
:10EFB000F27B040000000000E2710200000000008B
:10EFC0004200AF00FC770400000000008A12E2005B
:10EFD0004220AF008A780400000000008A32ED0071
:10EFE0008A12E2004220AE000E7804000000000009
:10EFF0008A780400000000000110200081006800F1
:10F000004220AE008A78040000000000400020008A
:10F01000109488000E780400000000009A78040024
:10F0200000000000E2710200000000004200AF009A
:10F0300032780400000000008A12E2004220AF0093
:10F040008A780400000000008A32ED008A12E20093
:10F050004220AE0044780400000000008A780400DA
:10F060000000000011002000810068004220AE0076
:10F070008A780400000000005000200010948800EE
:10F0800044780400000000009A78040000000000AA
:10F09000E2710200000000004200AF006878040046
:10F0A000000000008A12E2004220AF008A780400CB
:10F0B000000000008A32ED008A12E2004220AE0019
:10F0C00076780400000000008A7804000000000048
:10F0D000E10F2000810068004220AE008A78040021
:10F0E000000000007A780400000000009A78040014
:10F0F00000000000369480001664A000A0002000EC
:10F100005094880060002000109488009A780400D1
:10F1100000000000369480001664A100A0002000CA
:10F1200050948800C0002000109488009A78040051
:10F1300000000000F27B0400000000008A12E200E0
:10F140004220AF00B0780400000000008A32ED00D9
:10F150008A12E2004220AE00B478040000000000F1
:10F160007000200010948800F27B04000000000072
:10F17000369480009E710200000000002094800000
:10F180000000E8000110200001007000AE710200D4
:10F19000000000002630EF0056407800F10020000B
:10F1A0000100600001848000229480000208E100D8
:10F1B0004220AE00E2780400000000004100200080
:10F1C00001004000609488000104200001007000EC
:10F1D000318180008100400031818800AE710200E1
:10F1E000000000008C32EC00100020003181800013
:10F1F0008100400031818800AE71020000000000F3
:10F2000000012000318180008100400031818800B0
:10F21000AE71020000000000308180000080EA0032
:10F22000F10F200001006000AE710200000000003C
:10F23000369480002002200000034300469488009A
:10F240002003200050948800800020001094880043
:10F25000F27B040000000000E271020000000000E8
:10F260004200AF004C790400000000008A12E20066
:10F270004220AF00247A0400000000008A32ED0032
:10F280008A12E2004220AE005E7904000000000015
:10F29000247A0400000000000110200081006800B2
:10F2A0004220AE00247A04000000000090002000FC
:10F2B000109488005E79040000000000347A040095
:10F2C00000000000E2710200000000004200AF00F8
:10F2D00082790400000000008A12E2004220AF00A0
:10F2E000247A0400000000008A32ED008A12E20055
:10F2F0004220AE009679040000000000247A040049
:10F300000000000011002000810068004220AE00D3
:10F31000247A04000000000070948800A0002000FF
:10F32000109488009679040000000000347A0400EC
:10F3300000000000E2710200000000004200AF0087
:10F34000BA790400000000008A12E2004220AF00F7
:10F35000247A0400000000008A32ED008A12E200E4
:10F360004220AE00D879040000000000247A040096
:10F370000000000046948000005B780046948800FE
:10F380007194800081004000719488008C32ED00FF
:10F390008C12E2004220AE00D87904000000000088
:10F3A000B000200010948800D8790400000000000C
:10F3B000347A040000000000E27102000000000046
:10F3C0004200AF00FC790400000000008A12E20055
:10F3D0004220AF00247A0400000000008A32ED00D1
:10F3E0008A12E2004220AE00107A04000000000001
:10F3F000247A040000000000719480008180EA00FB
:10F40000F20F200082806000810050004220AE0098
:10F41000247A040000000000147A040000000000B8
:10F42000347A040000000000369480001664A000C6
:10F43000A000200050948800C00020001094880094
:10F44000347A040000000000369480001664A100A5
:10F45000A000200050948800C00020001094880074
:10F46000347A040000000000F27B04000000000079
:10F470008A12E2004220AF004A7A04000000000035
:10F480008A32ED008A12E2004220AE00527A040075
:10F4900000000000329480001250A10010002000F3
:10F4A00010948800F27B040000000000030220009A
:10F4B0009032EC0080948000010220000100500096
:10F4C0004200AF009032EF00E229210080948000DA
:10F4D000210320000100B80000014100329488009F
:10F4E00012407800F1002000010060004220AF00CF
:10F4F000927A0400000000001260A700927A0400D3
:10F50000000000001240A700927A040000000000F2
:10F510001250A000E000200010948800A47A04009B
:10F52000000000008301E9000300E0004220AE007B
:10F53000587A040000000000100020001094880099
:10F54000A47A040000000000F27B04000000000028
:10F55000369480009E7102000000000080948000BC
:10F560000000E8000110200001007000AE710200F0
:10F57000000000003000200000027800AE710200A0
:10F58000000000001000200004024000AE710200E4
:10F59000000000000000200004024000AE710200E4
:10F5A0000000000040838000F10F20000100600097
:10F5B00004024000AE7102000000000040838000A1
:10F5C0004800DE00F10F200001006000040240004E
:10F5D000AE71020000000000100020000402400094
:10F5E000AE7102000000000040062000040240004E
:10F5F000AE710200000000000480EA00F10F20005C
:10F6000001006000AE710200000000002003200035
:10F6100050948800F000200010948800F27B0400D1
:10F6200000000000E2710200000000004200AF0094
:10F63000327B0400000000008A12E2004220AF008A
:10F64000C07B0400000000008A32ED008A12E20054
:10F650004220AE00447B040000000000C07B040098
:10F660000000000001102000810068004220AE0070
:10F67000C07B0400000000000001200010948800FE
:10F68000447B040000000000D07B04000000000068
:10F69000E2710200000000004200AF00687B04003D
:10F6A000000000008A12E2004220AF00C07B04008C
:10F6B000000000008A32ED008A12E2004220AE0013
:10F6C0007A7B040000000000C07B04000000000002
:10F6D00011002000810068004220AE00C07B0400C1
:10F6E0000000000010012000109488007A7B0400C4
:10F6F00000000000D07B040000000000E271020066
:10F70000000000004200AF009E7B040000000000EB
:10F710008A12E2004220AF00C07B0400000000001B
:10F720008A32ED008A12E2004220AE00AC7B040077
:10F7300000000000C07B040000000000E10F20007A
:10F74000810068004220AE00C07B04000000000081
:10F75000B07B040000000000D07B0400000000002B
:10F76000369480001664A000A00020005094880009
:10F770002001200010948800D07B040000000000CD
:10F78000369480001664A100A000200050948800E8
:10F790002001200010948800D07B040000000000AD
:10F7A000F27B0400000000008A12E2004220AF0059
:10F7B000E67B0400000000008A32ED008A12E200BD
:10F7C0004220AE00EE7B0400000000003294800076
:10F7D0001250A1001000200010948800F27B040059
:10F7E000000000004F037800CF0278004F0278003D
:10F7F000CF0178004F017800CF0078004F007800EB
:10F8000005EEA90000E8A90000400600A0948000D1
:10F810004300DE0000007800156EA9000000000023
:10F8200000000000000000000000000000000000D8
:10F83000000000000000000010082000E660020048
:10F8400000000000A4948000F30720000300620081
:10F85000E660020000000000949480004822DE0070
:10F8600003006200E6600200000000009494800043
:10F87000F30F200003006200E660020000000000B9
:10F88000156EA8000000000000000000000000004D
:10F890000000000000000000000000000000000068
:10F8A0008662020000000000866202000000000084
:10F8B0008662020000000000866202000000000074
:10F8C00000000600A09480004300DE0000007800E5
:10F8D000156EA900000000000000000000000000FC
:10F8E0000000000000000000000000000000000018
:10F8F00080082000E660020000000000A494800060
:10F90000F307200003006200E66002000000000030
:10F91000949480004822DE0003006200E66002004A
:10F920000000000094948000F30F200003006200A8
:10F93000E660020000000000156EA8000000000054
:10F9400000000000000000000000000000000000B7
:10F9500000000000000000008662020000000000BD
:10F960000000060015EEA90015CEA90015AEA900ED
:10F970000000000000000000000000000000000087
:10F98000000000000000000000000000156EA9004B
:10F990000000000000000000000000000000000067
:10F9A000000000000000000000000000800E2000A9
:10F9B000E66002000000000000002000E660020097
:10F9C0000000000000002000E660020000000000CF
:10F9D00000002000E660020000000000000020009F
:10F9E000E66002000000000000002000E660020067
:10F9F0000000000000002000E6600200000000009F
:10FA000000002000E6600200000000003A610200F1
:10FA100000000000156EA8000000000000000000BB
:10FA200000000000000000000000000000000000D6
:10FA300000000000A10A20000100E1004220AE0009
:10FA4000287D040000000000D27F040000000000B8
:10FA50008662020000000000156EA9000000000090
:10FA60000000000000000000000000000000000096
:10FA7000000000000000000010082000E660020006
:10FA80000000000000002000E6600200000000000E
:10FA900010002000E66002000000000000002000CE
:10FAA000E660020000000000156EA80000000000E3
:10FAB0000000000000000000000000000000000046
:10FAC000000000000000000086620200000000004C
:10FAD0008662020000000000866202000000000052
:10FAE0008662020000000000156EA9000000000000
:10FAF0000000000000000000000000000000000006
:10FB0000000000000000000040082000E660020045
:10FB10000000000000002000E6600200000000007D
:10FB200010002000E660020000000000000020003D
:10FB3000E660020000000000F4808000F30F200067
:10FB400003006200E6600200000000004822DE00C0
:10FB500003006200E66002000000000004818000F3
:10FB6000F30F200003006200E660020000000000C6
:10FB70004822DE0003006200E66002000000000090
:10FB800064838000F30F200003006200E66002003F
:10FB9000000000004822DE0003006200E660020070
:10FBA0000000000074838000F30F20000300620057
:10FBB000E6600200000000004822DE000300620050
:10FBC000E66002000000000084838000F30F200044
:10FBD00003006200E6600200000000004822DE0030
:10FBE00003006200E66002000000000094838000D1
:10FBF000F30F200003006200E66002000000000036
:10FC00004822DE0003006200E660020000000000FF
:10FC1000A4838000F30F200003006200E66002006E
:10FC2000000000004822DE0003006200E6600200DF
:10FC300000000000B4838000F30F20000300620086
:10FC4000E6600200000000004822DE0003006200BF
:10FC5000E660020000000000C4838000F30F200073
:10FC600003006200E6600200000000004822DE009F
:10FC700003006200E660020000000000E4808000F3
:10FC8000F30F200003006200E660020000000000A5
:10FC90004822DE0003006200E6600200000000006F
:10FCA000E4838000F30F200003006200E66002009E
:10FCB000000000004822DE0003006200E66002004F
:10FCC00000000000F4838000F30F200003006200B6
:10FCD000E6600200000000004822DE00030062002F
:10FCE000E66002000000000004848000F30F2000A2
:10FCF00003006200E6600200000000004822DE000F
:10FD000003006200E660020000000000949480009E
:10FD1000F30F200003006200E66002000000000014
:10FD20004822DE0003006200E660020000000000DE
:10FD3000A4948000F30F200003006200E66002003C
:10FD4000000000004822DE0003006200E6600200BE
:10FD500000000000000000000000000000000000A3
:10FD6000156EA80000000000000000000000000068
:10FD70000000000000000000000000000000000083
:10FD80008662020000000000156EA900000000005D
:10FD90000000000000000000000000000000000063
:10FDA000000000000000000080082000E660020063
:10FDB0000000000000002000E660020000000000DB
:10FDC00010002000E660020000000000000020009B
:10FDD000E660020000000000156EA80000000000B0
:10FDE0000000000000000000000000000000000013
:10FDF0000000000000000000866202000000000019
:10FE0000866202000000000086620200000000001E
:10FE10008662020000000000156EA90000000000CC
:10FE200000000000000000000000000000000000D2
:10FE3000000000000000000010082000E660020042
:10FE40000000000000002000E6600200000000004A
:10FE500000002000E660020000000000000020001A
:10FE6000E660020000000000156EA800000000001F
:10FE70000000000000000000000000000000000082
:10FE80000000000000000000866202000000000088
:10FE9000866202000000000086620200000000008E
:10FEA0008662020000000000156EA900000000003C
:10FEB0000000000000000000000000000000000042
:10FEC000000000000000000040082000E660020082
:10FED0000000000000002000E660020000000000BA
:10FEE00000002000E660020000000000000020008A
:10FEF000E660020000000000A00A2000E6600200A8
:10FF000000000000156EA8000000000000000000C6
:10FF100000000000000000000000000000000000E1
:10FF2000000000008662020000000000156EA900BB
:10FF300000000000000000000000000000000000C1
:10FF40000000000000000000000000008008200009
:10FF5000E66002000000000000002000E6600200F1
:10FF60000000000000002000E66002000000000029
:10FF700000002000E660020000000000156EA800EE
:10FF80000000000000000000000000000000000071
:10FF90000000000000000000000000007C8204005F
:10FFA000000000008662020000000000156EA9003B
:10FFB0000000000000000000000000000000000041
:10FFC00000000000000000000000000010082000F9
:10FFD000E66002000000000000002000E660020071
:10FFE0000000000000002000E660020000000000A9
:10FFF00000082000E660020000000000156EA80066
:020000040001F9
:1000000000000000000000000000000000000000F0
:1000100000000000000000000000000086620200F6
:1000200000000000866202000000000086620200FC
:10003000000000008662020000000000156EA900AA
:1000400000000000000000000000000000000000B0
:100050000000000000000000000000004008200038
:10006000E66002000000000000002000E6600200E0
:100070000000000000002000E66002000000000018
:1000800000082000E660020000000000F48080000C
:10009000F30F200003006200E66002000000000091
:1000A0004822DE0003006200E6600200000000005B
:1000B00004818000F30F200003006200E66002006C
:1000C000000000004822DE0003006200E66002003B
:1000D0000000000064838000F30F20000300620032
:1000E000E6600200000000004822DE00030062001B
:1000F000E66002000000000074838000F30F20001F
:1001000003006200E6600200000000004822DE00FA
:1001100003006200E66002000000000084838000AB
:10012000F30F200003006200E66002000000000000
:100130004822DE0003006200E660020000000000CA
:1001400094838000F30F200003006200E660020049
:10015000000000004822DE0003006200E6600200AA
:1001600000000000A4838000F30F20000300620061
:10017000E6600200000000004822DE00030062008A
:10018000E660020000000000B4838000F30F20004E
:1001900003006200E6600200000000004822DE006A
:1001A00003006200E660020000000000C4838000DB
:1001B000F30F200003006200E66002000000000070
:1001C0004822DE0003006200E6600200000000003A
:1001D000E4808000F30F200003006200E66002006C
:1001E000000000004822DE0003006200E66002001A
:1001F00000000000E4838000F30F20000300620091
:10020000E6600200000000004822DE0003006200F9
:10021000E660020000000000F4838000F30F20007D
:1002200003006200E6600200000000004822DE00D9
:1002300003006200E6600200000000000484800009
:10024000F30F200003006200E660020000000000DF
:100250004822DE0003006200E660020000000000A9
:1002600094948000F30F200003006200E660020017
:10027000000000004822DE0003006200E660020089
:1002800000000000A4948000F30F2000030062002F
:10029000E6600200000000004822DE000300620069
:1002A000E660020000000000000000000000000006
:1002B00000000000156EA800000000000000000013
:1002C000000000000000000000000000000000002E
:1002D000000000008662020000000000156EA90008
:1002E000000000000000000000000000000000000E
:1002F0000000000000000000000000008008200056
:10030000E66002000000000000002000E66002003D
:100310000000000000002000E66002000000000075
:1003200000082000E660020000000000156EA80032
:1003300000000000000000000000000000000000BD
:1003400000000000000000000000000086620200C3
:1003500000000000866202000000000086620200C9
:10036000000000008662020000000000156EA90077
:10037000000000000000000000000000000000007D
:100380000000000000000000000000001008200035
:10039000E66002000000000000002000E6600200AD
:1003A0000000000000002000E660020000000000E5
:1003B00000002000E660020000000000156EA800AA
:1003C000000000000000000000000000000000002D
:1003D0000000000000000000000000008662020033
:1003E0000000000086620200000000008662020039
:1003F000000000008662020000000000156EA900E7
:1004000000000000000000000000000000000000EC
:100410000000000000000000000000004008200074
:10042000E66002000000000000002000E66002001C
:100430000000000000002000E66002000000000054
:1004400000002000E66002000000000050052000CF
:10045000E660020000000000156EA8000000000029
:10046000000000000000000000000000000000008C
:100470000000000000000000866202000000000092
:10048000156EA90000000000000000000000000040
:10049000000000000000000000000000000000005C
:1004A00080082000E660020000000000000020003C
:1004B000E66002000000000000002000E66002008C
:1004C0000000000000002000E660020000000000C4
:1004D000156EA800000000000000000000000000F1
:1004E000000000000000000000000000000000000C
:1004F0007C8204000000000000000600801F7800DD
:100500004400DE00F1002000010060009E82020035
:1005100000000000C4710200000000004F007800DD
:10052000F1002000010060009E8202000000000037
:10053000C47102000000000000000600A1002000BD
:1005400081005000010320004200AF007103200031
:100550000100400000000600F09380000000E80069
:1005600080818800B66B020000000000C08280001D
:100570000103200001004000FE62020000000000B4
:10058000D08280000103200001004000FE620200D2
:1005900000000000A0032000FE6202000000000036
:1005A00000022000FE6202000000000000000600C1
:1005B0000200000003000000050000000A00000027
:1005C00000100000920F00008000000000000000FA
:1005D000FFFFFF00FFFFFF00FFFFFF00FFFFFF0027
:1005E000FFFFFF00FFFFFF00FFFFFF00FFFFFF0017
:1005F000FFFFFF00FFFFFF00FFFFFF00FFFFFF0007
:10060000FFFFFF00FFFFFF00FFFFFF00FFFFFF00F6
:0200000400FFFB
:0200000401F009
:100008000300000083000000250000007F000000BE
:0C00180037000000D500000003000000CD
:04002400FF000000D9
:00000001FF
